:100000000C949B1A0C94CC1A0C94CC1A0C94CC1A09
:100010000C94CC1A0C94CC1A0C94CC1A0C94CC1AC8
:100020000C94CC1A0C94CC1A0C94CC1A0C94CC1AB8
:100030000C94CC1A0C94CC1A0C94CC1A0C94CC1AA8
:100040000C94CC1A0C9410DA0C94CC1A0C94CC1A94
:100050000C94CC1A0C94CC1A0C942EC10C94CEACEB
:100060000C94CC1A0C945A560C9450560C94CC1AEE
:100070000C94CC1A0C94CC1A0C94CC1A0C94CC1A68
:100080000C943B340C94CC1A0C94CC1A0C94CC1ACF
:100090000C94CC1A0C94CC1A0C94CC1A0C94CC1A48
:1000A0000C94CC1A0C94CC1A0C940D340C94CC1ADD
:1000B0000C94CC1A0C94CC1A0C94CC1A0C94CC1A28
:1000C0000C94CC1A0C94CC1A0C94CC1A0C94563771
:1000D0000C9420370C94CC1A0C94CC1A0C94CC1A97
:1000E0000C94CC1A084AD73B3BCE016E84BCBFFDB2
:1000F000C12F3D6C74319ABD56833DDA3D00C77FF8
:1001000011BED9E4BB4C3E916BAAAABE0000008090
:100110003F05A84CCDB2D44EB93836A9020C50B91F
:10012000918688083CA6AAAA2ABE000000803F004B
:100130000C9498560C94EC370C9417A90C9472A854
:100140000C942FA80D9417240D94B1120C94E1ABCC
:100150000C9460A80C9480A80C9476A80C940DA91B
:100160000D94800C0D94650E0C945AA80C9486A9DD
:100170000C94D2370D94F60E0D941F0F0C9400388A
:100180000C9445A90D942F0E0C944FA90C94F8379C
:100190000C9490A90D94B9020C9408A60C945042AA
:1001A0000D943A0B0C94C5AA0C94B4AB0D94E513C2
:1001B0000D94E3120C941A380C944DA80C9410452D
:1001C0000D94A8120D94E9040C94E1370C94F456A4
:1001D0000D94BF040C9433A90C94D6560C947CA8AF
:1001E0000C9407380C94F0560C942BA90C946B4487
:1001F0000D949F0D0C9464A80D94F6130D94811228
:100200000C9400AA0C949AA90C9416570C9404AC64
:100210000C9459A90C9408A90C9404570C94D84434
:100220000D945D0F0D94D30E0D9435240D94CF0CC9
:100230000C946EA80C9421A90C947CAA0C9445A84B
:100240000C9450A80C941DAA0C9412380D94B91457
:100250000C9424AB0D94A0080D94CA120C9468A8B9
:100260000C9449A80C9409AB0C9497440D94041376
:100270000C9485A50D94AE120C9468A90D94030DF1
:100280000C94EC560C9494370D9499170C94A2ABE3
:100290000C949F420C94F0370C941E570C94C75644
:1002A0000C9472A90C94F4370C942AA80C94F85668
:1002B0000D94D9120D943E0F0C94E8370C9400A9BC
:1002C0000C9407A60C94FC370C9400570D947410F2
:1002D0000C9441A80C94E5560D94B30C0D94B10FF9
:1002E0000D946F0F0C94C3370C9456A80C94A34232
:1002F0000D94DA030C94FC560D94C40F0C940B5718
:100300000D94F7120C947CA90D9451060D942207BC
:100310000C943BA94E414E494E495459494E46CD45
:10032000CCCC3D0AD7233C17B7D13877CC2B3295AC
:1003300095E6241FB14F0A000020410000C842008A
:10034000401C4620BCBE4CCA1B0E5AAEC59D740054
:10035000407A10F35A00A0724E18090010A5D4E894
:100360000000E87648170000E40B54020000CA9A27
:100370003B000000E1F50500008096980000004079
:10038000420F000000A086010000001027000000BE
:1003900000E803000000006400000000000A000004
:1003A0000000000100000000002C76D888DC674FB8
:1003B0000823DFC1DFAE59E1B1B796E5E3E453C6E8
:1003C0003AE651997696E8E6C28426EB898C9B62E0
:1003D000ED407C6FFCEFBC9C9F40F2BAA56FA5F48A
:1003E00090055A2AF75C936B6CF9676DC11BFCE0B2
:1003F000E40D47FEF520E6B500D0ED902E03009405
:100400003577050080841E080000204E0A00000099
:10041000C80C333333330F986E12831141EF8D21A3
:1004200014893BE65516CFFEE6DB18D1844B381B0A
:10043000F77C1D901DA4BBE424203284725E2281CF
:1004400000C9F124ECA1E53D27434F4D4D554E49E0
:10045000434154494F4E0044525952554E00455263
:10046000524F525300494E464F004543484F0045B6
:1004700072726F722077726974696E6720746F2070
:10048000454550524F4D210A0053544F505045445A
:100490002E20005072696E7465722073746F7070D4
:1004A00065642064756520746F206572726F727365
:1004B0002E2046697820746865206572726F7220FC
:1004C000616E6420757365204D39393920746F2051
:1004D000726573746172742E202854656D70657234
:1004E00061747572652069732072657365742E205E
:1004F0005365742069742061667465722072657337
:1005000074617274696E67290A004E6F20436865D2
:10051000636B73756D2077697468206C696E6520F4
:100520006E756D6265722C204C617374204C696E1F
:10053000653A20004E6F20436865636B73756D20CC
:1005400077697468206C696E65206E756D6265727E
:100550002C204C617374204C696E653A20006368EE
:1005600065636B73756D206D69736D617463682C61
:10057000204C617374204C696E653A20004C696EA2
:1005800065204E756D626572206973206E6F7420F0
:100590004C617374204C696E65204E756D62657296
:1005A0002B312C204C617374204C696E653A20000D
:1005B0004D3131300053657269616C207374617420
:1005C0007573206D69736D617463680A0077616982
:1005D000740A0053442072656164206572726F7200
:1005E0000A002121204B494C4C20636175736564DE
:1005F00020627920746F6F206D75636820696E6169
:1006000063746976652074696D65202D2063757249
:1006100072656E7420636F6D6D616E643A20004880
:100620006F74656E642049646C652054696D656FF4
:10063000757400486F74656E642049646C6520545D
:10064000696D656F75740A003D3D6F6E46696C613A
:100650006D656E7452756E6F75743D3D0070617599
:100660007365004D363030002066696C616D656ED3
:10067000745F72756E6F7574200066696C616D656C
:100680006E745F72756E6F757420540046696C618C
:100690006D656E7452756E6F75742054002A2A2A27
:1006A000496E6974696E67206361726420697320A2
:1006B0004F4B2A2A2A004D6564696120496E736593
:1006C00072746564004D656469612052656D6F7672
:1006D0006564004D313030305300627573793A20D3
:1006E00070617573656420666F7220696E707574D1
:1006F0000A00627573793A207061757365642066CB
:100700006F7220757365720A00627573793A207092
:10071000726F63657373696E670A002A2A2A6B69B0
:100720006C6C2A2A2A00706F7765726F6666004BC0
:10073000494C4C45442E20005072696E74657220FD
:1007400068616C7465642E206B696C6C2829206369
:10075000616C6C6564210A0053544F505045442E1F
:1007600020005072696E7465722073746F707065CA
:10077000642064756520746F206572726F72732EC9
:100780002046697820746865206572726F722061F6
:100790006E6420757365204D39393920746F20726D
:1007A0006573746172742E202854656D7065726172
:1007B000747572652069732072657365742E205399
:1007C0006574206974206166746572207265737443
:1007D000617274696E67290A006563686F3A004543
:1007E00072726F723A0042696C696E656172204C78
:1007F0006576656C696E6720477269643A0A002104
:10080000212053544F502063616C6C6564206265F5
:100810006361757365206F6620424C546F75636821
:10082000206572726F72202D20726573746172740C
:100830002077697468204D3939390A002121205305
:10084000544F502063616C6C656420626563617510
:100850007365206F6620424C546F75636820657223
:10086000726F72202D2072657374617274207769C3
:100870007468204D3939390A002F2F616374696F0C
:100880006E3A0070726F6D70745F00656E64005335
:10089000656E64204D31303820746F207265737539
:1008A0006D650A00496E736572742066696C616DCE
:1008B000656E7420616E642073656E64204D313006
:1008C000380A005265686561742066696E697368EC
:1008D00065642E0052656865617420446F6E650022
:1008E000526568656174696E672E2E2E00526568C8
:1008F000656174004865617465722054696D656F47
:1009000075740053656E64204D31303820746F204B
:1009100068656174206E6F7A7A6C650A004E6F7A32
:100920007A6C65205061726B656400486F74656E07
:100930006420746F6F20636F6C640A00706175735C
:1009400065640050617573650044697361626C652C
:1009500052756E6F75740050757267654D6F726574
:10096000005061757365640073686F770062757419
:10097000746F6E00626567696E004C6F616420463B
:10098000696C616D656E74004C6F61642046696CC2
:10099000616D656E74205400496E736572742066D3
:1009A000696C616D656E7420616E642073656E6440
:1009B000204D3130380A00726573756D65640052E0
:1009C0006573756D696E670057616974696E67203C
:1009D000666F72206865617475702E0A004C6561DF
:1009E00076696E6720473236003F537065636966EB
:1009F00069656420582C5920636F6F7264696E6159
:100A00007465206F7574206F6620626F756E6473F5
:100A10002E0A003F28522965706561742076616C4A
:100A20007565206E6F7420706C61757369626C659A
:100A30003B206D757374206265206174206C656164
:100A4000737420312E0A003F285229657065617445
:100A5000206D7573742062652073706563696669C3
:100A60006564207768656E206E6F74207573696E9B
:100A70006720616E204C43442E0A003F537065632B
:100A80006966696564206E6F7A7A6C652074656D3D
:100A90007065726174757265206E6F7420706C6120
:100AA000757369626C652E0A003F537065636966F1
:100AB0006965642066696C616D656E742073697A1E
:100AC00065206E6F7420706C61757369626C652E41
:100AD0000A003F53706563696669656420707269D6
:100AE0006D65206C656E677468206E6F7420706C25
:100AF00061757369626C652E0A003F5072696D659D
:100B0000206C656E677468206D7573742062652053
:100B1000737065636966696564207768656E206EC9
:100B20006F74207573696E6720616E204C43442E8C
:100B30000A003F537065636966696564206E6F7A69
:100B40007A6C652073697A65206E6F7420706C61B1
:100B5000757369626C652E0A003F52657472616339
:100B600074696F6E204D756C7469706C6965722064
:100B70006D7573742062652073706563696669655D
:100B8000642E0A003F53706563696669656420528C
:100B9000657472616374696F6E204D756C746970F1
:100BA0006C696572206E6F7420706C617573696218
:100BB0006C652E0A003F5370656369666965642041
:100BC0006C6179657220686569676874206E6F74FE
:100BD00020706C61757369626C652E0A0043292E62
:100BE0000A003F53706563696669656420626564E5
:100BF0002074656D7065726174757265206E6F74B6
:100C000020706C61757369626C65202834302D002A
:100C1000473236207374617274696E672E2E2E0A05
:100C2000004F46460A00466164652048656967686A
:100C3000742000426564204C6576656C696E67209F
:100C4000004661696C656420746F20656E61626C3A
:100C50006520426564204C6576656C696E670A00A4
:100C6000496E76616C6964206D6573682E0A005068
:100C7000726F62696E6720506F696E740025532031
:100C800025692F2569002E0A002F0050726F6269B6
:100C90006E67206D65736820706F696E7420002028
:100CA0002844525952554E29004732392041757413
:100CB0006F20426564204C6576656C696E67003F05
:100CC00020284C2C522C462C4229206F7574206F02
:100CD0006620626F756E64732E0A003F2856296580
:100CE00072626F7365206C6576656C20696D706CDF
:100CF00061757369626C652028302D34292E0A00D5
:100D0000426164205A2076616C75650A004E6F203E
:100D100062696C696E65617220677269640A004479
:100D20006576696174696F6E0025533A20257300FA
:100D300046696E6973686564210A003A207A3A2030
:100D400000206F662000476F696E6720746F3A203D
:100D5000580043570A00206469723A0020616E67A8
:100D60006C653A00537461727420726164697573C2
:100D70003A004D343820506F696E740025533A2084
:100D800025642F256400506F736974696F6E696EF6
:100D900067207468652070726F62652E2E2E0A00BF
:100DA0003F4C656773206F66206D6F76656D656E6D
:100DB0007420696D706C61757369626C6520283090
:100DC0002D3135292E0A003F2028582C5929206F13
:100DD0007574206F6620626F756E64732E0A005002
:100DE000726F6265206F7574206F6620626F756E1A
:100DF0006473003F53616D706C652073697A652080
:100E00006E6F7420706C61757369626C6520283434
:100E10002D3530292E0A004D3438205A2D50726F4E
:100E20006265205265706561746162696C6974798C
:100E300020546573740A003F2856296572626F73E7
:100E400065206C6576656C20696D706C6175736981
:100E5000626C652028302D34292E0A005374616E8F
:100E60006461726420446576696174696F6E3A20CA
:100E7000002052616E67653A2000204D61783A206B
:100E800000204D696E3A2000205369676D613A2059
:100E9000004D65616E3A20005741524E494E472140
:100EA000204C6F77205A204A65726B206D61792043
:100EB0006C65616420746F20756E77616E74656413
:100EC000207061757365732E0A004F4646004F4EC1
:100ED0000020204D61783A2000200020204D696ECE
:100EE0003A2000536F667420656E6473746F70737C
:100EF0003A20003D3D4F6E506F7765724C6F7373B3
:100F0000526573756D653D3D004D32342053256C3F
:100F1000642054256C64004739322E3920452573EE
:100F200000473120462564004739322E39205A25A2
:100F300073004731205A302046323030004731208C
:100F400058257320592573204633303030004D34F6
:100F5000323020532569205A2573004D3130362018
:100F600050256920532569004D32303020442573C7
:100F70000047323852305859004739322E3920450F
:100F800030205A300A47315A2573004D313039200C
:100F9000532569004D31393020532569004D3432D5
:100FA00030205330205A300020496E76616C6964DD
:100FB000206578747275646572200047322F47335C
:100FC0002062616420706172616D65746572730A7C
:100FD00000536C6565702E2E2E005A2050726F6281
:100FE000652050617374204265640A005A20507273
:100FF0006F62652050617374204265640047323827
:101000004C30004D3131372050726F62652066617F
:10101000696C65642E0A4732380A0070726F626527
:101020005F72657769706500473239205265747266
:1010300079696E670050726F62696E6720466169F8
:101040006C6564004D31313720426564206C6576F3
:10105000656C696E67206661696C65642E0A47304D
:10106000205A31300A4D3330302050323520533839
:1010700038300A4D333030205035302053300A4D4F
:101080003330302050323520533838300A4D333029
:1010900030205035302053300A4D3330302050321C
:1010A0003520533838300A4D333030205035302019
:1010B00053300A47342053310070726F62655F66A7
:1010C00061696C6564004D31313720426564206C84
:1010D0006576656C696E6720646F6E652E00205AB8
:1010E0003A200020593A200042656420583A2000F6
:1010F0004D65736820706F696E74206F7574206F12
:10110000662072616E67650A004D302053746F70FF
:10111000004D312053746F7000436F6E74696E75AB
:101120006500436C69636B20746F20526573756D45
:10113000652E2E2E004E6F204D6F76652E00456E6B
:10114000642066696C65206C6973740A0042656787
:10115000696E2066696C65206C6973740A004E6F55
:10116000206D656469610A00526573756D696E670B
:1011700020534400286E6F2066696C652900437512
:101180007272656E742066696C653A2000507269EF
:101190006E742074696D653A20000A53746174732B
:1011A0003A2046696C616D656E7420757365643AAA
:1011B00020002C204C6F6E67657374206A6F623A52
:1011C0002000546F74616C2074696D653A2000537F
:1011D000746174733A20002C204661696C65643A2E
:1011E00020002C2046696E69736865643A200050BF
:1011F00072696E74733A200053746174733A2000FC
:10120000436F6F6C696E672E2E2E0048656174699E
:101210006E672E2E2E0045202553006F6B006F66E3
:1012200066006A0465045E04570449044445425557
:10123000473A004D31313320530042656420436FFB
:101240006F6C696E672E2E2E0042656420486561C2
:1012500074696E672E2E2E00544D33442045352080
:10126000506C7573204F46462E002F2F00205200E1
:10127000416363656C65726174696F6E3A205000FA
:101280004D32303620580046523A0020466C6F7777
:101290003A20003A200020536572766F2000206FBC
:1012A0007574206F662072616E67650A00536572FF
:1012B000766F200020643A0020693A0020703A00DE
:1012C000496E76616C6964206578747275646572C4
:1012D0000A0020643A0020693A0020703A006469EC
:1012E0007300656E0043290A0061626C6564202802
:1012F0006D696E2074656D702000436F6C642065AD
:101300007874727564657320617265200050494479
:10131000204175746F74756E6500504944204175A5
:10132000746F74756E65206661696C656421204216
:101330006164206865617465722069640A004669A9
:101340006C616D656E742072756E6F757420646962
:101350007374616E636520286D6D293A20004669BB
:101360006C616D656E742072756E6F757420004DC2
:1013700034323120696E636F7272656374207061FC
:1013800072616D657465722075736167650A004DE1
:1013900065736820706F696E74206F7574206F6656
:1013A0002072616E67650A004F666673657473200C
:1013B0004170706C696564004572723A20546F6FB9
:1013C000206661722100546F6F2066617220667220
:1013D0006F6D207265666572656E636520706F69FA
:1013E0006E740A00454550524F4D204F4B0A002E57
:1013F0000A002028302D313029002076616C756577
:10140000206F7574206F662072616E67650041649D
:1014100076616E6365204B3D00506F7765722D6C71
:101420006F7373207265636F766572792000436114
:10143000703A004D4541545041434B00434F4F4C8F
:1014400045525F54454D5045524154555245004315
:1014500048414D4245525F54454D504552415455C7
:10146000524500424142595354455050494E47005D
:1014700041524353004D4F54494F4E5F4D4F4445E9
:101480005300544845524D414C5F50524F544543D0
:1014900054494F4E004C4F4E475F46494C454E41D4
:1014A0004D45004155544F5245504F52545F53449F
:1014B0005F5354415455530053445F575249544568
:1014C000005245504541540053444341524400505A
:1014D000524F4D50545F535550504F525400454D4C
:1014E000455247454E43595F504152534552004380
:1014F0004153455F4C494748545F4252494748541D
:101500004E45535300544F47474C455F4C4947485D
:10151000545300534F4654574152455F504F57451F
:1015200052004255494C445F50455243454E540089
:101530004C4556454C494E475F44415441005A5F23
:1015400050524F42450052554E4F5554004155544C
:101550004F4C4556454C005052494E545F4A4F42FD
:101560000050524F4752455353004155544F524536
:10157000504F52545F54454D5000564F4C554D45B9
:101580005452494300454550524F4D0042494E4147
:1015900052595F46494C455F5452414E534645525D
:1015A0000053455249414C5F584F4E5F584F464695
:1015B000004649524D574152455F4E414D453A4DC7
:1015C00061726C696E20322E302E375F4457372E91
:1015D0003320544D334420453550534D444242202E
:1015E0002841707220323420323032312031393A81
:1015F00035313A30362920534F555243455F434FDA
:1016000044455F55524C3A68747470733A2F2F6793
:1016100069746875622E636F6D2F496E73616E69B0
:1016200074794175746F6D6174696F6E2F4D61725D
:101630006C696E2F747265652F437265616C697495
:10164000794477696E5F322E302050524F544F43A9
:101650004F4C5F56455253494F4E3A312E30204D34
:10166000414348494E455F545950453A544D3344DF
:1016700020453520506C75732045585452554445CB
:10168000525F434F554E543A3120555549443A63C1
:10169000656465326132662D343161322D34373400
:1016A000382D396231322D63353563363266333643
:1016B0003766660A0050726F6265204F6666736512
:1016C00074205A0050726F6265204F6666736574AD
:1016D000205A00290A0020746F20003F5A206F759D
:1016E00074206F662072616E6765202800290A00E9
:1016F00020746F20003F59206F7574206F66207230
:10170000616E676520282D00290A0020746F200073
:101710003F58206F7574206F662072616E67652078
:10172000282D0050726F6265204F666673657420C5
:1017300058004D383400446F6E65207072696E74C5
:10174000696E672066696C650A004D3737004D3356
:10175000310043616E6E6F74206F70656E2073751B
:101760006264697220002569730025696D2025690E
:1017700073002569682025696D2025697300256936
:1017800064202569682025696D2025697300256915
:101790007920256964202569682025696D202569DF
:1017A00073003D3D4477696E20496E697420436F34
:1017B0006D706C6574653D3D002A2A2A4E6F7A7AF9
:1017C0006C6554656D705374617475735B325D2024
:1017D0003D003D3D48656174696E6720446F6E65EC
:1017E000204368616E67652046696C616D656E7443
:1017F0003D3D002020737461727470726F67726572
:10180000737320003D3D7761697477617920353DC0
:101810003D003D3D7761697477617920343D3D003D
:101820003D3D7761697477617920333D3D003D3DF1
:101830007761697477617920313D3D003D3D6F6E80
:101840005072696E7454696D657253746F7070650F
:10185000643D3D003D3D6F6E466163746F72795229
:10186000657365743D3D00270A0A000027202700A4
:101870002027002D006E6F74696669636174696F5B
:101880006E200063616E63656C005072696E742037
:1018900041626F72746564004469736D69737300AB
:1018A00055492041626F7274656400726573756D8D
:1018B00065004D3234002A2A2A43506C6179205445
:1018C0006F6E652A2A2A003D3D6F6E5072696E74F4
:1018D00054696D65725061757365643D3D00486F74
:1018E0006D696E67204661696C6564006F70656E36
:1018F00000545249474745524544003A2000666922
:101900006C616D656E74007A5F6D696E00795F6DF4
:10191000617800785F6D6178005265706F727469EC
:101920006E6720656E6473746F7020737461747574
:10193000730A0020746F6F206C6F6E672065787477
:10194000727573696F6E2070726576656E7465640A
:101950000A0020636F6C6420657874727573696F18
:101960006E2070726576656E7465640A00486F6DEE
:10197000652025732573257320466972737400579B
:1019800061726E696E673A20486F6D696E672042BA
:10199000756D702044697669736F72203C20310A3E
:1019A000000202040000B0430000B4430000000045
:1019B0000000B0430000B4430000C84300000041F1
:1019C00000000041000000400101FF000000010094
:1019D0000000010000800055555500000040003314
:1019E000333300AAAA2A004992240000002000C72D
:1019F000711C0099991900D1451700555515003BE8
:101A0000B113002449120011111100000010000F41
:101A10000F0F00E3380E0043790D00CCCC0C00C34F
:101A2000300C00E8A20B0064210B00AAAA0A007087
:101A30003D0A009DD80900427B090092240900DC80
:101A4000D30800888808001042080000000800F051
:101A5000C107008787070075500700711C07003E0B
:101A6000EB0600A1BC0600699006006666060070E1
:101A70003E06006118060017F4050074D105005BEE
:101A8000B00500B29005006272050055550500785A
:101A9000390500B81E0500050505004EEC04008759
:101AA000D40400A1BD040090A7040049920400C121
:101AB0007D0400EE690400C7560400444404005C41
:101AC0003204000821040041100400000004003F1B
:101AD000F00300F8E0030026D20300C3C30300CCE8
:101AE000B503003AA803000A9B0300388E0300C028
:101AF0008103009F750300D0690300505E03001D41
:101B000053030034480300913D03003333030016B0
:101B1000290300381F030097150300300C0300034E
:101B20000303000BFA020049F10200BAE802005C6C
:101B3000E002002DD802002DD0020059C80200B0EA
:101B4000C0020031B90200DAB10200AAAA0200A064
:101B5000A30200BC9C0200FA9502005C8F0200DF29
:101B600088020082820200457C020027760200275C
:101B7000700200436A02007C640200D05E02003FF3
:101B8000590200C8530200FFFDFCFAF8F6F4F2F027
:101B9000EEECEAE9E7E5E3E1E0DEDCDAD9D7D5D43B
:101BA000D2D0CFCDCBCAC8C7C5C3C2C0BFBDBCBAD7
:101BB000B9B7B6B4B3B2B0AFADACAAA9A8A6A5A444
:101BC000A2A1A09E9D9C9A99989795949392908F8C
:101BD0008E8D8B8A8988878684838281807F7E7DB3
:101BE0007B7A797877767574737271706F6E6D6CBD
:101BF0006B6A696867666564636261605F5E5D5CAD
:101C00005B5A5958585756555453525150504F4E8D
:101C10004D4C4B4A4A494847464645444342424157
:101C2000403F3E3E3D3C3B3B3A3938383736353510
:101C3000343332323130302F2E2E2D2C2B2B2A29BB
:101C40002928272726252524232322212120201F58
:101C50001E1E1D1C1C1B1B1A1919181817161615E9
:101C60001514131312121111100F0F0E0E0D0D0C6F
:101C70000C0B0A0A090908080707060605050404EB
:101C8000030302020100003D3D6F6E5072696E74E5
:101C900054696D6572537461727465643D3D0000F2
:101CA00000B0430000B4430000C84300000000003F
:101CB000000000000000003D3D6F6E53746F7265C0
:101CC00053657474696E67733D3D003D3D6F6E43AF
:101CD0006F6E66696775726174696F6E53746F7247
:101CE000655772697474656E3D3D0053657474691F
:101CF0006E67732053746F726564000A20696E69A1
:101D000074207A70726F62655F7A6F66667365744D
:101D1000203D20003D3D6F6E436F6E6669677572B2
:101D20006174696F6E53746F7265526561643D3D95
:101D300000454550524F4D20496E697469616C6988
:101D40007A65640A003B20003A0A0020204D3630B4
:101D500033200020440020204D34313220530046EF
:101D6000696C616D656E742072756E6F7574207329
:101D7000656E736F723A002055004C0046696C61C5
:101D80006D656E74206C6F61642F756E6C6F61642D
:101D9000206C656E677468733A0020204D393030CE
:101DA000204B004C696E65617220416476616E6300
:101DB000653A0020204D3835312058005A2D507298
:101DC0006F6265204F66667365740020204D343164
:101DD00033205300506F7765722D4C6F7373205210
:101DE00065636F766572793A0020440020490020CF
:101DF000204D333034205000204400204900202062
:101E00004D3330312050005049442073657474695B
:101E10006E67733A00204A0020204732392057204D
:101E2000490020204D3432302053004175746F201A
:101E3000426564204C6576656C696E673A002020C7
:101E40004D323036205800486F6D65206F666673DE
:101E500065743A0020580020530020204D32303560
:101E6000204200416476616E6365643A20423C6DB5
:101E7000696E5F7365676D656E745F74696D655FCC
:101E800075733E20533C6D696E5F66656564726173
:101E900074653E20543C6D696E5F74726176656C4A
:101EA0005F66656564726174653E20583C6D61785B
:101EB0005F785F6A65726B3E20593C6D61785F792F
:101EC0005F6A65726B3E205A3C6D61785F7A5F6A2B
:101ED00065726B3E20453C6D61785F655F6A657237
:101EE0006B3E0020540020520020204D3230342020
:101EF0005000416363656C65726174696F6E202880
:101F0000756E6974732F7332293A20503C70726970
:101F10006E745F616363656C3E20523C72657472DF
:101F20006163745F616363656C3E20543C747261ED
:101F300076656C5F616363656C3E0020204D3230D6
:101F4000312058004D6178696D756D20416363657E
:101F50006C65726174696F6E2028756E6974732F79
:101F60007332293A0020204D3230332058004D6121
:101F700078696D756D20666565647261746573203E
:101F800028756E6974732F73293A005374657073E2
:101F90002070657220756E69743A0020440020201C
:101FA0004D3230302053002044697361626C6564A7
:101FB0000A0046696C616D656E742073657474699E
:101FC0006E67733A0020286D6D290020204732315A
:101FD000202020203B20556E69747320696E206D8F
:101FE0006D003D3D6F6E4C6F616453657474696E36
:101FF00067733D3D0000803B4400803B440000206F
:1020000041000096420000A0420000A042000048AB
:10201000440080CC43D0070000D0070000640000DB
:10202000004B00000024F4D43050C38E20C2A240E4
:1020300017828B7011127A910D816CD90AA861E117
:1020400008C7586607615143061E4B5D05C145A789
:10205000041A411104093D9803713931034036DBFC
:102060000265339102D4305402802E1D02632CEE9F
:1020700001752AC501B028A001102781018F2564B0
:10208000012B244B01E0223401AC211F018D200DD6
:1020900001801FFC00841EED00971DDF00B81CD2DC
:1020A00000E61BC600201BBC00641AB200B219A8CF
:1020B000000A19A0006A189900D117910040178BE7
:1020C00000B516840031167E00B31579003A1573F9
:1020D00000C7146F0058146A00EE1366008813637B
:1020E0000025135E00C7125B006C125700151254D6
:1020F00000C111510070114F0021114B00D6104941
:10210000008D1047004610440002104200C00F40EE
:1021100000800F3E00420F3C00060F3B00CB0E3804
:1021200000930E37005C0E3500270E3400F30D329D
:1021300000C10D3100900D3000600D2E00320D2DCC
:1021400000050D2C00D90C2B00AE0C2900850C29A4
:10215000005C0C2700350C27000E0C2600E80B2431
:1021600000C40B2400A00B23007D0B23005A0B217D
:1021700000390B2100180B2000F80A1F00D90A1E95
:1021800000BB0A1E009D0A1D00800A1D00630A1C78
:1021900000470A1B002C0A1B00110A1A00F7091A33
:1021A00000DD091900C4091900AB091900920917CB
:1021B000007B091800630917004C09160036091640
:1021C00000200916000A091500F5081500E008149A
:1021D00000CC081400B8081400A4081400900813D8
:1021E000007D0812006B0813005808120046081200
:1021F0000034081100230811001208110001081111
:1022000000F0071000E0071000D0071000C0071012
:1022100000B0070F00A107100091070E0083070F01
:102220000074070F0065070E0057070E0049070EE0
:10223000003B070D002E070E0020070D0013070DB1
:102240000006070D00F9060C00ED060D00E0060C77
:1022500000D4060C00C8060C00BC060C00B0060C2E
:1022600000A4060B0099060C008D060B0082060BDD
:102270000077060B006C060B0061060A0057060B80
:10228000004C060A0042060A0038060A002E060A1A
:102290000024060A001A060A001006090007060AAA
:1022A00000FD050900F4050900EB050900E2050938
:1022B00000D9050900D0050900C7050900BE0509B8
:1022C00000B5050800AD050800A50509009C050836
:1022D00000940508008C050800840508007C0508AA
:1022E00000740508006C050700650508005D05071A
:1022F00000560508004E0507004705070040050881
:102300000038050700310507002A050700230507E7
:10231000001C050600160507000F05070008050646
:102320000002050700FB040600F5040700EE0406A2
:1023300000E8040600E2040700DB040600D50406FA
:1023400000CF040600C9040600C3040600BD04064D
:1023500000B7040600B1040500AC040600A604069C
:1023600000A00405009B04060095040500900406E7
:10237000008A04050085040500800406007A04052F
:102380000075040500700405006B04050066040573
:1023900000610405005C04050057040500520405B3
:1023A000004D04050048040500430405003E0404F4
:1023B000003A04050035040500300404002C04052F
:1023C0000027040400230405001E0404001A04046A
:1023D0000016040500110404000D0404000904059E
:1023E000000404040000040400FC030400F80304D7
:1023F00000F4030400F0030400EC030400E8030409
:1024000000E4030400E0030400DC030400D8030438
:1024100000D4030400D0030400CC030400C8030369
:1024200000C503030024F404D9201BC40C5C0E98DF
:1024300004C4095F0265077101F405F900FB04B3E8
:102440000048048700C10369005803550003034591
:1024500000BE023A008402310053022A00290225FC
:102460000004022000E4011C00C8011900AF01179C
:102470000098011400840113007101100061011023
:102480000051010E0043010D0036010B002B010B22
:102490000020010B00150109000C010900030108CF
:1024A00000FB000800F3000800EB000700E4000652
:1024B00000DE000600D8000600D2000600CC0005B1
:1024C00000C7000500C2000500BD000400B90004FB
:1024D00000B5000400B1000400AD000400A9000430
:1024E00000A5000300A20003009F0004009B00035E
:1024F0000098000300950002009300030090000381
:10250000008D0002008B000300880002008600029C
:102510000084000300810002007F0002007D0002B1
:10252000007B0002007900020077000100760002C3
:10253000007400020072000100710002006F0002CE
:10254000006D0001006C0002006A000100690002D9
:1025500000670001006600010065000100640002E0
:10256000006200010061000100600001005F0002E4
:10257000005D0001005C0001005B0001005A0001E9
:1025800000590001005800010057000100560001E9
:1025900000550001005400010053000000530001E9
:1025A000005200010051000100500001004F0001E5
:1025B000004E0000004E0001004D0001004C0001E3
:1025C000004B0000004B0001004A000100490001DF
:1025D00000480000004800010047000100460000DC
:1025E00000460001004500000045000100440001D4
:1025F00000430000004300010042000000420001CF
:10260000004100000041000100400001003F0000C7
:10261000003F0001003E0000003E0001003D0000C0
:10262000003D0001003C0000003C0000003C0001B7
:10263000003B0000003B0001003A0000003A0001AE
:1026400000390000003900010038000000380000A7
:10265000003800010037000000370001003600009C
:102660000036000000360001003500000035000093
:102670000035000100340000003400000034000187
:10268000003300000033000000330001003200007E
:102690000032000000320001003100000031000073
:1026A0000031000100300000003000000030000167
:1026B000002F0000002F0000002F0000002F00015D
:1026C000002E0000002E0000002E0001002D000052
:1026D000002D0000002D0000002D0001002C000046
:1026E000002C0000002C0000002C0001002B00003A
:1026F000002B0000002B0000002B0001002A00002E
:10270000002A0000002A0000002A00010029000021
:102710000029000000290000002900000029000114
:102720000028000000280000002800000028000009
:1027300000280001002700000027000000270000FB
:1027400000270000002700010026000000260000EE
:1027500000260000002600000026000100250000E1
:1027600000250000002500000025000000250000D5
:1027700000250001002400000024000000240000C7
:1027800000240000002400010023000000230000BA
:1027900000230000002300000023000000230000AD
:1027A000002300010022000000220000002200009F
:1027B0000022000000220000002200010021000091
:1027C0000021000000210000002100000021000085
:1027D0000021000000210001002000000020000076
:1027E0000020000000200000002000000020000069
:1027F0000020000000200001001F0000001F00005A
:10280000001F0000001F0000001F0000001F00004C
:10281000001F0001001E0000001E0000001E00003E
:10282000001E000000232C0000B8220000561800F3
:10283000003A0F0000B8080000B104000071020067
:10284000003E01000020436F756E7420583A00234B
:10285000646566696E652044454641554C545F0089
:1028600000626564004B6420004B6920004B7020BF
:1028700000504944204175746F74756E6520666917
:102880006E697368656421205075742074686520D2
:102890006C617374204B702C204B6920616E642036
:1028A0004B6420636F6E7374616E74732066726F15
:1028B0006D2062656C6F7720696E746F20436F6E58
:1028C00066696775726174696F6E2E680A00504997
:1028D00044204175746F74756E65206661696C651E
:1028E00064212074696D656F75740A005049442035
:1028F0004175746F74756E65206661696C656421DD
:102900002054656D706572617475726520746F6FA7
:1029100020686967680A00204B643A2000204B69F0
:102920003A2000204B703A200020436C6173736999
:102930006320504944200A00204E6F206F76657254
:1029400073686F6F740A002054753A2000204B752D
:102950003A2000206D61783A2000206D696E3A209F
:102960000020643A200020626961733A20005049D7
:1029700044204175746F74756E6520737461727450
:102980000A00504944204175746F74756E65206665
:1029900061696C6564212054656D70657261747540
:1029A000726520746F6F20686967680A0042656409
:1029B00000453100626564002C2073797374656D85
:1029C0002073746F7070656421204865617465724E
:1029D0005F49443A200048656174696E672046612A
:1029E000696C65640048656174696E672066616939
:1029F0006C6564004D3131322053687574646F77B3
:102A00006E001000C90210012C014001220170016A
:102A10001801B0010E01F00104015002FA00B002E9
:102A2000F0003003E600D003DC009004D200700513
:102A3000C800A006BE000008B400B009AA00D00B70
:102A4000A000600E960060118C0000158200201915
:102A50007800C01D6E00A0226400B0275A00902CA0
:102A6000500000314600E0343C0010383200903A0B
:102A70002800603C1E00A03D1400803E0A00203F5C
:102A80000000544845524D414C2052554E4157414B
:102A90005900546865726D616C2052756E61776182
:102AA00079004572723A204D415854454D50004DC1
:102AB000415854454D50207472696767657265646A
:102AC000004572723A204D494E54454D50004D49D3
:102AD0004E54454D50207472696767657265640095
:102AE000202F002042403A0020403A0020573A0070
:102AF00020573A00496E76616C696420657874727B
:102B0000756465720A007C3C3E5E2B3D3F2F5B5D29
:102B10003B2C2A225C0043616E6E6F74206F7065DF
:102B20006E207375626469722000534420496E6997
:102B300074204661696C0053442063617264206FA5
:102B40006B0A006F70656E526F6F74206661696CFE
:102B500065640A00766F6C756D652E696E69742008
:102B60006661696C65640A004E6F2053442063619E
:102B700072640A000A4D3234004D3233202573004E
:102B80002E0A006F70656E206661696C65642C208A
:102B900046696C653A200046696C652073656C6512
:102BA000637465640A002053697A653A20004669B7
:102BB0006C65206F70656E65643A2000454E442058
:102BC000535542524F5554494E450A002220706FCA
:102BD00073002220706172656E743A220053554270
:102BE000524F5554494E452043414C4C207461721C
:102BF0006765743A220053756263616C6C204F768E
:102C00006572666C6F7700457863656564656420FE
:102C10006D617820535542524F5554494E452064BA
:102C2000657074683A002E0A0044656C6574696FBB
:102C30006E206661696C65642C2046696C653A207B
:102C40000046696C652064656C657465643A005380
:102C500044207072696E74696E67206279746520B1
:102C6000004E6F74205344207072696E74696E67F1
:102C70000A0057726974696E6720746F2066696C08
:102C8000653A2000667265736800646F696E67005C
:102C90002066696C653A20004E6F7720002F6175C1
:102CA000746F25632E67002020506C616E6E657214
:102CB00042756666657242797465733A20002046F3
:102CC000726565204D656D6F72793A2000436F6DB6
:102CD00070696C65643A2041707220323420323061
:102CE00032310A00204C6173742055706461746540
:102CF000643A20323032312D30342D3138207C206E
:102D0000417574686F723A2054696E794D616368D9
:102D1000696E657333440A00322E302E375F445794
:102D2000372E330A004D61726C696E0020536F6656
:102D300074776172652052657365740A002057616B
:102D4000746368646F672052657365740A0020427B
:102D5000726F776E206F75742052657365740A0008
:102D60002045787465726E616C2052657365740AD3
:102D700000506F77657255700A0073746172740A3F
:102D8000004732385859004D313030310065727289
:102D90006F722077726974696E6720746F2066693C
:102DA0006C650A00446F6E6520736176696E6720FA
:102DB00066696C652E0A004D323900456E64737485
:102DC0006F70730025532025632025632025632021
:102DD000256300205A3A0020593A0020583A0065ED
:102DE0006E6473746F7073206869743A2000000019
:102DF0000A0B02090C0D0E08070304010000000075
:102E000000000000000000000000000000000000C2
:102E1000000000000000000000001211100000007F
:102E200000000000000000000000000000000000A2
:102E30000000000070012C0190012701B001220167
:102E4000C0011D01F00118011002130130020E0132
:102E50006002090190020401C002FF000003FA00B1
:102E60004003F5008003F000D003EB002004E600EF
:102E70007004E100E004DC004005D700C005D2008A
:102E80004006CD00D006C8008007C3003008BE0051
:102E9000F008B900C009B400B00AAF00B00BAA0036
:102EA000D00CA500000EA000500F9B00C010960093
:102EB0005012910000148C00C0158700B0178200DA
:102EC000B0197D00D01B7800001E730040206E00FA
:102ED00090226900F024640040275F0090295A0086
:102EE000E02B5500102E500020304B0010324600D1
:102EF000E033410090353C00103737007038320025
:102F0000A0392D00B03A2800A03B2300603C1E00F1
:102F1000103D1900903D1400103E0F00703E0A0055
:102F2000C03E0500003F0000403FFBFF803FF6FF32
:102F3000C03FF1FF50726F62696E67204661696C35
:102F4000656400205A3A200020593A200042656406
:102F500020583A20003D3D6F6E55736572436F6E89
:102F60006669726D52657175697265643D3D0022D6
:102F70000A00556E6B6E6F776E20636F6D6D616EBC
:102F8000643A2022002042002050006F6B00204550
:102F900000205A00205900204D3932205800204589
:102FA0003A00205A3A0020593A00583A0020746FEB
:102FB0006F206C6F6E6720657874727573696F6EC1
:102FC0002070726576656E7465640A0020636F6CAC
:102FD0006420657874727573696F6E20707265769F
:102FE000656E7465640A0043616E6E6F7420656E71
:102FF000746572207375626469723A20004D3235CF
:1030000020500A4D323400526573756D6500554984
:10301000205061757365004E6F204D6174636820A8
:103020003A0050675570005067446F776E004973DF
:103030002046696C6520004973204469722000476E
:103040006F557044697200486173204D6564696111
:103050000046696C656E616D652053656C656374CF
:103060006564004D3130303043004D313030300038
:1030700046696C616D656E742053746174203020F4
:103080002D20330046696C616D656E742053746148
:10309000742030202D20320046696C616D656E749D
:1030A00020537461742030202D2031002046696C3B
:1030B000616D656E7420526573706F6E7365204E1E
:1030C0006F00526573756D65205965732064757264
:1030D000696E67207072696E74000A204E6F204618
:1030E000696C616D656E7400496E76616C6964200F
:1030F0004F7074696F6E004D3530300053746F72CD
:10310000652053657474696E67730042656420506E
:1031100049442053746172746564004D3939390A29
:103120004D32383050305331363000424C546F7588
:103130006368205265736574004D3530320A4D3531
:10314000303000496E697420454550524F4D00485B
:103150006F74656E642050494420537461727465C5
:103160006400456E676C69736820416C72656164C8
:103170007920536574004368696E657365204E6FEE
:103180007420537570706F7274656400496E4C6181
:103190006E6743686F696365000A202A2A2A726590
:1031A000636461742E646174615B305D203D00472F
:1031B00032380A4731204631303030205A31300021
:1031C000556E737570706F72746564204F7074699A
:1031D0006F6E2053656C65637465640047323652C8
:1031E000323535004D3139305335350A4732380ADA
:1031F0004732390A4D3430300A4D31303453323190
:10320000350A4732380A4D313039533231350A4D9B
:1032100034323053310A473158313030593130303F
:1032200046353030300A47315A300A4D3530300A91
:103230004D31313720536574205A204F66667365CF
:1032400074004731204631303030205A302E300063
:103250004732380A4731204631303030205A302E3C
:1032600030004D353030005A204F6666736574204B
:103270003A202573004D353030005A204F66667372
:103280006574203A202573004732380A47314631A9
:103290003530305A302E30004732385A0A473146DE
:1032A000313530305A302E30004D383400473146F9
:1032B000313030305A302E30004732380A473146EC
:1032C000313030305A302E30004D616E75616C53A4
:1032D000657454656D70005A204F6666736574207E
:1032E0003A2025730053746F7020547269676765C4
:1032F0007265640053746F70204E6F0053746F706A
:103300005072696E740048616E646C65204461742B
:10331000612041646A757374203220536574746946
:103320006E672053637265656E200048616E646C41
:10333000652044617461205072696E7446696C65E1
:1033400020332053657474696E672053637265651A
:103350006E200048616E646C652044617461205089
:1033600072696E7446696C652032205365747469A5
:103370006E672053637265656E20004D38340048D7
:10338000616E646C652044617461205072696E7472
:1033900046696C6520506F73740048616E646C659B
:1033A0002044617461205072696E7446696C6520B6
:1033B00050726500426567696E537769746368008F
:1033C0003D3D20436865636B6B65793D3D007265EB
:1033D000636461742E61646472203D3D00726563B4
:1033E0006461742E646174615B305D203D3D0077E3
:1033F000616974776179203D3D0020202A2A2A2ABC
:103400002A2A2A5254535F48616E646C6544617481
:10341000612A2A2A2A2A2A2A2A2000526573656EDE
:10342000643A200000002200250028002B002E0016
:103430003100340002010000050108010B01000009
:103440002100240027002A002D0030003300010154
:103450000000040107010A01050505050705080824
:103460000808020202020A0A08080404040401010E
:103470000101010101010303030303030303040723
:1034800007070C0C0C0C0C0C0C0C020202020606BA
:103490000606060606060B0B0B0B0B0B0B0B0102AD
:1034A0001020200808102040102040800201020156
:1034B000080402010102040810204080804020100E
:1034C0000804020180040201804020100804020167
:1034D00008040201010204081020408001020408CF
:1034E00010204080544D334420453520506C757376
:1034F0002052656164792E005072696E74696E673E
:103500002E2E2E005072696E7420506175736564A2
:10351000006E6F74696669636174696F6E20005034
:1035200049442054756E652046696E697368656408
:1035300000001401A20011241FBECFEFD1E2DEBFB4
:10354000CDBF00E00CBF14E0A0E0B2E0E0E9FAE695
:1035500002E00BBF02C007900D92A431B107D9F76A
:1035600026E1A4E1B4E001C01D92A73AB207E1F759
:103570001AE1CAE9DAE100E006C021970109802FCB
:10358000FE010F947531C939D10780E00807A9F70A
:103590000F94CD1E0D9436350C9400009F92AF927F
:1035A000BF92CF92DF92EF92FF920F931F93CF9330
:1035B000DF9300D01F921F92CDB7DEB7E7E8FBE1A3
:1035C0000027BB27462F572FA82FAA2341F4A52F4A
:1035D000542FB85FAA2319F4A52F5527B85FA0313F
:1035E00038F45295A295452F4F70507FA42BBC5FA5
:1035F000A03428F4550FAA1F550FAA1FBE5FA0388C
:1036000018F4550FAA1FB395550FAA1FEA0FF01F04
:10361000449151E0AA27B85081F1C8F0B0FF02C030
:10362000440F551FB1FF04C0440F551F440F551FD1
:10363000B2FF06C052954295142F1F70407F512B48
:10364000B3FF1BC0A52F542F44270C943D1BB195ED
:10365000B0FF02C055954795B1FF04C055954795F9
:1036600055954795B2FF05C05295407F4295452B31
:103670005F70B3FF02C0452F5527DD24CC24BB2447
:10368000B2E0649FD018C108B00AB00B749FC01894
:10369000B108B00B849FB018B109659FC018B1087C
:1036A000B00B759FB018B109859FB0196A9FB0180B
:1036B000B1097A9FB0194D9DA12C992433279927E0
:1036C00022275D9DA00C911C301F901F201FAD9DD7
:1036D000900C311D901F201F4C9DA00C911C301F81
:1036E000901F201F5C9D900C311D901F201FAC9DD2
:1036F000300D911D201F4B9D900C311D901F201FE0
:103700005B9D300D911D201FAB9D900D211D4B9F8A
:10371000300D911D201F5B9F900D211DAB9F200D33
:10372000B1E0BB24CC24DD24639FD018C108B00ACB
:10373000B00B739FC018B108B00B839FB018B109CC
:10374000699FC018B108B00B799FB018B109899F63
:10375000B019629FB018B109729FB019D61AC70A82
:10376000B80A20F0B1E03B0F901F201F1124792FE1
:10377000632F90E0822F0F900F900F900F900F907B
:10378000DF91CF911F910F91FF90EF90DF90CF903D
:10379000BF90AF909F900895AF92BF92CF92DF926B
:1037A000EF92FF920F931F93CF93DF93C5EADCE074
:1037B00008EF18E085EBA82E8CE0B82EC12CD12C98
:1037C0007601C39469917991899199910F94B32A63
:1037D000288939894A895B890F94142B0F94F13217
:1037E000F80161937193819391938F01C616D70667
:1037F000E806F90610F46B017C01AC16BD0611F762
:103800006FEF7FEFCB01A70196010F94F230209369
:1038100008093093090940930A0950930B09DF9175
:10382000CF911F910F91FF90EF90DF90CF90BF90BD
:10383000AF900895CF92DF92EF92FF92809114089B
:10384000882309F457C0C0901008D0901108E09068
:103850001208F090130820E030E0A901C701B6017A
:103860000F94AE2A882309F445C020E030E040E000
:103870005FE3C701B6010F94142B9B01AC010F94B9
:10388000142B2BED3FE049E450E40F94142B9B01E3
:10389000AC0160E070E080E89FE30F9478326B0148
:1038A0007C01C092A10CD092A20CE092A30CF092E9
:1038B000A40C60917D0270917E02072E000C880B93
:1038C000990B0F94B52A2AE037ED43E25CE30F949D
:1038D000142BA70196010F94142B60937902709317
:1038E0007A0280937B0290937C02FF90EF90DF90AE
:1038F000CF900895C12CD12C80E8E82E8FE3F82ECC
:10390000D0CF0F931F93CF93DF9350E0FC01E40FD0
:10391000F51F8081440F551F440F551F4E545A4FB9
:10392000EA01882329F188819981AA81BB81EB0171
:10393000088119812A813B810097A105B10569F4AD
:103940000C591F4F2F4F3F4FDA010D931D932D93AD
:103950003C9313978FEF808306C0081B190B2A0B2B
:103960003B0B37FDF7CFDF91CF911F910F9108955A
:10397000188219821A821B82F6CFCF93DF9324E03C
:10398000829FC0011124EC01C551D74FFC01EF5DAE
:10399000F74F8B5E974FDC012D913D914D915C91DE
:1039A00060817181828193810F947E3168837983F4
:1039B0008A839B83DF91CF9108958091AD0590918B
:1039C000AE05A091AF05B091B005809349029093E8
:1039D0004A02A0934B02B0934C028091AB059091A8
:1039E000AC059093800280937F02089580914902F4
:1039F00090914A02A0914B02B0914C028093AD0588
:103A00009093AE05A093AF05B093B00580917F026F
:103A1000909180029093AC058093AB0584E690E092
:103A20009093800280937F0208958091F01290918C
:103A3000F112891B877089F48091F80D81110DC0F6
:103A40008091ED0C9091EE0C892B39F481E09091EE
:103A5000BB06911103C080E0089581E00895CF93E3
:103A6000DF93DB01F9019C919130C1F0943080F03B
:103A700094509C938830D1F480819181009771F0AB
:103A8000019791838083480F591FEA01188206C06D
:103A90008C3539F49C5F9C93943041F4DF91CF9145
:103AA00008958B3339F781E08C93F8CF20813181F1
:103AB000B9016F5F7F4F71836083420F531FEA012B
:103AC0008883808191818F3591056CF7E7CF0F93C3
:103AD0001F9381E00091A4141091A5142091A614C5
:103AE0003091A7144091A0145091A1146091A21498
:103AF0007091A314041715072607370708F480E010
:103B00001F910F91089590E080E00895282F9091E3
:103B10000F08833021F495FD0FC094FD0FC0892F4D
:103B200090E0B0E0A0E004C0B695A7959795879582
:103B30002A95D2F78170089581E0089580E0089574
:103B4000FC01659175918591949108958F929F9252
:103B5000AF92BF92CF92DF92EF92FF92CF93DF931B
:103B6000EC018090E7089090E808A090E908B090F8
:103B7000EA0820E030E0A901C501B4010F94AE2AA3
:103B8000882309F454C0C880D980EA80FB80A7014B
:103B90009601C501B4010F94AE2A18160CF04CC062
:103BA0002091DF083091E0084091E1085091E2084F
:103BB000C701B6010F94AE2A882331F1C092DF0805
:103BC000D092E008E092E108F092E2082091E30848
:103BD0003091E4084091E5085091E60868817981C8
:103BE0008A819B810F94142B9B01AC0160E070E0F3
:103BF00080E89FE30F947D3160930F027093100271
:103C0000809311029093120260910F027091100242
:103C10008091110290911202DF91CF91FF90EF906D
:103C2000DF90CF90BF90AF909F908F90089560E00D
:103C300070E080E89FE3F0CF60E070E0CB01ECCF74
:103C4000CF92DF92EF92FF92CF93DF93EC01CC8083
:103C5000DD80EE80FF8027E137EB41ED58EBC701B7
:103C6000B6010F94DE3387FD23C023E030E044EB40
:103C700053E4C701B6010F94AE2A1816CCF0C880E1
:103C8000D980EA80FB8027E137EB41ED58EBC70193
:103C9000B6010F94DE3387FD0BC0C1E023E030E0B6
:103CA00040EB53E4C701B6010F94AE2A18160CF48A
:103CB000C0E08C2FDF91CF91FF90EF90DF90CF90FD
:103CC00008952FEB280F2A3108F047C0E22FF0E0CB
:103CD0008091470590914805A0914905B0914A050A
:103CE00004C0B695A795979587952A95D2F780FD3C
:103CF00002C081700895E75DFA4FE081EE2341F143
:103D00008091A1079091A207E80FF92FF11D808102
:103D100090ED980F9A3030F08E3251F481818053BB
:103D20008A3098F4F0931805E093170581E0089520
:103D30008D3211F08B3249F4818190ED980F9A30D9
:103D400088F38E3211F48281EACFF0E0E0E0EACF2E
:103D50001092180510921705E9CF80E008950E948F
:103D6000611E882341F081E02091170530911805EC
:103D7000232B09F480E008958F929F92AF92BF9217
:103D8000CF92DF92EF92FF92C090E905D090EA05C2
:103D9000E090EB05F090EC0520E030E0A901C701D0
:103DA000B6010F94AE2A8823E1F1A701960160E0E5
:103DB00070E080E89FE30F9478326B017C01809083
:103DC000ED059090EE05A090EF05B090F00520E095
:103DD00030E0A901C501B4010F94AE2A882329F16E
:103DE000A501940160E070E080E89FE30F947832D1
:103DF000C092F004D092F104E092F204F092F30445
:103E00006093F4047093F5048093F6049093F704A0
:103E1000FF90EF90DF90CF90BF90AF909F908F90EA
:103E20000895C12CD12C7601CACF60E070E0CB019F
:103E3000DFCF129A08955F9A80919F0C8E7F8093B6
:103E40009F0C8A9A80919F0C8D7F80939F0C80910C
:103E50000801809581708093060180919F0C8B7F73
:103E600080939F0C0C94191F269A2E9A08958C32D9
:103E700021E0920714F08CE291E090935512809328
:103E800054120C9465E9E5E2F6E010821182128288
:103E9000138214820C9465E94F925F926F927F9225
:103EA0008F929F92AF92BF92CF92DF92EF92FF924A
:103EB0000F931F93CF93DF93EC012091E105309195
:103EC000E2054091E3055091E405688179818A819A
:103ED0009B810F947D316B017C012091E505309130
:103EE000E6054091E7055091E8056C817D818E8162
:103EF0009F810F947D314B015C01A7019601609178
:103F000003027091040280910502909106020F94C1
:103F1000AE2A882309F450C0C0920302D092040252
:103F2000E0920502F09206022091F0043091F10433
:103F30004091F2045091F304C701B6010F94142B81
:103F40002B013C010F9420336B017C0120E030E019
:103F5000A9010F94AE2A87FD70C020E030E040E454
:103F600050E4C701B6010F94DE3318162CF4C12CAF
:103F7000D12CC0E4EC2EFE2CA7019601C301B201A6
:103F80000F947D316093E8047093E9048093EA0410
:103F90009093EB04C701B6010F94EA326093E604F4
:103FA000062E000C770B6F5F7F4F6430710514F0A5
:103FB00064E070E06093E404D09101021091E604A3
:103FC000A501940160910702709108028091090295
:103FD00090910A020F94AE2A811133C0D11381C08F
:103FE0002091CC043091CD044091CE045091CF0467
:103FF0006091E8047091E9048091EA049091EB04E7
:104000000F94142B2091D0043091D1044091D2040C
:104010005091D3040F947E31DF91CF911F910F9176
:10402000FF90EF90DF90CF90BF90AF909F908F90D8
:104030007F906F905F904F900895C12CD12C7601A6
:104040009BCF8092070290920802A0920902B09240
:104050000A022091F4043091F5044091F604509145
:10406000F704C501B4010F94142B4B015C010F94AC
:1040700020336B017C0120E030E0A9010F94AE2ACF
:1040800087FDF3C020E030E040E450E4C701B60112
:104090000F94DE3318162CF4C12CD12CB0E4EB2E87
:1040A000FE2CA7019601C501B4010F947D316093E8
:1040B000EC047093ED048093EE049093EF04C70139
:1040C000B6010F94EA326093E704062E000C770BDA
:1040D0006F5F7F4F6430710514F064E070E06093AF
:1040E000E504C091E704D11305C0809102028C174A
:1040F00009F470C08091E6049091E7049093020265
:10410000809301020C2E000CDD0B25E01203C00190
:104110001124FC01EC0FFD1FEE0FFF1FEE0FFF1F20
:10412000E555F84F20813181428153812093E0048D
:104130003093E1044093E2045093E3040091E504DA
:10414000002E000C110BFC01E00FF11FEE0FFF1F02
:10415000EE0FFF1FE555F84F6081718182819381D9
:104160000F947D316093DC047093DD048093DE0452
:104170009093DF042091E40435E02303F00111243F
:10418000CE0FDF1FCC0FDD1FCC0FDD1FC555D84F65
:10419000288139814A815B812093D8043093D904E6
:1041A0004093DA045093DB04E00FF11FEE0FFF1F82
:1041B000EE0FFF1FE555F84F608171818281938179
:1041C0000F947D316093D4047093D5048093D6040A
:1041D0009093D7048090EC049090ED04A090EE04AE
:1041E000B090EF042091DC043091DD044091DE04B6
:1041F0005091DF04C501B4010F94142B2091E00409
:104200003091E1044091E2045091E3040F947E3137
:104210006B017C01C092D004D092D104E092D20410
:10422000F092D3042091D4043091D5044091D60467
:104230005091D704C501B4010F94142B2091D804D8
:104240003091D9044091DA045091DB040F947E310F
:10425000A70196010F947D316093CC047093CD0437
:104260008093CE049093CF04BBCEC12CD12C760189
:1042700018CFCF92DF92EF92FF92CF93DF93EC01B2
:1042800008960E94A61D6B017C0120E030E0A90188
:104290000F94AE2A20E030E0A901882359F0CE0126
:1042A0000E944C1F9B01AC01C701B6010F94142B57
:1042B0009B01AC01688579858A859B850F947D314A
:1042C000688779878A879B87DF91CF91FF90EF90EE
:1042D000DF90CF9008952F923F924F925F926F920E
:1042E0007F928F929F92AF92BF92CF92DF92EF9286
:1042F000FF920F931F93CF93DF93D62FC72FFC010D
:1043000080809180A280B380C501B40120E831E5AE
:1043100041E050E00F94F230C9016DE671E00F9476
:1043200061316B017C01C501B40120E13EE040E058
:1043300050E00F94F230CA01B90128E130E040E0CA
:1043400050E00F94F230362E272E062F172F8CE3D5
:10435000482E512C612C712CC501B401A30192018E
:104360000F94F230B62EA72ECA01B901A301920113
:104370000F94F230CB01C114D10479F1AF92BF9206
:104380007F936F932F923F92FF92EF92DF92CF92A3
:104390008EE897E19F938F93CF93DF930F94452AF5
:1043A0008DB79EB70E960FB6F8949EBF0FBE8DBF09
:1043B0008D2F9C2FDF91CF911F910F91FF90EF9048
:1043C000DF90CF90BF90AF909F908F907F906F9035
:1043D0005F904F903F902F900895E114F104C9F041
:1043E000AF92BF927F936F932F923F92FF92EF9283
:1043F0008EE797E19F938F93CF93DF930F94452A96
:10440000EDB7FEB73C960FB6F894FEBF0FBEEDBFFA
:10441000CFCF012BB9F0AF92BF927F936F932F92C2
:104420003F9282E797E19F938F93CF93DF930F940F
:10443000452A8DB79EB70A960FB6F8949EBF0FBE59
:104440008DBFB6CF892BA9F0AF92BF927F936F93A8
:104450008AE697E19F938F93CF93DF930F94452A3A
:10446000EDB7FEB738960FB6F894FEBF0FBEEDBF9E
:104470009FCFAF92BF9286E697E19F938F93CF93A2
:10448000DF930F94452A0F900F900F900F900F908D
:104490000F908ECFEF92FF920F931F93CF93DF93E6
:1044A000CDB7DEB78C01EDB6FEB60F94FB290196B1
:1044B0002DB73EB7281B390B0FB6F8943EBF0FBE81
:1044C0002DBF8DB79EB70196B8010F94F4290F94B4
:1044D000D71B0FB6F894FEBE0FBEEDBEDF91CF9195
:1044E0001F910F91FF90EF9008958C38910514F073
:1044F0008CE890E09093EA118093E9110C9466C1E6
:10450000AB01BC014093A4145093A5146093A6146E
:104510007093A7148CE096E10C941EB22F923F92F8
:104520004F925F926F927F928F929F92AF92BF92C3
:10453000CF92DF92EF92FF920F931F93CF93DF936F
:10454000CDB7DEB760970FB6F894DEBF0FBECDBF14
:104550008B876C87042F122F282F30E03E872D8702
:10456000462F50E05A87498785E0982E929EC001D9
:10457000939E900D1124988B8F87FA01E80FF91FF5
:10458000EE0FFF1FEE0FFF1FE555F84F60817181A1
:10459000828193819B01AC010F947034882309F4CC
:1045A00045C14B85400F6C85610F949EC00111245D
:1045B000E985FA85E80FF91FEE0FFF1FEE0FFF1FC9
:1045C000E555F84FC080D180E280F380040F909EC3
:1045D000A0011124E985FA85E40FF51FEE0FFF1FF6
:1045E000EE0FFF1FE555F84F0081918082807380A8
:1045F000262F30E0EF85F889E20FF31FEE0FFF1F43
:10460000EE0FFF1FE555F84F20807181798372818D
:104610007A8373817B83610F70E0EF85F889E60F01
:10462000F71FEE0FFF1FEE0FFF1FE555F84FF88B3A
:10463000EF87F081FC83EF85F889F181FD83EF85B9
:10464000F889F281FE83EF85F889F381FF83FC010D
:10465000E20FF31FEE0FFF1FEE0FFF1FE555F84FA0
:1046600020812887A180B2806380FA01E60FF71FBE
:10467000EE0FFF1FEE0FFF1FE555F84F40805180F2
:1046800032801381202F392D482D572D602F792D01
:10469000882D972D0F947034882321F000E0912C01
:1046A000812C712C9601A701B601C7010F947034BB
:1046B000882321F0C02ED92CE82CF72C2C813D81A9
:1046C0004E815F816C817D818E819F810F947034DA
:1046D000882321F01C821D821E821F82222D398197
:1046E0004A815B81622D79818A819B810F9470342C
:1046F000882339F02C803D8139834E814A835F8144
:104700005B839201432D512FB201832D912F0F9482
:104710007034882321F0412C512C312C10E0288555
:104720003A2D4B2D562D68857A2D8B2D962D0F9475
:104730007034882321F04886A52CB32C612E85E0A7
:104740002D853E85829FF001839FF00D11244985C0
:104750005A85E40FF51FEE0FFF1FEE0FFF1FE55503
:10476000F84FFA87E9879601A701B601C7010F94B0
:104770007E31202F392D482D572D0F947D316B011F
:104780007C01222D39814A815B81622D79818A8168
:104790009B810F947E312C813D814E815F810F94EE
:1047A0007D319B01AC01C701B6010F947E316B01D5
:1047B0007C0128853A2D4B2D562D68857A2D8B2D21
:1047C000962D0F947E319201432D512F0F947D3100
:1047D0009B01AC01C701B6010F947E3120E030E0AF
:1047E00040E450E40F947832E985FA856083718360
:1047F000828393836C858B8560960FB6F894DEBFB9
:104800000FBECDBFDF91CF911F910F91FF90EF9021
:10481000DF90CF90BF90AF909F908F907F906F90E0
:104820005F904F903F902F900D94171A60960FB69F
:10483000F894DEBF0FBECDBFDF91CF911F910F91D6
:10484000FF90EF90DF90CF90BF90AF909F908F90B0
:104850007F906F905F904F903F902F900895809140
:10486000170590911805009731F04AE050E070E08C
:1048700060E00D94C92860E070E0CB01089580915C
:10488000170590911805009731F04AE050E070E06C
:1048900060E00D949B2760E070E0CB010895CF931A
:1048A000DF93EB010E94AF1E882319F00E943F2482
:1048B000EB01CE01DF91CF9108950E943F2497FD37
:1048C0000CC00E943F246F3F71058105910509F0DE
:1048D00034F40E943F24862F089580E008958FEFDE
:1048E0000895CF93C62F0E94AF1E882319F0CF9151
:1048F0000C945D248C2FCF91089580911705909191
:104900001805892B41F00E945D2491E0811101C0BE
:1049100090E0892F089591E0FCCFCF93DF93C82FCB
:10492000D62F0E94AF1E882321F0DF91CF910C94E7
:104930007D248C2F0E94611E811101C08D2FDF917B
:10494000CF9108950E943F24CB010895CF93DF9328
:10495000EB010E94AF1E882321F0DF91CF910C94D0
:10496000A224CE01DF91CF9108950F931F93CF938F
:1049700080911705909118050097E9F0FC018F01CF
:10498000C1912C2F2F7D81F0C53411F0C536B9F7B8
:10499000F801108270E060E00F943D26F801C083BA
:1049A000CF911F910F91089570E060E0CF911F911A
:1049B0000F910D943D2660E070E0CB01F1CFCF92D6
:1049C000DF92EF92FF926A017B010E94AF1E882363
:1049D00031F0FF90EF90DF90CF900C94B524C70199
:1049E000B601FF90EF90DF90CF9008954F925F92C5
:1049F0006F927F928F929F92AF92BF92CF92DF92EF
:104A0000EF92FF921F93CF93DF9300D01F92CDB709
:104A1000DEB719821A821B821C82CE0101964C01DC
:104A20008FE8C82E87E0D82E99E6E92E92E0F92E7D
:104A30002BEEA22E28E0B22E10E088E5810F0E9416
:104A4000AF1EF40181934F01882309F4E0C00E9456
:104A5000B5242B013C01812F0E94861D882309F477
:104A6000CCC0F7012081318142815381C301B20161
:104A70000F947E31F60160837183828393831F5F7D
:104A8000F4E0CF0ED11C84E0E80EF11C94E0A90EF6
:104A9000B11C133091F685E40E94AF1E8C838823ED
:104AA00009F4C0C00E94B5246B017C0183E00E9420
:104AB000861D882371F02091750230917602409115
:104AC000770250917802C701B6010F947E316B01D5
:104AD0007C01C0929B07D0929C07E0929D07F092C8
:104AE0009E078091E005882359F18091A81482FFE8
:104AF00027C08C81882321F18981811103C08A819B
:104B00008823F1F02DEC3CEC4CE45DE36091360839
:104B10007091370880913808909139080F947E3150
:104B20009B01AC01609171027091720280917302DD
:104B3000909174020F94DE33181614F40F945D19DB
:104B400040E050E0BA0186E40E94DF2420E030E03B
:104B5000A9010F94DE33181684F40E94B52420E0D6
:104B600030E040E752E40F9478326093490270934A
:104B70004A0280934B0290934C0280915D0C83FD1E
:104B800028C08091A606882321F1209175023091DA
:104B90007602409177025091780260919B07709164
:104BA0009C0780919D0790919E070F947D312091E5
:104BB000B3063091B4064091B5065091B6060F94F5
:104BC0007E316093B3067093B4068093B5069093DC
:104BD000B6060F900F900F900F90DF91CF911F911D
:104BE000FF90EF90DF90CF90BF90AF909F908F900D
:104BF0007F906F905F904F900895F50120813181F3
:104C000042815381C301B2010F947D3133CFF7014B
:104C100080819181A281B381F60180839183A283F7
:104C2000B3832DCF8091750290917602A091770287
:104C3000B091780280939B0790939C07A0939D0767
:104C4000B0939E074ECFCF92DF92EF92FF926B010F
:104C50007C0183E3C816D104E104F10470F082E31F
:104C6000C81AD108E108F10862E370E080E090E042
:104C70000E949FA90E94E0C4ECCFC701B6010E9428
:104C80009FA9FF90EF90DF90CF900C94E0C4CF925B
:104C9000DF92EF92FF920F931F93CF93DF936B01FD
:104CA0007A01EC01C455DB4F28813CE0389F80013C
:104CB000399F100D112427FF24C0FB01118210829F
:104CC00088818F5F888388819801280F311D87FD37
:104CD0003A95C9012091DB12F6012817190629F02F
:104CE00024F088818C300CF43CC080819181049642
:104CF00080349C4908F475C0F60180819181049646
:104D000072C088819801280F311D87FD3A95C9012D
:104D10002091DB122817190699F294F28881A801D4
:104D2000480F511D87FD5A95FA01EE0FFF1FE40F42
:104D3000F51FED56FD4E808187FFC2CF8881F801B7
:104D4000E80FF11D87FDFA95CF01EE0FFF1FE80F69
:104D5000F91FED56FD4E808160E08F770E94FAA723
:104D6000AFCF808191812881A801420F511D27FD7D
:104D70005A959A01FA01EE0FFF1FE20FF31FED564D
:104D8000FD4E21813281820F931FF7019183808331
:104D900088819801280F311D87FD3A95F901EE0FA2
:104DA000FF1FE20FF31FED56FD4E808187FF20C0ED
:104DB0008881080F111D87FD1A95F801EE0FFF1F5E
:104DC000E00FF11FED56FD4E808161E08F77DF919E
:104DD000CF911F910F91FF90EF90DF90CF900C94A7
:104DE000FAA780E49CE9F701918380838FEF8883A1
:104DF000DF91CF911F910F91FF90EF90DF90CF90B7
:104E000008950F931F93CF93DF9309EB1CE0CDEC34
:104E1000D1E1F80121913191419151918F0160E0EF
:104E200070E080E89FE30F947832699379938993D7
:104E30009993F1E1CD3DDF0761F70F949C17DF9166
:104E4000CF911F910F910C94CC1BCF92DF92EF92D8
:104E5000FF92CF93DF932091A00C222329F1EC0144
:104E600008960E94A61D6B017C0120E030E0A9019C
:104E70000F94AE2A20E030E0A901882359F0CE013A
:104E80000E944C1F9B01AC01C701B6010F94142B6B
:104E90009B01AC01688579858A859B850F947E315D
:104EA000688779878A879B87DF91CF91FF90EF9002
:104EB000DF90CF9008952F923F924F925F926F9222
:104EC0007F928F929F92AF92BF92CF92DF92EF929A
:104ED000FF920F931F93CF93DF93CDB7DEB76C97FD
:104EE0000FB6F894DEBF0FBECDBF8C015B015A83B5
:104EF0004983FC01EF5AFF4F208131814281538168
:104F000029873A874B875C87CA01B9010F94B32A76
:104F10006B017C01D5012D913D914D915C910F94D8
:104F2000142B0F945C322B013C01E981FA81208122
:104F3000318142815381C701B6010F94142B0F9424
:104F40005C324B015C01C301B2010F94F132698BF9
:104F50007A8B8B8B9C8B683771058105910540F4AA
:104F600028E730E040E050E0298B3A8B4B8B5C8B9C
:104F7000C501B4010F94F1326D877E878F87988BBE
:104F8000683771058105910540F448E750E060E01D
:104F900070E04D875E876F87788BF801E35AFF4F8B
:104FA0004080518062807380C301B2010F94B52AA2
:104FB00069837A838B839C8369897A898B899C89AD
:104FC0000F94B32A6D8B7E8B8F8B988F20E030E00F
:104FD000A90169817A818B819C810F94AE2A8823F3
:104FE00009F4E1C1A7019601C701B6010F94142B82
:104FF0004B015C012D893E894F89588DCA01B90149
:105000000F94142B9B01AC01C501B4010F947D31A9
:105010004B015C0129813A814B815C81CA01B90154
:105020000F947E319B01AC01C501B4010F9478321D
:105030000F945C320F94F1326D837E838F83988757
:1050400066277727CB0164197509860997090F949C
:10505000B52A4B015C016D857E858F8598890F94FB
:10506000B32A2B013C0120E030E0A901C501B401C5
:105070000F94AE2A882309F49AC1A3019201C301B7
:10508000B2010F94142B698F7A8F8B8F9C8FA7019D
:105090009601C701B6010F94142B9B01AC01698DD9
:1050A0007A8D8B8D9C8D0F947D316B017C01A501D8
:1050B0009401C501B4010F947E319B01AC01C7017D
:1050C000B6010F9478320F942033D80195968D90C5
:1050D0009D90AD90BC909897750164012D813E81A3
:1050E0004F815885C21AD30AE40AF50A0F94F132A7
:1050F000C61AD70AE80AF90AF7FE8EC02D893E893A
:105100004F89588DCA01B9010F94142B6B017C0192
:1051100029813A814B815C81CA01B9010F947E31AA
:1051200069877A878B879C8720E030E0A9016981B5
:105130007A818B819C810F94AE2A882309F43BC12C
:10514000C501B4010F94B32A29853A854B855C8546
:105150000F94142BA70196010F947D316D837E83EC
:105160008F839887A3019201C301B2010F94142B7E
:105170009B01AC016D817E818F8198850F947E317A
:105180002B013C0120E030E040E850E469817A8165
:105190008B819C810F94142B9B01AC01C301B20144
:1051A0000F9478320F945C322B013C0120E030E008
:1051B000A9010F94DE3318161CF0412C512C32013A
:1051C000C301B2010F94F1326D837E838F83988780
:1051D00086169706A806B90620F48D829E82AF82B5
:1051E000B8866D817E818F8198850F94B32A298539
:1051F0003A854B855C850F94142BA70196010F947B
:105200007E310F942C340F94F13269877A878B8723
:105210009C87C12CD12C760169857A858B859C85EC
:1052200029893A894B895C89621B730B840B950B26
:105230000F94B32A29813A814B815C810F94783293
:1052400020E034E244EF59E40F94142B0F94F13230
:105250004B015C0169857A858B859C852D853E8512
:105260004F855889621B730B840B950B0F94B32ADF
:1052700029813A814B815C810F94783220E034E2BD
:1052800044EF59E40F94142B0F94F1322B013C019D
:105290003FE683169104A104B10408F090C0F40124
:1052A000EE0FFF1FEE0FFF1FE553F64E8591959110
:1052B000A591B4918983292E3A2EBD8B4FE64416D1
:1052C00051046104710408F083C0F201EE0FFF1F66
:1052D000EE0FFF1FE553F64E459155916591749180
:1052E0009A01CB014D815E816F817885D8019996B5
:1052F0004D935D936D937C939C974C0D5D1D6E1D3E
:105300007F1DF80145A756A767A770ABEB5AFF4F63
:1053100049895A896B897C8940835183628373836D
:10532000D5968D929D92AD92BC92D897F80141AEE0
:1053300052AE63AE74AEFD964981408321823282C3
:105340005D89538334962083318382839383698577
:105350007A858B859C85D1966D937D938D939C9357
:10536000D49778962D853E854F8558892083318343
:10537000428353836C960FB6F894DEBF0FBECDBF49
:10538000DF91CF911F910F91FF90EF90DF90CF9021
:10539000BF90AF909F908F907F906F905F904F9055
:1053A0003F902F90089560E070E0CB0141CE60E027
:1053B00070E0CB0188CE60E070E0CB01F3CEC50198
:1053C000B4010E94CE1A6983272E382E9D8B76CF8A
:1053D000C301B2010E94CE1A9B0184CF8091F012CA
:1053E0009091F112891B877019F490E080E0089584
:1053F0009091ED12992351F0833030F48FEF890FA3
:1054000019F08093ED12F1CF1092ED128091F1120C
:1054100027E6829FC00111248B5D964FFC012081FD
:1054200020FDE3CF2091F1122F5F27702093EE1221
:105430003091F1122091EF12321304C02091EE123C
:105440002093EF12089590916F0081E091FD02C0CA
:1054500080E0089590916F009D7F90936F00089574
:1054600080FF04C090919F0C90FD8E7F81FF05C04E
:1054700090919F0C969590FD8D7F82FF06C0909134
:105480009F0C9695969590FD8B7F08958F929F9295
:10549000AF92BF92CF92DF92EF92FF92CF93DF93C2
:1054A00020914D02222309F49EC0EC018091B105A8
:1054B000C82ED12CF12CE12C80FF2CC080904F0203
:1054C00090905002A0905102B090520228813981F0
:1054D0004A815B81C501B4010F94DE33181624F4B0
:1054E00088829982AA82BB8280905B0290905C0243
:1054F000A0905D02B0905E02288139814A815B8173
:10550000C501B4010F94AE2A87FF04C08882998236
:10551000AA82BB82D701C601B695A79597958795B4
:1055200080FF2CC08090530290905402A0905502AE
:10553000B09056022C813D814E815F81C501B4013E
:105540000F94DE33181624F48C829D82AE82BF82C3
:1055500080905F0290906002A0906102B090620221
:105560002C813D814E815F81C501B4010F94AE2A2B
:1055700087FF04C08C829D82AE82BF8282E0F69457
:10558000E794D794C7948A95D1F7C0FE2CC0C090F9
:105590005702D0905802E0905902F0905A022885A4
:1055A00039854A855B85C701B6010F94DE3318162D
:1055B00024F4C886D986EA86FB86C0906302D09020
:1055C0006402E0906502F0906602288539854A857C
:1055D0005B85C701B6010F94AE2A87FF04C0C88659
:1055E000D986EA86FB86DF91CF91FF90EF90DF901E
:1055F000CF90BF90AF909F908F900895CF92DF9201
:10560000EF92FF920F931F93C12CD12C76018C0146
:1056100025E732E041E752E06DE672E089E692E08C
:105620000F9434001F910F91FF90EF90DF90CF9077
:1056300008950D949C1780919E05659B6EC08061B6
:1056400080939E059091030180919E0591FF67C014
:10565000806280939E0580919E054B9B62C0846012
:1056600080939E0580919E0590919D05981709F461
:105670005AC092E090939C0580939D058091B80656
:10568000811105C080919F07882309F459C080913A
:10569000050680FF10C08091B90680FD0CC0809186
:1056A0009B0584FF08C08091FB0680618093FB0608
:1056B00080E00E946ACD80910506869580FF11C02A
:1056C0008091B906869580FD0CC080919B0585FF71
:1056D00008C08091FB0680628093FB0681E00E94F7
:1056E0006ACD809105068695869580FF29C08091B8
:1056F000B9068695869580FF23C080919F078823F1
:10570000F9F080919B0582FF1BC08091FB068460AD
:105710008093FB0682E00C946ACD8F7E91CF8F7DC3
:1057200098CF8B7F9DCF80919C05882309F4A6CFCD
:10573000815080939C058111A1CF90939B059ECFB2
:1057400008958091B806811104C080919F07882335
:1057500031F062E070E080E090E00C942326089540
:105760000F931F9380918B11813019F50E94D2A95C
:105770000091BA051091BB052091BC053091BD0583
:10578000601B710B820B930B28EE33E040E050E07E
:105790000F94F2306091BE057091BF058091C005F5
:1057A0009091C105620F731F841F951F1F910F9168
:1057B00008956091C2057091C3058091C4059091D0
:1057C000C505D6CF10928B111092BA051092BB0569
:1057D0001092BC051092BD051092C2051092C3052F
:1057E0001092C4051092C5051092BE051092BF0517
:1057F0001092C0051092C1050895CF92DF92EF92EA
:10580000FF92CF93DF93C62FFC01C080D180E2804E
:10581000F38020E030E0A901C701B6010F94AE2A61
:1058200020E030E0A90187FD14C020E030E048EC22
:1058300052E4C701B6010F94DE3324E630E040E0C5
:1058400050E0181634F0C701B6010F94EA329B01FC
:10585000AC01C230A0F4D0E0C05ED64FAFEFB0E0F4
:105860000F94333124E630E040E050E00F941431DF
:105870002F3F310519F010F02FEF30E02883DF9132
:10588000CF91FF90EF90DF90CF9008958091090124
:1058900080FD06C08091A81483FB882780F90895B5
:1058A00080E00895CF92DF92EF92FF92FC01C080DA
:1058B000D180E280F380663019F510922A061092AA
:1058C0002B0610922C0610922D0610922E060E9486
:1058D00066C120E030E0A901C701B6010F94AE2AED
:1058E00087FF1DC0C12CD12C7601C701B6010F94D2
:1058F000EB33CB01FF90EF90DF90CF900C947522AB
:105900000E94431F20E030E0A901C701B6010F94B7
:10591000AE2A87FF15C0C12CD12C760121C020E012
:1059200030E04CE053E4C701B6010F94DE331816A3
:10593000E4F6C12CD12C9CE0E92E93E4F92ED5CFCE
:1059400020E030E046E953E4C701B6010F94DE33AE
:10595000181634F4C12CD12C86E9E82E83E4F82EF5
:10596000C701B6010F94EB33CB01FF90EF90DF90AE
:10597000CF900C94371F90919F0C977081E09730D7
:1059800009F080E008952091990520FF14C020E8D7
:105990003EE3629FA001639F500D729F500D112442
:1059A000CA019695879596958795009731F08A95C7
:1059B0000000E9F708950C9423260895CF93DF9310
:1059C00010925E0C1092F10C1092F30C1092F20CEB
:1059D0001092980510929705CFEFDFEF8091A814F1
:1059E00085FD07C00E947FADD0932713C093261377
:1059F000F5CF8FEF9FEF9093271380932613DF91BE
:105A0000CF9108958F929F92AF92BF92CF92DF92E3
:105A1000EF92FF920F931F93CF93DF9310924C0559
:105A200010924B052FE320934605109245051092E6
:105A300044051092430510924705109248051092B4
:105A4000490510924A059C01F90190812F5F3F4F53
:105A50009032D1F39E34C9F4818190ED980F9A3041
:105A600020F08D3211F08B3281F432969F012F5F3E
:105A70003F4F808180538A3008F47BC09F012F5FA5
:105A80003F4F8081803209F476C0F093A207E09303
:105A9000A1078F010F5F1F4FC0816AE270E0C8014C
:105AA0000F94CC34009731F0FC0131978081803223
:105AB000E1F31182CD3429F0C43519F0C73409F06F
:105AC0004BC0F80180810F5F1F4F8032D1F38053AC
:105AD0008A3008F041C0C093460530E020E04AE03B
:105AE000DF011196429FC001439F900D11249C013C
:105AF000205331098081280F311D87FD3A9581811E
:105B000090ED980F9A30C8F13093450520934405E5
:105B10008E3261F4329690E04AE0DF0131968C914A
:105B200050ED580F5A3058F190934305CD01DC01E8
:105B300001964C914032D9F3CD3489F52E3131059F
:105B400039F018F52731310519F02C31310539F5C7
:105B5000B0934C05A0934B05DF91CF911F910F910E
:105B6000FF90EF90DF90CF90BF90AF909F908F907D
:105B70000895F9017BCFF90181CFFD01B1CF949F49
:105B8000800D112490ED980FC8CF2537310538F0DE
:105B900027373105E8F2203A83E03807C9F2D0917F
:105BA000A10740E050E0BA0110E000E0C12CD12C88
:105BB0007601C394FD0131968C91882309F47FC04E
:105BC0008132E1F4CD34D1F420323105B9F440937F
:105BD0004705509348056093490570934A05F09333
:105BE0004C05E0934B0563E270E0CF010F94CC3499
:105BF000009709F4B1CFFC011082AECF81548A31F5
:105C000008F058C0DF019D91903291F0A0EDA90FEE
:105C1000AA30E8F09E3271F4918190539A30B8F036
:105C20000115110519F48F010150110990E013C0FD
:105C3000FD01E8CF9D3211F09B3291F79181A0EDEB
:105C4000A90FAA3020F09E3259F79281E6CF9E2FFD
:105C50009D1B309759F3A82FB0E04601570104C0AF
:105C6000880C991CAA1CBB1C8A95D2F74829592973
:105C70006A297B29A75DBA4F9C9380818154DF01FB
:105C80008A3108F497CFDF018191882309F492CFFC
:105C900090ED980F9A30B8F393ED980F923098F3F7
:105CA0008B3289F3CD010196EC91E03209F082CF7D
:105CB000DC01F8CF0115110501F78D01DECF10933E
:105CC0004C0500934B05409347055093480560935E
:105CD000490570934A0540CF4F925F926F927F9231
:105CE0008F929F92AF92BF92CF92DF92EF92FF92EC
:105CF000CF93DF9300D000D01F921F92CDB7DEB7B5
:105D00005C01DB01CD90DD90ED90FC90E091EB1219
:105D1000F091EC12FE83ED8384819581A681B78199
:105D200089839A83AB83BC839C01AD01C701B60113
:105D30000F947D312B013C01F50180809180A28080
:105D4000B380AD81BE818D919D910D90BC91A02DB0
:105D50008D839E83AF83B88727E137EB41ED58EB06
:105D6000C301B2010F94DE3387FDD1C023E030E0E0
:105D700044EB53E4C301B2010F94AE2A18160CF49D
:105D8000C6C02D813E814F815885C501B4010F9455
:105D90007D312B013C0127E137EB41ED58EB0F94AE
:105DA000DE3387FDB4C023E030E040EB53E4C301B1
:105DB000B2010F94AE2A18160CF4A9C020E030E00E
:105DC000A9016D817E818F8198850F947E312B0191
:105DD0003C0120E030E040E450E40F94AE2A87FF1D
:105DE00005C0412C512C30E4632E762C27E137EB93
:105DF00041ED58E3C301B2010F947D319B01AC0129
:105E0000C501B4010F94DE3387FD81C020E030E08E
:105E100040EB53E46D817E818F8198850F947E31B4
:105E20002B013C0120E030E84EEA53E40F94DE33CE
:105E300018163CF4412C20E8522E2EEA622E23E460
:105E4000722E27E137EB41ED58E3C301B2010F9405
:105E50007E319B01AC01C501B4010F94AE2A181626
:105E60000CF455C020E030E0A90169817A818B8172
:105E70009C810F947E314B015C0120E030E040EECC
:105E800051E40F94AE2A87FF06C0812C912C90EE2E
:105E9000A92E91E4B92E27E137EB41ED58E3C50176
:105EA000B4010F947D319B01AC01C701B6010F9481
:105EB000DE3387FD2CC020E030E044EB53E4698101
:105EC0007A818B819C810F947E314B015C0120E0B3
:105ED00030E046EA53E40F94DE33181634F4812C94
:105EE000912C86EAA82E83E4B82E27E137EB41ED0A
:105EF00058E3C501B4010F947E319B01AC01B1E0C0
:105F0000B983C701B6010F94AE2A18160CF4198292
:105F1000898128960FB6F894DEBF0FBECDBFDF9102
:105F2000CF91FF90EF90DF90CF90BF90AF909F9078
:105F30008F907F906F905F904F900895EDE2F8E022
:105F400082EBDF011D928A95E9F708958091E005C3
:105F5000811104C00E949E2F0C94E0BA8091A81475
:105F600082FD0D945D19089580912D08882361F0BC
:105F70009091DE08891308C08091A81483FF04C0A3
:105F80008BE698E00C94AAB980E00895FC01238187
:105F900021110C94DFB50895EFE6F0E08081826076
:105FA00080830895CF92DF92EF92FF92CF93DF9399
:105FB000C82F0E94232A94E0C99FE0011124FE010A
:105FC000ED5EF94FC080D180E280F38081110E94A4
:105FD000CC2FC353DE4EC701B6010F94B52A2881DA
:105FE00039814A815B810F94142BDF91CF91FF900F
:105FF000EF90DF90CF9008958F929F92AF92BF92D3
:10600000CF92DF92EF92FF921F93CF93DF93CDB7A2
:10601000DEB760970FB6F894DEBF0FBECDBF182F66
:1060200080E00E94D22F4B015C0180929F059092EC
:10603000A005A092A105B092A20581E00E94D22FF6
:106040006B017C01C092A305D092A405E092A50546
:10605000F092A60582E00E94D22F6093A70570936C
:10606000A8058093A9059093AA051D861E861F8604
:10607000188A89829A82AB82BC82CD82DE82EF82CC
:10608000F88669877A878B879C8783E00E94D22F66
:106090006D877E878F87988B8091A00C882321F055
:1060A000CE0101960E9439211E3FD9F480E1FE0104
:1060B0003196A9E6B2E001900D928A95E1F76096DB
:1060C0000FB6F894DEBF0FBECDBFDF91CF911F9109
:1060D000FF90EF90DF90CF90BF90AF909F908F9008
:1060E000089584E0189FF0011124DF01A759BD4FE6
:1060F00081E090E08C0F9D1FE80FF91F40815181D6
:10610000628173814D935D936D937C931397D7CF89
:10611000CF92DF92EF92FF92CF93DF93C82F0E942E
:10612000232A94E0C99FE0011124FE01E95FF94FA1
:10613000C080D180E280F38081110E94CC2FC353B4
:10614000DE4EC701B6010F94B52A288139814A81F4
:106150005B810F94142BDF91CF91FF90EF90DF9034
:10616000CF9008950E94232A9091F1129093F012FB
:106170009093EF129093EE1294E69093ED1220ED2F
:1061800033E0309324092093230981110E94CC2FFE
:1061900081E0809306060895CF93DF93CDB7DEB7F5
:1061A0002C970FB6F894DEBF0FBECDBF0F947A18B0
:1061B0000E94232A9CE0E3E1F6E0DE0111960190C3
:1061C0000D929A95E1F781110E94CC2FCE01019694
:1061D0000E944ACD2C960FB6F894DEBF0FBECDBFFD
:1061E000DF91CF9108952F923F924F925F926F92DD
:1061F0007F928F929F92AF92BF92CF92DF92EF9257
:10620000FF920F931F93CF93DF9300D0CDB7DEB7EC
:106210008090690290906A02A0906B02B0906C022C
:1062200040906D0250906E0260906F02709070020C
:10623000C0907102D0907202E0907302F0907402EC
:106240000E94CC1B0E941A1C0BEA1CE18FE492E016
:106250009B838A838FE9282E8CE1382E19828981CD
:106260000E94BD1CC8010E94A01DEA81FB816193B0
:10627000719381939193FB83EA83C1010E94A01DD6
:10628000EA81FB816087718782879387F981FF5F4D
:10629000F9830C5F1F4F84E0280E311CF330F9F6B0
:1062A00081EF95E00F94DF180E94BC1E0E94012729
:1062B000A50194016091690270916A0280916B025C
:1062C00090916C020F94AE2A81111CC0A30192011F
:1062D00060916D0270916E0280916F0290917002D8
:1062E0000F94AE2A81110EC020917102309172027A
:1062F0004091730250917402C701B6010F94AE2A07
:106300008823B9F00F900F900F90DF91CF911F91DC
:106310000F91FF90EF90DF90CF90BF90AF909F9044
:106320008F907F906F905F904F903F902F900C9444
:10633000CC300F900F900F90DF91CF911F910F9164
:10634000FF90EF90DF90CF90BF90AF909F908F9095
:106350007F906F905F904F903F902F900895809125
:10636000E1119091E211892B79F48091E1119091E2
:10637000E211892B49F42091E1113091E21181E081
:10638000232B19F480E0089581E008951092FD0414
:106390008091220290912302A0912402B0912502C3
:1063A0008093FD059093FE05A093FF05B093000632
:1063B00008959091F8111092F811923071F0943084
:1063C00079F0913099F4813089F48091FD0488232B
:1063D00069F0109226020C94C63110929E0C08951A
:1063E00082EB98E19093EE0C8093ED0C08959091E0
:1063F000A81493FB882780F993FF06C081E0909151
:106400000F16911101C080E00895CF93C0919A05B5
:10641000CF7739F50E94F731882319F18091A014C4
:106420009091A114A091A214B091A3140097A1057A
:10643000B105B9F0BC01CD016D597F4F8F4F9F4F12
:1064400024E630E040E050E00F94F2306091A41474
:106450007091A5148091A6149091A7140F94F23016
:10646000C22F8C2FCF910895E0E2F9E010821182C3
:10647000089581E00895DC01EC918E2F90E0FC01FD
:10648000EE0FFF1FE80FF91FED56FD4E80818F774D
:10649000808308958F929F92AF92BF92CF92DF92A6
:1064A000EF92FF920F93CF93DF931F92CDB7DEB79A
:1064B0005C017B0149016B01C40ED51EF501808191
:1064C00091810F94CC308983002311F0F7018083F0
:1064D000BE016F5F7F4FC4010E944FE9F5018081CB
:1064E0009181019691838083FFEFEF1AFF0AEC14EC
:1064F000FD0421F780E00F90DF91CF910F91FF9085
:10650000EF90DF90CF90BF90AF909F908F900895C5
:106510000F93AB010091F50521E0022726EF35E04E
:10652000BC0186ED95E00E944A320F9108950097D4
:1065300081F41092900082E0809391001092950077
:1065400010929400C19A80917100826080937100D2
:106550000895019761F41092A00082E08093A10059
:106560001092A5001092A40089BB80937200089538
:106570007F928F929F92AF92BF92CF92DF92EF92D3
:10658000FF920F931F93CF93DF93EC017B018881E0
:10659000883108F0C3C090E0FC01EE0FFF1FE80F48
:1065A000F91FED56FD4E80818F770E943BF01982D6
:1065B0001A8288812CE0622F0F945531829FB0019E
:1065C000112430E020E0AB01420F531FFA01EE0F1F
:1065D000FF1FE40FF51FED56FD4E908197FD08C09B
:1065E0002F5F3F4F2C30310571F790E00E949732BA
:1065F0007880072D10E06801CC0CDD1CF601E00F5F
:10660000F11FED56FD4E80818068808377FC86C047
:1066100080E2E81682E0F8060CF03FC08A8128E5A7
:1066200032E0281B310987FD3395220F331F220FDB
:10663000331F032E000C440B550B898178E8872EFD
:10664000912C881A910887FD9394880C991C880CCA
:10665000991C092C000CAA08BB0860E070E0CB0173
:10666000F7FC0AC0B701653B710514F064EB70E0FC
:10667000072E000C880B990B281939094A095B0968
:106680000F94E23024EB30E040E050E00F941431FE
:10669000820E931EA41EB51E740187E18715D8F0E3
:1066A000298188E890E0821B910927FD9395880F46
:1066B000991F880F991FE816F90604F502972FB75E
:1066C000F894E601C00FD11FCD56DD4E880F991FFB
:1066D0009A8389832FBF62E370E080E090E0DF91CE
:1066E000CF911F910F91FF90EF90DF90CF90BF90CF
:1066F000AF909F908F907F900C9423262A8188E5FD
:1067000092E0821B910927FD9395880F991F880FAE
:10671000991FE816F90694F6C701D0CFDF91CF9103
:106720001F910F91FF90EF90DF90CF90BF90AF90AF
:106730009F908F907F900895CF93DF93EB01682F08
:1067400070E08CED92E10E94B832688179818A8193
:106750009B81643F21E072078105910520F464EF7D
:1067600071E080E090E00E94232689B183FB8827B6
:1067700080F9DF91CF910895CF93DF9300D01F92DE
:10678000CDB7DEB78EEE92E0A0E0B0E089839A83C9
:10679000AB83BC83BE016F5F7F4F8AE50E949C3351
:1067A0000F900F900F900F90DF91CF910895CF939E
:1067B000DF9300D01F92CDB7DEB78EEE92E0A0E05F
:1067C000B0E089839A83AB83BC83BE016F5F7F4F48
:1067D0008AE00E949C330F900F900F900F90DF91F2
:1067E000CF910895CF93DF9300D01F92CDB7DEB73E
:1067F00084EF91E0A0E0B0E089839A83AB83BC830F
:10680000BE016F5F7F4F80EA0E949C330F900F9014
:106810000F900F90DF91CF9108951F920F920FB6B6
:106820000F9211240BB60F922F933F934F935F93C8
:106830006F937F938F939F93AF93BF93EF93FF9348
:1068400048EA50E064EA70E081E090E00E94472668
:10685000FF91EF91BF91AF919F918F917F916F9138
:106860005F914F913F912F910F900BBE0F900FBEF4
:106870000F901F9018951F920F920FB60F92112430
:106880000BB60F922F933F934F935F936F937F932A
:106890008F939F93AF93BF93EF93FF9348E950E09B
:1068A00064E970E090E080E00E944726FF91EF915C
:1068B000BF91AF919F918F917F916F915F914F9118
:1068C0003F912F910F900BBE0F900FBE0F901F9016
:1068D00018959091D10095FD0CC09091D00095FF36
:1068E00008C08093D6008091D00080648093D0004F
:1068F000089520912A042F5F2F770FB607FC27C039
:1069000090912B04921328C09091D00095FF1EC047
:1069100090912B0440912A04941306C09091D100C9
:106920009F7D9093D10012C0E92FF0E0E65DFB4F10
:1069300032819F5F9F773093D60090932B043091E4
:10694000D00030643093D000491741F3D9CF9091F3
:106950002B04921301C0FBCFE0912A04F0E0E65D26
:10696000FB4F828320932A048091D1008062809320
:10697000D10008958F929F92AF92BF92CF92DF92F3
:10698000EF92FF920F931F93CF93DF937C0121E54A
:10699000E20EF11CD7014C914A3509F0A4C06C01FC
:1069A000B2E5CB0ED11CF6013081353A09F09BC01F
:1069B000EC01C05BDF4F2881233008F494C08C01C8
:1069C00000561F4FD8014C93E15BFF4F3083319647
:1069D0002083EF54F1093081E05BFF4F3083303882
:1069E000B1F43196AC54B1093C913083E854F109CB
:1069F000AF5ABF4F50E040E02250330B42175307CD
:106A0000CCF4808132968D934F5F5F4FF7CF233068
:106A100031F5313809F074C0FC01EC55FF4FDC0151
:106A2000AC5ABF4F2C9120833196885A9F4FDC017E
:106A30008C9180834801B12CA12C888190E0029632
:106A40008A159B050CF43FC0F40181914F010E940F
:106A500069340E9492E9FFEFAF1ABF0AEECF3238D5
:106A600021F5FC01EC5AFF4F30814181E05BFF4F83
:106A7000408331963083DC01AA55BF4F50E040E09F
:106A80002350330B42175307ACF6FA01EE7FE45A5A
:106A9000FF4FE80FF91F608171817C9311966C9311
:106AA00011974E5F5F4F1296EDCF243019F63338B1
:106AB00009F6FC01EC5AFF4F20813181E05BFF4F6A
:106AC00030833196B0CF80E5DE011D928A95E9F7DB
:106AD0008AE1F80111928A95E9F78AE5D7018C934A
:106AE00085EAF6018083DF91CF911F910F91FF908E
:106AF000EF90DF90CF90BF90AF909F908F900895D0
:106B0000323809F097CFADCFAF92BF92CF92DF92DC
:106B1000EF92FF920F931F93CF93DF93EC0184E6E4
:106B2000C82E80E2D82EE12CF12C02E8A12C90E2B4
:106B3000B92E15E000933514C0923614D092371454
:106B4000E0923814F0923914B0923F14A0923E149F
:106B50001093321482EE93E10E94BA348FEFC81A78
:106B6000D80AE80AF80A88E7C81680E2D806E104DD
:106B7000F10401F724E630E240E050E0BE0182EE8D
:106B800093E1DF91CF911F910F91FF90EF90DF90F4
:106B9000CF90BF90AF900C9497E9CF92DF92EF9295
:106BA000FF920F931F93CF93DF93CDB7DEB77C0196
:106BB000CDB6DEB60F94FB2901962DB73EB7281B44
:106BC000390B0FB6F8943EBF0FBE2DBF0DB71EB7E1
:106BD0000F5F1F4FB701C8010F94F429F80101900E
:106BE0000020E9F73197E01BF10B759720F083E95E
:106BF00092E0F801848BC8010E9484350FB6F894A6
:106C0000DEBE0FBECDBEDF91CF911F910F91FF90E1
:106C1000EF90DF90CF9008958F929F92AF92BF92A6
:106C2000CF92DF92EF92FF920F931F93CF93DF9358
:106C30000E94DE2C3AE0C32E30E2D32EE12CF12C60
:106C400015E002E846015701CAE0D0E010923F1477
:106C500010923E141093321400933514809236141F
:106C600090923714A0923814B092391482EE93E1C6
:106C70000E94BA3421978FEF881A980AA80AB80A96
:106C8000209721F78AE0C80ED11CE11CF11C82ED8F
:106C9000C81680E2D806E104F104A1F6C12C20E276
:106CA000D22EE12CF12CD5E0C2E810923F141092C4
:106CB0003E14D0933214C0933514C0923614D0923F
:106CC0003714E0923814F092391482EE93E10E9466
:106CD000BA3410923F1410923E14D0933214C093E1
:106CE0003514D701C6018C529F4FAF4FBF4F8093D1
:106CF000361490933714A0933814B093391482EE5D
:106D000093E10E94BA348FEFC81AD80AE80AF80A49
:106D10008AE0C81680E2D806E104F10431F69EED5F
:106D2000C92E90E2D92EE12CF12CD5E0C2E81092C8
:106D30003F1410923E14D0933214C0933514C09275
:106D40003614D0923714E0923814F092391482EE4F
:106D500093E10E94BA348FEFC81AD80AE80AF80AF9
:106D600086EEC81680E2D806E104F10401F7CC24CF
:106D7000C39482E1D82EE12CF12C0AE010E0D5E09A
:106D8000C2E810933F1400933E14D0933214C09382
:106D90003514C0923614D0923714E0923814F09221
:106DA000391482EE93E10E94BA3410933F14009399
:106DB0003E14D0933214C0933514D701C601809687
:106DC000A11DB11D8093361490933714A0933814ED
:106DD000B093391482EE93E10E94BA348FEFC81A4F
:106DE000D80AE80AF80A85E1C81682E1D806E10463
:106DF000F10439F682E190E090933F1480933E14C1
:106E0000D0933214C093351484E190E1A0E0B0E057
:106E10008093361490933714A0933814B093391498
:106E200082EE93E1DF91CF911F910F91FF90EF9050
:106E3000DF90CF90BF90AF909F908F900C94BA341A
:106E40001F920F920FB60F9211240BB60F922F9331
:106E50008F939F93EF93FF9380912B0420912A04AB
:106E6000821306C08091D1008F7D8093D10012C023
:106E7000E82FF0E0E65DFB4F92818F5F8F77909374
:106E8000D60080932B049091D00090649093D00012
:106E9000281741F3FF91EF919F918F912F910F90C0
:106EA0000BBE0F900FBE0F901F9018951F920F9260
:106EB0000FB60F9211240BB60F920F931F932F93BF
:106EC0003F934F935F936F937F938F939F93AF9372
:106ED000BF93CF93DF93EF93FF93C091D6000091C0
:106EE0004E05D0914D0511E01D0F1F73909129049F
:106EF000913108F09FC0E92FF0E08827ED57F84C5A
:106F00008F4F0D9475319437C337D237E137E83757
:106F10001A38EC371A38F037F4371A38F837FC37A4
:106F2000003807381A381238C03229F028F5CA302C
:106F300011F0CD3031F5011731F0ED2FF0E0E35BCA
:106F4000FA4FC283D12FD0934D05FF91EF91DF917E
:106F5000CF91BF91AF919F918F917F916F915F91F1
:106F60004F913F912F911F910F910F900BBE0F905A
:106F70000FBE0F901F901895CD3481F081E0CE3474
:106F800071F080E10CC0CA3338F4C033A0F6C032CF
:106F900091F2CD32B1F7CFCFCD3499F782E0809323
:106FA0002904C9CFC13359F018F4C03221F2E9CF16
:106FB00088E0C433A1F38BE0C83389F3E2CF83E0E8
:106FC000EECF84E0C03359F386E0C13341F3D9CF2B
:106FD00085E0C833B1F6E3CF87E0C23391F6DFCF67
:106FE00089E0C13371F6DBCF8AE0C03351F6D7CFE9
:106FF0008CE0C73331F6D3CF8DE0C63311F6CFCF57
:10700000C03209F498CF8EE0C33549F2BACF80ED93
:107010008C0F8A3008F08FCF9FE0909329048093E3
:10702000280489CFCA3019F0CD3009F084CF1092EE
:10703000290481CFCA3019F0CD3009F07CCF80917E
:107040009C148823A1F3973089F038F4953079F7B0
:107050001092440210929E0CEACF9A3059F09F3061
:1070600031F7809128040E94D931E1CF81E08093EB
:107070002406DDCF81E080932306D9CF9091C00014
:1070800095FFFCCF8093C6000895CF93DF93EC016A
:107090008991882319F00E943E38FACF8DE00E9432
:1070A0003E388AE0DF91CF910C943E38CF92DF9248
:1070B000EF92FF92CF936B017C01C42F4A3069F4A9
:1070C000F7FE0BC0F094E094D094C094C11CD11C86
:1070D000E11CF11C8DE20E943E384C2FC701B60125
:1070E000CF91FF90EF90DF90CF900C9418ADCF939D
:1070F000DF93EC01FE0184912196882319F00E9410
:107100003E38F8CFDF91CF910895CF93DF93D091A0
:107110008B1187E89CE10E9477388AE00E943E3814
:1071200080910A0D873009F449C083E08093080DEF
:1071300081E08093860280E190E090933F148093F9
:107140003E1485E080933214C2E8C093351484E184
:1071500090E1A0E0B0E08093361490933714A093B0
:107160003814B093391482EE93E10E94BA3461E08E
:1071700070E080E090E00E94C32C81E09AE590935B
:107180003F1480933E1485E390E0909341148093E4
:10719000401487E080933214C093351484E890E063
:1071A000A0E0B0E08093361490933714A093381485
:1071B000B093391482EE93E10E94BA3480918B111E
:1071C000813089F1823061F50E94B02B6093BE0559
:1071D0007093BF058093C0059093C10581E08093B3
:1071E0008B110E94D2A96093BA057093BB0580935E
:1071F000BC059093BD05D23089F08091A70690918F
:10720000A80601969093A8068093A7061092C6053B
:107210001092C7051092C8051092C90581E004C0FC
:107220000E94E22BDBCF80E0DF91CF910895CF93D6
:10723000C82FCB010E9477388BEF98E10E947738F6
:107240008CEE98E1CC2311F081EF98E10E94773821
:107250008AE0CF910C943E38CF93DF9300D01F92F9
:10726000CDB7DEB784EF91E0A0E0B0E089839A83E8
:10727000AB83BC83BE016F5F7F4F8CE30E949C3366
:1072800089E199E10E9477388CB163E179E185FB6E
:10729000882780F90E941739809103016DE079E118
:1072A000869581700E94173989B167E079E183FB87
:1072B000882780F90E9417398CB16EEF78E18295AA
:1072C00081700E9417394B9909C00E94D7330F90E3
:1072D0000F900F900F90DF91CF9108950E94BC33D3
:1072E0000F900F900F900F90DF91CF9108958091A4
:1072F0008B118130C1F587EC98E10E9477388AE0E4
:107300000E943E3881E09AE590933F1480933E14AA
:1073100087E590E0909341148093401487E0809338
:10732000321482E88093351484E890E0A0E0B0E065
:107330008093361490933714A0933814B093391473
:1073400082EE93E10E94BA3482E080938B110E9416
:10735000D2A96093C2057093C3058093C40590932E
:10736000C50581E0089580E008950F931F930E9462
:10737000D2A90091A2061091A3062091A4063091F3
:10738000A506011511052105310509F067C02091F9
:107390001413222309F45FC0E091121321502093AB
:1073A000141321E02E0F2093121330911513231381
:1073B00002C01092121324E0E29FF0011124EA5E51
:1073C000FC4E008111812281338100939E0610932F
:1073D0009F062093A0063093A106600F711F811DA8
:1073E000911D6093A2067093A3068093A4069093C8
:1073F000A5068091A0069091A106892B61F11FB787
:10740000F89486EB98E10E9477388AE00E943E3833
:1074100084E096E090933F1480933E1480EA90E8D5
:10742000909341148093401487E08093321482E853
:107430008093351480EA90E0A0E0B0E080933614A9
:1074400090933714A0933814B093391482EE93E1DB
:107450000E94BA341FBF1F910F910895601B710BDA
:10746000820B930B97FDF7CF40981092A2061092D3
:10747000A3061092A4061092A506EDCF0F931F93BA
:10748000CF93DF938C01EB0190911413209115138E
:10749000921305C00E94B5390E94E0C4F5CF8091D7
:1074A000131334E0839FF0011124EA5EFC4E118334
:1074B0000083D383C2839F5F909314138F5F281739
:1074C00039F080931313DF91CF911F910F9108959D
:1074D00010921313F8CFCF92DF92EF92FF921F9387
:1074E000CF93DF93182F662351F01092FC04109273
:1074F000F8041092F9041092FA041092FB040E940E
:10750000D2A96B017C018091F8049091F904A091BB
:10751000FA04B091FB04A7019601281B390B4A0B12
:107520005B0BDA01C901B7FD3DC02091FC0417FDDA
:1075300013C0412F012E000C550B4C5F5F4F822F63
:10754000022E000C990B4817590764F184EF91E063
:10755000A0E0B0E0211724F488EE93E0A0E0B0E0D2
:107560008C0D9D1DAE1DBF1D8093F8049093F904F2
:10757000A093FA04B093FB042170C22F30E0D32F04
:1075800084E28C9FB0018D9F700D7C1B112460598B
:107590007C4F82E390E00E943E3A8091FC048F5F32
:1075A0008093FC04DF91CF911F91FF90EF90DF90CB
:1075B000CF900895CF93DF9300D01F92CDB7DEB761
:1075C0008CE398E10E9477388AE00E943E388091EF
:1075D0000A0D8330D9F119821A821B821C8260E065
:1075E000CE0101960E94FD2B19821A821B821C82F9
:1075F00061E0CE0101960E94FD2B81E0809385021F
:107600001092070D8093860281E09AE590933F14D3
:1076100080933E1483E390E0909341148093401450
:1076200087E08093321482E88093351484E890E0F8
:10763000A0E0B0E08093361490933714A0933814F0
:10764000B093391482EE93E10E94BA340F900F90F8
:107650000F900F90DF91CF9108956F927F928F924C
:107660009F92AF92BF92CF92DF92EF92FF920F93D1
:107670001F93CF93DF93CDB7DEB764970FB6F8941F
:10768000DEBF0FBECDBF1092D0008091D0008260CF
:107690008093D0001092D50080E18093D400809137
:1076A000D10080618093D1008091D1008860809367
:1076B000D1008091D10080688093D1008091D10069
:1076C0008F7D8093D1008AE5809333148093E313F8
:1076D00085EA809334148093E413E2E8F4E18AE1CC
:1076E000DF011D928A95E9F78091060D882309F440
:1076F00074C283E090E090933F1480933E1485E041
:107700008093321482E8809335148FE190E1A0E0F9
:10771000B0E08093361490933714A0933814B0934C
:10772000391482EE93E10E94BA3484E690E090939B
:107730003F1480933E1405E00093321412E8109336
:10774000351486E090E1A0E0B0E080933614909389
:107750003714A0933814B093391482EE93E10E9449
:10776000BA348BE090E090933F1480933E140093E2
:1077700032141093351480E092E1A0E0B0E08093E1
:10778000361490933714A0933814B093391482EEC2
:1077900093E10E94BA3410923F1410923E14009369
:1077A00032141093351484E390E1A0E0B0E08093AC
:1077B000361490933714A0933814B093391482EE92
:1077C00093E10E94BA3410923F1410923E14009339
:1077D0003214109335148AE390E1A0E0B0E0809376
:1077E000361490933714A0933814B093391482EE62
:1077F00093E10E94BA348091521290915312909367
:107800003F1480933E14009332141093351486E392
:1078100090E1A0E0B0E08093361490933714A093E9
:107820003814B093391482EE93E10E94BA348091F7
:10783000E7119091E81190933F1480933E140093C8
:107840003214109335148CE390E1A0E0B0E0809303
:10785000361490933714A0933814B093391482EEF1
:1078600093E10E94BA3482E090E090933F148093B9
:107870003E1400933214109335148EE190E1A0E091
:10788000B0E08093361490933714A0933814B093DB
:10789000391482EE93E10E94BA3481E0809385022C
:1078A00070E6C72E70E1D72EE12CF12C10923F1418
:1078B00010923E140093321410933514C092361473
:1078C000D0923714E0923814F092391482EE93E19A
:1078D0000E94BA34BFEFCB1ADB0AEB0AFB0AE4E7DB
:1078E000CE16E0E1DE06E104F10401F7CE010196D7
:1078F0007C0184E1D7011D928A95E9F781E08F939D
:1079000090E99F938F9390E69F938F9388E68F9350
:1079100085EA93E09F938F93FF92EF920F94063541
:1079200020E630E140E050E062EB73E082EE93E16C
:107930000E9497E92AE630E140E050E06FEB73E007
:1079400082EE93E10E9497E924E730E140E050E0C5
:10795000B70182EE93E10E9497E92EE730E140E023
:1079600050E06BEC73E082EE93E10E9497E9109295
:107970003F1410923E1400933214109335148EE08D
:1079800090E1A0E0B0E08093361490933714A09378
:107990003814B093391482EE93E10E94BA341092F5
:1079A0003F1410923E1400933214109335148FE05C
:1079B00090E1A0E0B0E08093361490933714A09348
:1079C0003814B093391482EE93E10E94BA340FB6A2
:1079D000F894DEBF0FBECDBF4AE0C42E40E2D42EE5
:1079E000E12CF12C55E0752E62E8662E4601570118
:1079F0000AE010E010923F1410923E14709232147C
:107A0000609235148092361490923714A0923814F4
:107A1000B092391482EE93E10E94BA3401501109F8
:107A2000FFEF8F1A9F0AAF0ABF0A0115110511F760
:107A30008AE0C80ED11CE11CF11C92EDC91690E23F
:107A4000D906E104F10491F6C12C30E2D32EE12CE9
:107A5000F12C05E012E810923F1410923E140093AE
:107A6000321410933514C0923614D0923714E09229
:107A70003814F092391482EE93E10E94BA341092D5
:107A80003F1410923E140093321410933514D70112
:107A9000C6018C529F4FAF4FBF4F809336149093C7
:107AA0003714A0933814B093391482EE93E10E94F6
:107AB000BA34AFEFCA1ADA0AEA0AFA0ABAE0CB16FF
:107AC000B0E2DB06E104F10431F62EEDC22E20E235
:107AD000D22EE12CF12C05E012E810923F14109206
:107AE0003E140093321410933514C0923614D09281
:107AF0003714E0923814F092391482EE93E10E9428
:107B0000BA34EFEFCE1ADE0AEE0AFE0AF6EECF1610
:107B1000F0E2DF06E104F10401F7CC24C39482E132
:107B2000D82EE12CF12C9AE0A92EB12C05E012E818
:107B3000B0923F14A0923E14009332141093351467
:107B4000C0923614D0923714E0923814F09239145F
:107B500082EE93E10E94BA34B0923F14A0923E1498
:107B60000093321410933514D701C6018096A11DDD
:107B7000B11D8093361490933714A0933814B093AA
:107B8000391482EE93E10E94BA348FEFC81AD80AF2
:107B9000E80AF80A95E1C91692E1D906E104F10470
:107BA00039F682EA97E10E9477388AE00E943E38EF
:107BB00064960FB6F894DEBF0FBECDBFDF91CF91B4
:107BC0001F910F91FF90EF90DF90CF90BF90AF90FB
:107BD0009F908F907F906F90089582E090E08BCD82
:107BE0000E942D3B1092960581E08093860284E5E9
:107BF00098E10E9477388AE00C943E380F931F93E7
:107C0000CF938C01C62F8EE294E10E947738C80191
:107C10000E9477388AE30E943E3880E38C0F0E94EE
:107C20003E388AE0CF911F910F910C943E3881EB42
:107C300095E10E94773860E081EA95E10E94FE3D7F
:107C400060E08CE895E10E94FE3D61E085E895E109
:107C50000E94FE3D61E08AE795E10E94FE3D61E001
:107C60008AE695E10E94FE3D60E081E695E10E9492
:107C7000FE3D61E087E595E10E94FE3D61E08DE417
:107C800095E10E94FE3D61E086E495E10E94FE3DA3
:107C900061E08EE395E10E94FE3D61E080E395E1C5
:107CA0000E94FE3D61E082E295E10E94FE3D60E0BF
:107CB00083E195E10E94FE3D60E085E095E10E9450
:107CC000FE3D60E08FEE94E10E94FE3D61E08EEDAE
:107CD00094E10E94FE3D61E08FEC94E10E94FE3D44
:107CE00061E088EC94E10E94FE3D60E081EC94E16B
:107CF0000E94FE3D61E088EB94E10E94FE3D61E060
:107D000083EA94E10E94FE3D61E085E994E10E94EE
:107D1000FE3D61E082E894E10E94FE3D60E085E77F
:107D200094E10E94FE3D61E080E794E10E94FE3D07
:107D300061E083E694E10E94FE3D60E08FE494E11F
:107D40000E94FE3D60E08CE394E10E94FE3D60E015
:107D50008BEA94E10E94831D682F617083E394E1B4
:107D60000C94FE3D80914705827149F4809149054C
:107D70008C7829F480914A05837009F475C082E4F7
:107D80000E94611E882351F00E942F246093B50C3D
:107D90007093B60C8093B70C9093B80C83E50E9457
:107DA000611E882351F00E94B5246093E50C709306
:107DB000E60C8093E70C9093E80C84E50E94611E2A
:107DC000882351F00E94B5246093E90C7093EA0C6B
:107DD0008093EB0C9093EC0C88E50E94611E882345
:107DE00051F00E94B52460930C0970930D098093A3
:107DF0000E0990930F0989E50E94611E882351F0B6
:107E00000E94B524609310097093110980931209A0
:107E1000909313098AE50E94611E8823B1F00E94A5
:107E2000B5246093140970931509809316099093F3
:107E300017092DEC3CEC4CEC5DE30F94AE2A1816C0
:107E400024F088E99EE00E94773885E40E94611E54
:107E5000882351F00E94B524609318097093190982
:107E600080931A0990931B090895AF92BF92CF9205
:107E7000DF92EF920F931F93CF93DF935B01EA01A1
:107E80006901882309F463C081E99EE00E94773884
:107E9000F501608171818281938146E00E9420BD5D
:107EA000E1100BC088E89EE00E94773868817981F4
:107EB0008A819B8146E00E9420BD81E89EE00E946D
:107EC0007738F601608171818281938143E00E945D
:107ED00020BD8AE79EE00E947738F80160817181B9
:107EE0008281938143E00E9420BD81E79EE00E9451
:107EF0007738F6012081318142815381F801608118
:107F00007181828193810F947D3143E00E9420BD75
:107F1000EE20F9F08AE00E943E388CE59EE00E9457
:107F20007738688179818A819B8146E00E9420BDF3
:107F30008AE00E943E388AE0DF91CF911F910F9135
:107F4000EF90DF90CF90BF90AF900C943E38E1104F
:107F5000E4CFDF91CF911F910F91EF90DF90CF9001
:107F6000BF90AF9008950F931F93CF938C01C62FAE
:107F700089E798E00E947738C8010E947738CC23BF
:107F800031F08AE0CF911F910F910C943E38CF9140
:107F90001F910F9108950E94A3ED10929E0C1092D4
:107FA00044020E94F731882351F08091A81482FD89
:107FB00006C082EB98E19093EE0C8093ED0C61E0AB
:107FC0008BEA98E10E94B33F0C9485380F931F937E
:107FD000CF93DF938C016F3F19F41092CC1160E0C6
:107FE0002091CC11862F062E000C990B281719060C
:107FF00009F08CF56093CC1160E085E798E10E9470
:10800000B33FC8010E9477388AE00E943E38C80119
:108010000F94FB29800F911FEC01C01BD10BC034C2
:10802000D1053CF00197FC012491207C2038D1F34C
:10803000F3CFDD27AE01B8018CE891E10F941C2A43
:10804000C457DE4E18828CE891E1DF91CF911F91E9
:108050000F910C948435DF91CF911F910F9108956A
:1080600010929E0C109244028091A8148064809318
:10807000A81461E083E898E10E94B33F48E958E121
:1080800060EA78E185E00E94B1EB60E08AE898E17F
:108090000C94E63F0F931F93CF938C01C62F60E0A3
:1080A00083E898E00E94B33FC8010E947738CC2350
:1080B00031F08AE0CF911F910F910C943E38CF910F
:1080C0001F910F91089561E08BE898E00C944A406D
:1080D000EF92FF920F931F93CF937C018B01C42FDC
:1080E00060E083E898E00E94B33FC7010E947738C0
:1080F00080E20E943E38C8010E947738CC2319F0F4
:108100008C2F0E943E388AE0CF911F910F91FF90F3
:10811000EF900C943E38DF92EF92FF920F931F93F3
:10812000CF93DF93D82E7B018A01E9010E9463403F
:10813000D092F81140E0B70184E799E00E946840CE
:108140000115110531F040E0B8018DE699E00E947B
:108150006840209731F040E0BE018DE699E00E9432
:10816000684061E088E699E0DF91CF911F910F911F
:10817000FF90EF90DF900C944A40AF92BF92CF9265
:10818000DF92EF92FF920F931F93CF93DF9386EED0
:1081900097E00E947738C0E0D7E0D15021F080E22C
:1081A0000E943E38FACF8C2F0E94EAE9CF5FC5309B
:1081B00099F78AE00E943E380BEA17E0C0E080E2BF
:1081C0000E943E388C2F0E94EAE95801D5E080E2F7
:1081D0000E943E38F501C080D180E280F380A70183
:1081E0009601C701B6010F947034882369F180E2CB
:1081F0000E943E388DE30E943E388DE30E943E3857
:108200008DE30E943E388DE30E943E388DE30E944C
:108210003E38D150F4E1AF0EB11CD111D8CF8AE075
:108220000E943E38CF5F0C5F1F4FC53041F68AE099
:10823000DF91CF911F910F91FF90EF90DF90CF9042
:10824000BF90AF900C943E3820E030E0A901C70108
:10825000B6010F94DE3387FD03C08BE20E943E38E7
:1082600043E0C701B6010E9420BDD3CF811107C0F2
:108270008AEC9EE00E9477388AE00C943E388EECBF
:108280009EE0F8CFCF93DF93EB010E947738CE01C9
:10829000DF91CF910C94A8EACF93C62F0E94773834
:1082A0008C2FCF910C94EAE9CF92DF92EF92FF925C
:1082B0006A017B010E94773842E0C701B601FF9056
:1082C000EF90DF90CF900C9420BDCF92DF92EF9291
:1082D000FF926A017B010E9477384AE0C701B6012C
:1082E000FF90EF90DF90CF900C945638CF93DF93B0
:1082F000EB010E947738CE01DF91CF910C94F1E928
:108300004F925F926F927F928F929F92AF92BF92A5
:10831000CF92DF92EF92FF920F931F93CF93DF9351
:1083200000D000D01F921F92CDB7DEB78091950587
:1083300081110AC480919305909194059C012F5F4F
:108340003F4F30939405209393058E3E924008F45E
:10835000FBC3809152129091531290933F148093DB
:108360003E1405E00093321412E81093351486E3AE
:1083700090E1A0E0B0E08093361490933714A0937E
:108380003814B093391482EE93E10E94BA3480918C
:10839000E7119091E81190933F1480933E1400935D
:1083A0003214109335148CE390E1A0E0B0E0809398
:1083B000361490933714A0933814B093391482EE86
:1083C00093E10E94BA348091541290915512909387
:1083D0003F1480933E14009332141093351484E3B9
:1083E00090E1A0E0B0E08093361490933714A0930E
:1083F0003814B093391482EE93E10E94BA3480911C
:10840000E9119091EA1190933F1480933E140093E8
:108410003214109335148AE390E1A0E0B0E0809329
:10842000361490933714A0933814B093391482EE15
:1084300093E10E94BA3481E08093950510929405EF
:108440001092930580910A0D882339F10E94151D21
:10845000811123C0809192058F5F80939205809156
:108460009205853620F01092920510920A0DE09147
:108470000A0DE150E73008F06AC00E2E000CFF0B29
:108480008827EA5BFD4B8F4F0D94753150429F4218
:108490006B449744D8441045A34210929205DFCF15
:1084A0000E94BB2C882309F452C081E0809386028D
:1084B0008EE298E10E9477388AE00E943E3880E19F
:1084C00090E090933F1480933E1485E080933214A3
:1084D00012E81093351484E190E1A0E0B0E08093BD
:1084E000361490933714A0933814B093391482EE55
:1084F00093E10E94BA3481E09AE590933F1480930F
:108500003E1486E390E0909341148093401487E0FA
:10851000809332141093351484E890E0A0E0B0E02A
:108520008093361490933714A0933814B093391471
:1085300082EE93E10E94BA3410920A0D08C00E94A4
:10854000BB2C882321F00E94151D8823A9F380915C
:108550008602882309F433C7809196058111C0C231
:1085600084E096E090933F1480933E1480EA90E874
:10857000909341148093401417E01093321402E852
:108580000093351480EA90E0A0E0B0E080933614C8
:1085900090933714A0933814B093391482EE93E17A
:1085A0000E94BA348091810290918202A09183024C
:1085B000B09184020097A105B10509F03FC2109265
:1085C0003F1410923E1415E01093321400933514AA
:1085D0008AE890E1A0E0B0E08093361490933714DD
:1085E000A0933814B093391482EE93E10E94BA3408
:1085F00089E090E090933F1480933E1410933214DE
:10860000009335148CE890E1A0E0B0E0809336143C
:1086100090933714A0933814B093391482EE93E1F9
:108620000E94BA348091810290918202A0918302CB
:10863000B09184020097F1E0AF07B10508F441C2A0
:10864000B0933F14A0933E14909341148093401430
:1086500087E08093321482E88093351488E890E1B3
:10866000A0E0B0E08093361490933714A0933814B0
:10867000B093391482EE93E10E94BA348091810262
:1086800090918202A0918302B0918402BA2FA92F07
:10869000982F8827009721E0A207B10508F417C298
:1086A000B0933F14A0933E149093411480934014D0
:1086B00087E08093321412E81093351481EA90E039
:1086C000A0E0B0E08093361490933714A093381450
:1086D000B093391482EE93E10E94BA348091A00CD9
:1086E000882309F4FAC183E090E090933F148093CB
:1086F0003E1485E0809332141093351485E490E1A4
:10870000A0E0B0E08093361490933714A09338140F
:10871000B093391482EE93E10E94BA3480919605A9
:10872000875E8093960520919605822F90E02536EE
:1087300008F021C290933F1480933E1485E080930B
:10874000321482E88093351480E090E1A0E0B0E03C
:108750008093361490933714A0933814B09339143F
:1087600082EE93E10E94BA340E94151D811114C259
:108770000E94F731811105C09091990591FD0E94E9
:10878000151D9091990580FB91F99093990591FDA4
:1087900003C28091A81482FDFFC180918B1181508A
:1087A000823008F4F9C16091E9117091EA11072E45
:1087B000000C880B990B0F94B52A6B017C0120E00B
:1087C00030E0A9010F94AE2A882309F4BBC660915A
:1087D000E7117091E811072E000C880B990B0F948C
:1087E000B52A2B013C0120E030E040E050E4C70115
:1087F000B6010F947D31A30192010F94DE33181658
:108800000CF4C2C66091521270915312072E000CE4
:10881000880B990B0F94B52A6D837E838F8398877D
:108820006091541270915512072E000C880B990B11
:108830000F94B52A4B015C0120E030E040E251E4A6
:108840000F947D312D813E814F8158850F94DE3309
:1088500018160CF499C620E030E040E050E4C7015F
:10886000B6010F947E31A30192010F94AE2A87FDC9
:1088700010C020E030E040E251E4C501B4010F94A3
:108880007E312D813E814F8158850F94AE2A87FF1E
:108890006AC684E190E090933F1480933E1485E093
:1088A0008093321482E88093351484E190E1A0E053
:1088B000B0E08093361490933714A0933814B0939B
:1088C000391482EE93E10E94BA348091080D81112F
:1088D0007CC682E07AC680E298E10E9477388AE01E
:1088E0000E943E3881E09AE590933F1480933E14B5
:1088F00080E490E0909341148093401417E010932B
:10890000321482E88093351484E890E0A0E0B0E06F
:108910008093361490933714A0933814B09339147D
:1089200082EE93E10E94BA3410930A0D10CE80912A
:10893000F70C882309F40BCE0E94BB2C882309F482
:1089400006CE0E94151D811102CE82E198E10E949F
:1089500077388AE00E943E388091F80C90E0B0E0D1
:10896000A0E0895B9F4FAE4FB54A21E03AE53093D6
:108970003F1420933E14909341148093401487E059
:108980008093321482E88093351484E890E0A0E06C
:10899000B0E08093361490933714A0933814B093BA
:1089A000391482EE93E10E94BA341092F70CC4CDD0
:1089B0000E94BB2C882309F4CACD0E94151D811189
:1089C000C6CD81E08093860210920A0D84E098E182
:1089D0000E9477388AE00E943E3881E09AE59093C1
:1089E0003F1480933E148EE490E090934114809362
:1089F000401487E08093321482E88093351484E831
:108A000090E0A0E0B0E08093361490933714A093E8
:108A10003814B093391482EE93E10E94BA3497CDA2
:108A20000E94151D811193CD19821A821B821C820E
:108A300062E0CE0101960F9496007ECD0196A11DB5
:108A4000B11D35E0B695A795979587953A95D1F7DD
:108A50000197A109B1090097E1E0AE07B10548F11E
:108A6000B0933F14A0933E1490934114809340140C
:108A70001093321412E8109335148AE890E1A0E0C4
:108A8000B0E08093361490933714A0933814B093C9
:108A9000391482EE93E10E94BA3488E090E090931A
:108AA0003F1480933E1485E0809332141093351464
:108AB000A9CD90933F1480933E1485E080933214A7
:108AC000D9CF90933F1480933E1485E0C2CD90930C
:108AD0003F1480933E1485E0ECCD82E090E005CE1B
:108AE0008A3F08F020CE8EEF8093960583EF97E1C2
:108AF0000E9477388AE00E943E3881E080938602A7
:108B000081E09AE590933F1480933E148DE290E0CB
:108B1000909341148093401487E08093321482E84C
:108B20008093351484E890E0A0E0B0E080933614A0
:108B300090933714A0933814B093391482EE93E1D4
:108B40000E94BA341092950528960FB6F894DEBFAD
:108B50000FBECDBFDF91CF911F910F91FF90EF908E
:108B6000DF90CF90BF90AF909F908F907F906F904D
:108B70005F904F9008958456910990933F1480938D
:108B80003E1485E08093321482E88093351481E0AE
:108B900090E1A0E0B0E0DCCD8CE090E090933F1459
:108BA00080933E1415E01093321482E880933514BC
:108BB00084E190E1A0E0B0E0809336149093371404
:108BC000A0933814B093391482EE93E10E94BA3422
:108BD0000E94B02B20E13EE040E050E00F94F230E4
:108BE0002115310581E04807510508F470C0509304
:108BF0003F1440933E14309341142093401487E077
:108C00008093321412E81093351480E190E1A0E0D3
:108C1000B0E08093361490933714A0933814B09337
:108C2000391482EE93E10E94BA340E94B02B20E105
:108C30003EE040E050E00F94F2302CE330E040E0C2
:108C400050E00F94F23030933F1420933E1405E02F
:108C5000009332141093351482E190E1A0E0B0E06B
:108C60008093361490933714A0933814B09339142A
:108C700082EE93E10E94BA340E940532882309F4FF
:108C80005CC48F5F80939105E82EF12C833330F51F
:108C9000EE0CFF1CF0923F14E0923E14009332144D
:108CA000109335148EE090E1A0E0B0E0809336148C
:108CB00090933714A0933814B093391482EE93E153
:108CC0000E94BA3410923F1410923E142BC030937D
:108CD0003F1420933E141093321494CF84E690E016
:108CE00090933F1480933E140093321410933514E4
:108CF0008EE090E1A0E0B0E08093361490933714BA
:108D0000A0933814B093391482EE93E10E94BA34E0
:108D1000A2E3EA1AA0E8FA0AEE0CFF1CF0923F1454
:108D2000E0923E1400933214109335148FE090E1DA
:108D3000A0E0B0E08093361490933714A0933814D9
:108D4000B093391482EE93E10E94BA340E94053246
:108D500090E090933F1480933E1485E0809332140A
:108D600082E88093351486E190E1A0E0B0E0809342
:108D7000361490933714A0933814B093391482EEBC
:108D800093E10E94BA3420E030E0A9016091E7123B
:108D90007091E8128091E9129091EA120F947E315D
:108DA00020E030E048EC52E40F94142B0F94EA32A8
:108DB00070933F1460933E1405E00093321412E860
:108DC0001093351486E290E1A0E0B0E08093361471
:108DD00090933714A0933814B093391482EE93E132
:108DE0000E94BA3480917D0290917E0290933F144C
:108DF00080933E14009332141093351480E093E175
:108E0000A0E0B0E08093361490933714A093381408
:108E1000B093391482EE93E10E94BA3420E030E03E
:108E200040E251E46091B90C7091BA0C8091BB0C96
:108E30009091BC0C0F94142B0F94F13270933F144B
:108E400060933E14009332141093351482E492E13F
:108E5000A0E0B0E08093361490933714A0933814B8
:108E6000B093391482EE93E10E94BA3420E030E0EE
:108E700040E251E46091BD0C7091BE0C8091BF0C3A
:108E80009091C00C0F94142B0F94F13270933F14F7
:108E900060933E14009332141093351486E492E1EB
:108EA000A0E0B0E08093361490933714A093381468
:108EB000B093391482EE93E10E94BA3420E030E09E
:108EC00040E251E46091C10C7091C20C8091C30CDE
:108ED0009091C40C0F94142B0F94F13270933F14A3
:108EE00060933E1400933214109335148AE492E197
:108EF000A0E0B0E08093361490933714A093381418
:108F0000B093391482EE93E10E94BA3420E030E04D
:108F100040E251E46091C50C7091C60C8091C70C81
:108F20009091C80C0F94142B0F94F13270933F144E
:108F300060933E1400933214109335148EE492E142
:108F4000A0E0B0E08093361490933714A0933814C7
:108F5000B093391482EE93E10E94BA3420E030E0FD
:108F600048EC52E46091DF127091E0128091E112BE
:108F70009091E2120F94142B0F94EA3270933F14E5
:108F800060933E14009332141093351486E392E1FB
:108F9000A0E0B0E08093361490933714A093381477
:108FA000B093391482EE93E10E94BA3420E030E0AD
:108FB00048EC52E46091E3127091E4128091E51262
:108FC0009091E6120F94142B0F94EA3270933F1491
:108FD00060933E1400933214109335148AE392E1A7
:108FE000A0E0B0E08093361490933714A093381427
:108FF000B093391482EE93E10E94BA3480918D02CD
:1090000090918E0290933F1480933E1400933214FB
:109010001093351482E592E1A0E0B0E0809336141D
:1090200090933714A0933814B093391482EE93E1DF
:109030000E94BA3480918B0290918C0290933F14DD
:1090400080933E14009332141093351484E592E11A
:10905000A0E0B0E08093361490933714A0933814B6
:10906000B093391482EE93E10E94BA3420E030E0EC
:1090700040E251E460915712709158128091591258
:1090800090915A120F94142B0F94F13270933F1455
:1090900060933E14009332141093351486E592E1E8
:1090A000A0E0B0E08093361490933714A093381466
:1090B000B093391482EE93E10E94BA342CEA35EC75
:1090C00047E25EE360915B1270915C1280915D12E9
:1090D00090915E120F94783220E030E040E251E44B
:1090E0000F94142B0F94F13270933F1460933E143D
:1090F00000933214109335148AE592E1A0E0B0E0B9
:109100008093361490933714A0933814B093391485
:1091100082EE93E10E94BA342CEA35EC47E25EE33A
:1091200060915F1270916012809161129091621251
:109130000F94142B20E030E040E251E40F94142B04
:109140000F94F13270933F1460933E1400933214E5
:10915000109335148EE592E1A0E0B0E080933614D0
:1091600090933714A0933814B093391482EE93E19E
:109170000E94BA3420E030E040E251E46091EC110A
:109180007091ED118091EE119091EF110F94142BCD
:109190000F94F13270933F1460933E140093321495
:1091A0001093351482E692E1A0E0B0E0809336148B
:1091B00090933714A0933814B093391482EE93E14E
:1091C0000E94BA342CEA35EC47E25EE36091F0117C
:1091D0007091F1118091F2119091F3110F94783206
:1091E00020E030E040E251E40F94142B0F94F13270
:1091F00070933F1460933E1400933214109335140F
:1092000086E692E1A0E0B0E08093361490933714A4
:10921000A0933814B093391482EE93E10E94BA34CB
:109220002CEA35EC47E25EE36091F4117091F511A0
:109230008091F6119091F7110F94142B20E030E0FB
:1092400040E251E40F94142B0F94F13270933F14C9
:1092500060933E1400933214109335148AE692E121
:10926000A0E0B0E08093361490933714A0933814A4
:10927000B093391482EE93E10E94BA348091010DCB
:10928000811105C08091030D882309F46DC06091A0
:10929000521270915312072E000C880B990B0F94E9
:1092A000B52A20E030E048EC52E40F94142B6B0117
:1092B0007C016091541270915512072E000C880B9E
:1092C000990B0F94B52A9B01AC01C701B6010F940D
:1092D00078320F94F1326536710510F064E670E073
:1092E00070933F1460933E1405E00093321412E82B
:1092F0001093351484E290E1A0E0B0E0809336143E
:1093000090933714A0933814B093391482EE93E1FC
:109310000E94BA346091521270915312072E000CC1
:10932000880B990B0F94B52A6B017C0120E030E08B
:109330004AE253E40F94DE33181624F48091010DB1
:10934000811146C16091541270915512072E000C84
:10935000880B990B0F94B52A9B01AC01C701B6018C
:109360000F94DE3387FFAFC18091F70C882339F16A
:109370008091F60C91E0980F9093F60C90E090930A
:109380003F1480933E1485E08093321482E88093EA
:10939000351482E490E1A0E0B0E08093361490931D
:1093A0003714A0933814B093391482EE93E10E94DD
:1093B000BA348091F60C8A3010F01092F60C0E94AC
:1093C000462C882309F4B5C16091EF0C7091F00C24
:1093D000EE24E394F12C61157105A9F090E080E092
:1093E0000F94B32A20E030E040E85EE30F94142BA2
:1093F0000F945C3220E030E040E85FE30F947E3170
:109400000F94F1327B0101E010E08091F10C8111A9
:1094100002C010E000E080912613909127138F3F47
:10942000980711F40E9475B6909327138093261322
:10943000080F191FB80190E080E00F94B32A20E0D4
:1094400030E040E85EE30F94142B0F945C324B0144
:109450005C01F0923F14E0923E1405E00093321458
:1094600012E81093351480E193E1A0E0B0E080931E
:10947000361490933714A0933814B093391482EEB5
:1094800093E10E94BA34C501B4010F94F132709394
:109490003F1460933E14009332141093351482E10C
:1094A00093E1A0E0B0E08093361490933714A0933A
:1094B0003814B093391482EE93E10E94BA3402E872
:1094C00014E1AAE1FA2E80914D0590914E0520916C
:1094D0008F0530919005891B8F7309F449C12A319A
:1094E00031050CF0DBC190914D0580914E054FEF99
:1094F0005FEF981749F0E82FF0E0E35BFA4F428105
:109500008F5F8F7380934E05F901EE57FB4E4083BA
:10951000809182148A3509F0B3C162E070E080E086
:1095200090E00E94C32C80918F0590919005019648
:109530009093900580938F05C6CF10923F141092A0
:109540003E14ACCB6091541270915512072E000C52
:10955000880B990B0F94B52A20E030E0A9010F94F5
:10956000AE2A811134C98CE090E090933F1480932F
:109570003E1485E08093321482E88093351484E1B0
:1095800090E1A0E0B0E0F3CB8DE090E090933F1449
:1095900080933E1485E08093321482E880933514E2
:1095A00084E190E1A0E0B0E080933614909337140A
:1095B000A0933814B093391482EE93E10E94BA3428
:1095C0008091080D811101C081E08093080DDBCBF3
:1095D0001092010D20E030E040E251E46091F90C7E
:1095E0007091FA0C8091FB0C9091FC0C0F94142B51
:1095F0000F94EA3270933F1460933E140093321438
:109600001093351484E590E1A0E0B0E08093361427
:1096100090933714A0933814B093391482EE93E1E9
:109620000E94BA3420E030E040E251E46091FD0C49
:109630007091FE0C8091FF0C9091000D0F94142BF3
:109640000F94EA3270933F1460933E1400933214E7
:109650001093351488E590E1A0E0B0E080933614D3
:1096600090933714A0933814B093391482EE93E199
:109670000E94BA3482ED97E10E9477388AE00E9416
:109680003E3881E09AE590933F1480933E1481E444
:1096900090E0909341148093401487E080933214BB
:1096A0001093351484E890E0A0E0B0E08093361485
:1096B00090933714A0933814B093391482EE93E149
:1096C0000E94BA3451CE6091030D662309F44CCE4A
:1096D000062E000C770B89EB97E10E9476418AE019
:1096E0000E943E381092030D84E090E090933F1466
:1096F00080933E1485E08093321412E81093351461
:109700008EE890E1A0E0B0E0809336149093371497
:10971000A0933814B093391482EE93E10E94BA34C6
:1097200081E09AE590933F1480933E1483E590E0A6
:10973000B0CF10923F1410923E1405E00093321403
:1097400012E81093351480E193E1A0E0B0E080933B
:10975000361490933714A0933814B093391482EED2
:1097600093E10E94BA3410923F1410923E1493CEAB
:10977000121613060CF492C08091E6139091E71331
:10978000A091E813B091E9138C34E0E19E07A105A4
:10979000B10509F4D7C98A349041A105B10509F48E
:1097A000D1C920E030E040E251E46091690270915B
:1097B0006A0280916B0290916C020F94142B0F94AB
:1097C000EA3270933F1460933E1405E00093321424
:1097D00012E81093351488E490E1A0E0B0E08093A3
:1097E000361490933714A0933814B093391482EE42
:1097F00093E10E94BA3420E030E040E251E460910D
:109800006D0270916E0280916F02909170020F94C0
:10981000142B0F94EA3270933F1460933E1400931C
:109820003214109335148AE490E1A0E0B0E0809304
:10983000361490933714A0933814B093391482EEF1
:1098400093E10E94BA3420E030E040E251E46091BC
:1098500071027091720280917302909174020F9460
:10986000142B0F94EA3270933F1460933E140093CC
:109870003214109335148CE490E1A0E0B0E056C9A6
:10988000121613060CF01FCEF8012F2D11922A95F7
:10989000E9F71092900510928F0515CE9091E31381
:1098A00080918214981321C09091E41380918314C5
:1098B00098131BC023303105C4F090918414909309
:1098C000E213809185148093E5139330D1F4982F9F
:1098D0009D7F9038B1F4909186149F3409F059C05F
:1098E000909187149B3409F054C0E2E8F4E18AE1D6
:1098F000DF011D928A95E9F71092900510928F056D
:109900003BCF833809F045C080918614909187142D
:10991000982789279827B0E0A0E08093E6139093DA
:10992000E713A093E813B093E913C0908814D12CE7
:10993000F12CE12CC092EA13D092EB13E092EC13DD
:10994000F092ED1329E834E140E050E0BA014C1503
:109950005D056E057F0508F04AC0DB01CA01B695BA
:10996000A795979587950696880F991FFC01EE514C
:10997000FC4ED9018C9111969C91892798278927B3
:10998000918380834E5F5F4F6F4F7F4F2E5F3F4FBE
:10999000DECF813861F58091861490E0B0E0A0E0E0
:1099A0008093E6139093E713A093E813B093E91321
:1099B00080918714482F50E070E060E04093EA13F4
:1099C0005093EB136093EC137093ED13A8E8B4E19C
:1099D000EEEEF3E190E030E020E08217930739F0FB
:1099E0004D9150E0419351932F5F3F4FF6CFE2E806
:1099F000F4E18AE1DF011D928A95E9F71092900562
:109A000010928F050F943801B7CE3F924F925F921C
:109A10006F927F928F929F92AF92BF92CF92DF927E
:109A2000EF92FF920F931F93CF93DF93809149059D
:109A300087FD38C080914A058370A1F5C091EB1273
:109A4000D091EC12488159816A817B8183E297E150
:109A50000E9454414C815D816E817F8184E99FE247
:109A60000E9454414091E7125091E8126091E9122E
:109A70007091EA1281E99FE20E9454418AE0DF91ED
:109A8000CF911F910F91FF90EF90DF90CF90BF90FB
:109A9000AF909F908F907F906F905F904F903F908E
:109AA0000C943E386090DF127090E0128090E112CA
:109AB0009090E212A090E312B090E4120091E512AF
:109AC0001091E612C090E712D090E812E090E912EF
:109AD000F090EA1288E50E94AF1EC82F882309F48F
:109AE0009AC00E94B524362E472E582ED92F20E03A
:109AF00030E040EB53EC0F94DE3387FD0DC020E0E7
:109B000030E040EB53E4632D742D852D9D2F0F9491
:109B1000AE2A18160CF081C060E671E080E197E192
:109B20000E94764160E671E08BE097E10E94764109
:109B300088E097E10E947738C0E089E50E94AF1E77
:109B4000882361F10E94B524362E472E582ED92F36
:109B500020E030E044EB53EC0F94DE3387FD0DC082
:109B600020E030E044EB53E4632D742D852D9D2FD0
:109B70000F94AE2A18160CF055C068E671E085EF18
:109B800096E10E94764168E671E080EF96E10E94DE
:109B900076418DEE96E10E947738C0E08AE50E941A
:109BA000AF1E882309F443C00E94B5246B017C01D9
:109BB00020E030E040E151EC0F94DE3387FD0AC035
:109BC00020E030E040E151E4C701B6010F94AE2A35
:109BD00018166CF567EF7FEF8BED96E10E947641EA
:109BE00069E070E086ED96E10E94764183ED96E1B2
:109BF000DF91CF911F910F91FF90EF90DF90CF9069
:109C0000BF90AF909F908F907F906F905F904F909C
:109C10003F900C947738C1E090CF632C742C852C46
:109C20009D2E8BCFA32CB42C052D1D2FB7CFCC236D
:109C3000E1F0C301D4018093DF129093E012A0936E
:109C4000E112B093E212C501D8018093E312909320
:109C5000E412A093E512B093E612C092E712D092FC
:109C6000E812E092E912F092EA12DF91CF911F918F
:109C70000F91FF90EF90DF90CF90BF90AF909F90AB
:109C80008F907F906F905F904F903F9008958FEDF1
:109C900097E00C94773889ED97E00C94773884E658
:109CA00090E09093D7058093D6051092F705109217
:109CB000F6050C9444E4EF92FF920F931F93CF9319
:109CC000DF93CDB7DEB762970FB6F894DEBF0FBE55
:109CD000CDBF0E94302A882309F43FC04AEF53E0E9
:109CE00082FF02C04EED53E02AEF33E081FF02C055
:109CF00020EE33E080FD2EC08AEF93E05F934F9318
:109D00003F932F939F938F938DE699E19F938F932A
:109D10008E010F5F1F4F1F930F930F94452A0E94D0
:109D20004B4EC8010E944538C8010E946BED0FB62A
:109D3000F894DEBF0FBECDBF81E062960FB6F894F7
:109D4000DEBF0FBECDBFDF91CF911F910F91FF906E
:109D5000EF90089582EE93E0D1CF80E0EECFCF92E6
:109D6000DF92EF92FF928AE50E94AF1E882309F4EA
:109D70005AC00E94B52420E030E040E050EC0F943F
:109D8000AE2AC12CD12CE12C90ECF92E87FD0FC00E
:109D90000E94B52420E030E040E050E40F94DE3330
:109DA00018160CF462C00E94B5246B017C0120914E
:109DB000C10C3091C20C4091C30C5091C40CC7012E
:109DC000B6010F94142B0F94EA32CB010E94F4ECED
:109DD00080E50E94611E81114EC0A701960160912D
:109DE000E7127091E8128091E9129091EA120F94B3
:109DF0007E316093E7127093E8128093E91290939A
:109E0000EA120E944B4E4091E7125091E812609185
:109E1000E9127091EA1284EC96E10E9454418AE0C2
:109E20000E943E3805C083E50E94AF1E8111A1CF7C
:109E30008091490587FD24C080914A05837001F512
:109E40000E944B4E4091E7125091E8126091E91246
:109E50007091EA1285EB96E10E9454418AE0FF90EE
:109E6000EF90DF90CF900C943E38C12CD12CE12C98
:109E700080E4F82E9CCF0E947D248111AECFD8CFF4
:109E800082E50E94611E8111DBCFFF90EF90DF9091
:109E9000CF900895CF9384E50E94AF1EC0E0882341
:109EA000D9F00E945D24C82F1816B4F40E944B4EBE
:109EB0008DE40E943E3880914405909145050E94B2
:109EC000A8EA6C2FCC0F770B88EA9FE00E947641BE
:109ED0008AE00E943E38CFEF8C2FCF9108954F92A9
:109EE0005F926F927F928F929F92AF92BF92CF922A
:109EF000DF92EF92FF92CF93DF93CDB7DEB72C972F
:109F00000FB6F894DEBF0FBECDBF4090EB08509067
:109F1000EC086090ED087090EE0820914F023091AF
:109F200050024091510250915202C301B2010F946C
:109F30007E3169837A838B839C838090EF08909035
:109F4000F008A090F108B090F208209153023091EF
:109F500054024091550250915602C501B4010F942C
:109F60007E316D837E838F839887C090F308D09075
:109F7000F408E090F508F090F6082091570230912F
:109F800058024091590250915A02C701B6010F94EC
:109F90007E3169877A878B879C8720915B0230911D
:109FA0005C0240915D0250915E02C301B2010F94C8
:109FB0007E312B013C0120915F0230916002409183
:109FC000610250916202C501B4010F947E314B01D0
:109FD0005C012091630230916402409165025091CE
:109FE0006602C701B6010F947E316B017C010E94AD
:109FF0004B4E83EE9EE00E94773883E50E94611EFF
:10A00000882321F00E947D2480934D0280914D028F
:10A01000811151C08AEC9EE00E9477388BED9EE062
:10A020000E94773849815A816B817C8184E59EE169
:10A030000E9454414D815E816F81788584E99FE261
:10A040000E94544149855A856B857C8581E99FE250
:10A050000E94544189ED9EE00E94773881ED9EE098
:10A060000E947738B301A20184E59EE10E94544129
:10A07000B501A40184E99FE20E945441B701A60101
:10A0800081E99FE20E9454418AE02C960FB6F89431
:10A09000DEBF0FBECDBFDF91CF91FF90EF90DF907D
:10A0A000CF90BF90AF909F908F907F906F905F9078
:10A0B0004F900C943E388EEC9EE0AECF5F926F9244
:10A0C0007F928F929F92AF92BF92CF92DF92EF9248
:10A0D000FF920F931F93CF93DF931F92CDB7DEB7FD
:10A0E0007C0139018B015B01A40EB51ED12CC12C62
:10A0F000A016B10609F450C0F70180809180F801E4
:10A1000051908F015982C4010F94CC305816B9F187
:10A11000652DC4010F94D430FFEFCF1ADF0AC601BA
:10A120008F779927892B21F162E070E080E090E041
:10A130000E949FA9C4010F94CC3099818917F9F02E
:10A140000E944B4E8FE694E00E94773881E00F909A
:10A15000DF91CF911F910F91FF90EF90DF90CF9003
:10A16000BF90AF909F908F907F906F905F90089579
:10A1700062E070E080E090E00E942326DBCFBE0129
:10A180006F5F7F4FC3010E944FE9F701808191818A
:10A19000019691838083ACCF80E0D9CFDF92EF929C
:10A1A000FF920F931F93CF93DF93CDB7DEB7CA5AB9
:10A1B000D1090FB6F894DEBF0FBECDBFCF55DF4F2C
:10A1C000188219821A821B82C15AD0408091E403FE
:10A1D0009091E503A091E603B091E703CB55DF4FE3
:10A1E00088839983AA83BB83C55AD04084E690E0D4
:10A1F0009093D7058093D6051092F7051092F60537
:10A200001092F80526EF35E044E050E0BE016B55B2
:10A210007F4F86ED95E00E945E508091D60590912B
:10A22000D70502969093D7058093D6051092F7052F
:10A230001092F60581E0C655DF4F8883CA5AD04098
:10A24000CE0186559F4F0E946BDA26EF35E048E439
:10A2500050E065EA7CE086ED95E00E945E5026EFD6
:10A2600035E040E150E06CE079E086ED95E00E9459
:10A270005E508AE097EDA3EABCE3CF55DF4F8883B9
:10A280009983AA83BB83C15AD040CE018F559F4F7B
:10A290000E9462DA81E298E00E947DDA86E292E032
:10A2A0000E9474DA82E292E00E9462DA8091E7080A
:10A2B0009091E808A091E908B091EA0889839A830F
:10A2C000AB83BC838E010F5F1F4FC8010E9462DA0F
:10A2D000CF55DF4F188219821A821B82C15AD04093
:10A2E0007E018DE6E80EF11C83E0D7018C93898313
:10A2F000CE018F559F4F0E9462DAC7010E946BDA30
:10A30000C8010E946BDA4AE0D42EDA94DD2031F0E5
:10A31000CE018F559F4F0E9462DAF7CF8FED92E109
:10A320000E947DDACF55DF4F188219821A821B8274
:10A33000C15AD0403AE0D32EDA94DD2031F0CE017C
:10A340008F559F4F0E9462DAF7CF85E0D82ED982D1
:10A35000F701D082C8010E946BDAC7010E946BDA54
:10A3600026EF35E048E050E069EE75E086ED95E0D7
:10A370000E945E5026EF35E048E050E061EE75E067
:10A3800086ED95E00E945E5026EF35E044E650E011
:10A390006BEA77E086ED95E00E945E5019828FEFC0
:10A3A000D7018C93C8010E9474DAC7010E946BDA4E
:10A3B00026EF35E044E050E06EEF72E086ED95E088
:10A3C0000E945E508091BA068983C8010E9474DAA7
:10A3D000198A1A8A1B8A1C8A80E090E0A0E8BFE3F1
:10A3E0008D879E87AF87B88B8091571290915812B6
:10A3F000A0915912B0915A1289839A83AB83BC837E
:10A400002CEA35EC47E25EE360915B1270915C12DE
:10A4100080915D1290915E120F9478326D837E83ED
:10A420008F8398872CEA35EC47E25EE360915F12F8
:10A430007091601280916112909162120F94142BAE
:10A4400069877A878B879C8726EF35E044E150E067
:10A45000B80186ED95E00E945E5084E190E09A8319
:10A460008983C8010E9450DA8091EC119091ED111E
:10A47000A091EE11B091EF1189839A83AB83BC83D5
:10A480002CEA35EC47E25EE36091F0117091F11136
:10A490008091F2119091F3110F9478326D837E8345
:10A4A0008F8398872CEA35EC47E25EE36091F411E4
:10A4B0007091F5118091F6119091F7110F94142B72
:10A4C00069877A878B879C87C8010E9459DA8CE05C
:10A4D000E5E9F2E0D80101900D928A95E1F7C80113
:10A4E0000E9459DA1982C8010E946BDA8FE790E066
:10A4F0009A838983C8010E9450DAE1EAF2E0D80128
:10A5000001900D92DA94E1F726EF35E045E050E056
:10A51000B80186ED95E00E945E508091E005898348
:10A52000C8010E9474DA80E2E6EAF2E0D801019004
:10A530000D928A95E1F726EF35E040E250E0B80150
:10A5400086ED95E00E945E50F7011082C7010E94DF
:10A5500074DA84E198E00E9474DA80E198E00E9465
:10A5600062DACF55DF4F188219821A821B82C15AD4
:10A57000D040CE018F559F4F0E9462DA80E2D80111
:10A580001D928A95E9F726EF35E040E250E0B801E8
:10A5900086ED95E00E945E50FE01F99688E0DF01AD
:10A5A0001D928A95E9F744E650E060E070E0498347
:10A5B0005A836B837C834D835E836F83788783E0CC
:10A5C00090E0A0E0B0E089879A87AB87BC874D8791
:10A5D0005E876F87788B498B5A8B6B8B7C8B8D8BCF
:10A5E0009E8BAF8BB88F898F9A8FAB8FBC8F8D8FDF
:10A5F0009E8FAF8FB8A38EE190E0A0E0B0E089A37A
:10A600009AA3ABA3BCA38DA39EA3AFA3B8A789A70E
:10A610009AA7ABA7BCA78DA79EA7AFA7B8AB89ABDE
:10A620009AABABABBCAB8DAB9EABAFABB8AF26EFD1
:10A6300035E040E450E0B80186ED95E00E945E50C0
:10A6400090E1D92EF8018D2D11928A95E9F726EF28
:10A6500035E040E150E0B80186ED95E00E945E50A3
:10A66000D8011D92DA94E9F726EF35E040E150E099
:10A67000B80186ED95E00E945E508CE199E00E9461
:10A6800062DA2CE0D22EF8018D2D11928A95E9F72D
:10A6900026EF35E04CE050E0B80186ED95E00E94F1
:10A6A0005E508CE6D8011D928A95E9F726EF35E0D9
:10A6B0004CE650E0B80186ED95E00E945E508AECD1
:10A6C00095E00E9459DA26EF35E048E050E068ED69
:10A6D00075E086ED95E00E945E50F7011192DA94E4
:10A6E000E9F7C755DF4F1882C95AD04080E090E0A3
:10A6F000A0E4B0E4C356DF4F88839983AA83BB8369
:10A70000CD59D040C7010E947DDACE0187559F4FB9
:10A710000E946BDACE0183569F4F0E9462DA80E37B
:10A72000D7011D928A95E9F787EB9CE10E94773863
:10A730008AE00E943E3826EF35E040E350E0B70162
:10A7400086ED95E00E945E508091F805811128C049
:10A750000091D6051091D7058091F6059091F705E7
:10A76000F7019183808384E690E09093D7058093EE
:10A77000D60526EF35E044E050E062E073E086ED78
:10A7800095E00E945E50C7010E9450DA91E00536C4
:10A79000134009F490E08091F805892B8093F80527
:10A7A0008091F805811105C060E08BEE9CE10E946C
:10A7B000E63F8BEC9CE10E9477388AE00E943E38AD
:10A7C0009091F80581E08927C655DF4F0FB6F894C0
:10A7D000DEBF0FBECDBFDF91CF911F910F91FF90D4
:10A7E000EF90DF900895CF93DF9300D01F92CDB705
:10A7F000DEB78091A6068823C1F083E390E09C83B6
:10A800008B831A8219829E012F5F3F4F40E150E0F7
:10A8100067EA76E0CE0103960E945E508BEC9CE1E5
:10A820000E9477388AE00E943E380F900F900F9078
:10A830000F90DF91CF910895CF92DF92EF92FF9228
:10A84000CF93C82F80918B118150823008F069C05E
:10A850000E94DA3A10928B110E94D2A96093C2052D
:10A860007093C3058093C4059093C505C090C60539
:10A87000D090C705E090C805F090C9050E94B02BA4
:10A88000AB01BC014093C6055093C7056093C80552
:10A890007093C9058091AB069091AC06A091AD066E
:10A8A000B091AE068C199D09AE09BF09840F951FA2
:10A8B000A61FB71F8093AB069093AC06A093AD067E
:10A8C000B093AE06C1110AC0C1E00E94F3538C2FB1
:10A8D000CF91FF90EF90DF90CF9008958091A906DF
:10A8E0009091AA0601969093AA068093A9060E94C9
:10A8F000B02BC090AF06D090B006E090B106F090BB
:10A90000B206C616D706E806F906F0F60E94B02B86
:10A910006093AF067093B0068093B1069093B20631
:10A92000D3CFC0E0D2CF81E00C941C540E9493C1DD
:10A930000E94935480E00F94241B8091FC06813088
:10A94000A1F40E94474E82E697E00E94773860E0CB
:10A9500088E597E00E94E63F6EE571E080E090E0D8
:10A960000E94232688E08093FC060895CF92DF9210
:10A97000EF92FF921F93CF93DF9300D01F92CDB73A
:10A98000DEB78EEEC82E82E0D82EE12CF12CC982E3
:10A99000DA82EB82FC82BE016F5F7F4F8AE50E9404
:10A9A0009C3381110EC010E0812F0F900F900F90FB
:10A9B0000F90DF91CF911F91FF90EF90DF90CF909C
:10A9C00008950E94F233C982DA82EB82FC82BE01D2
:10A9D0006F5F7F4F8AE50E949C33182F882319F3FD
:10A9E0000E94474E8CE398E00E9477380E9496546C
:10A9F000DBCFCF92DF92EF92FF921F93CF93DF9343
:10AA000000D01F92CDB7DEB78EEEC82E82E0D82ED2
:10AA1000E12CF12CC982DA82EB82FC82BE016F5FED
:10AA20007F4F8AE00E949C3381110EC010E0812F7D
:10AA30000F900F900F900F90DF91CF911F91FF908B
:10AA4000EF90DF90CF9008950E94F2330E94BC33C4
:10AA50000E94D7330E94BC33C982DA82EB82FC8227
:10AA6000BE016F5F7F4F8AE00E949C33182F8823BE
:10AA7000E9F20E94474E8FEF97E00E9477380E94DC
:10AA80009654D5CFCF93DF9300D01F921F92CDB7AE
:10AA9000DEB781E08093A60680E1E7EAF6E0DF0119
:10AAA0001D928A95E9F70E94F35386E18D8382E334
:10AAB00090E09C838B831A8219829E012F5F3F4F07
:10AAC00041E050E0BE016B5F7F4FCE0103960E94D4
:10AAD0005E500F900F900F900F900F90DF91CF91DD
:10AAE0000895CF93DF93CDB7DEB7A8970FB6F8944C
:10AAF000DEBF0FBECDBF8C01F42E0E9493C10E9419
:10AB0000474E88E397E00E9477380115110511F44C
:10AB10000FE217E08091990580FD79C081608093F4
:10AB200099058BE197E00E9477388AE00E943E38D1
:10AB3000CC24C3948AE5D82ED0923F14C0923E1400
:10AB40008FE090E0909341148093401497E0792E29
:10AB50007092321422E8E22EE092351434E8832E0B
:10AB6000912CA12CB12C8092361490923714A09283
:10AB70003814B092391482EE93E10E94BA34D09224
:10AB80003F14C0923E1488E590E090934114809366
:10AB9000401470923214E0923514809236149092E0
:10ABA0003714A0923814B092391482EE93E10E94C7
:10ABB000BA348AE289838A838B838C83F801DE012D
:10ABC0001596BE016F5F7F4FCD01861B970B2491B9
:10ABD000319621110CC0FB01E80FF91F8AE29F0199
:10ABE000261B370B2832310524F48193F8CF2D939F
:10ABF000EBCF20E630E140E050E082EE93E10E94AE
:10AC000097E96AE070E080E090E00E94C32C61E088
:10AC100086E297E00E94B33F89EE93E030E6019729
:10AC200029F0232F2A950000E9F7F9CFF89489EE4F
:10AC300093E038EE019729F0232F2A950000E9F7D9
:10AC4000F9CF0E9493C1FF2031F00E941B1F0E9488
:10AC5000341FA895FECF0E94191FF9CF8091FB06E3
:10AC6000882319F01092FB06089540E070E060E040
:10AC70008EED98E10E94715580910B0D90910C0D15
:10AC80002FEF3FEF981751F0E92FF0E0E55FF24F1B
:10AC9000228130E09F5F9F7790930C0DC90108954A
:10ACA0001F920F920FB60F9211240F900FBE0F90AC
:10ACB0001F9018951F920F920FB60F9211240BB68A
:10ACC0000F920F931F932F933F934F935F936F9325
:10ACD0007F938F939F93AF93BF93CF93DF93EF9324
:10ACE000FF93C091C60000910C0DD0910B0D11E0A7
:10ACF0001D0F1F7790912704913108F09FC0E92F15
:10AD0000F0E08827E957F94A8F4F0D94753198562E
:10AD1000C756D656E556EC561E57F0561E57F456F3
:10AD2000F8561E57FC56005704570B571E57165718
:10AD3000C03229F028F5CA3011F0CD3031F50117B5
:10AD400031F0ED2FF0E0E55FF24FC283D12FD093C9
:10AD50000B0DFF91EF91DF91CF91BF91AF919F913B
:10AD60008F917F916F915F914F913F912F911F91A3
:10AD70000F910F900BBE0F900FBE0F901F90189564
:10AD8000CD3481F081E0CE3471F080E10CC0CA3363
:10AD900038F4C033A0F6C03291F2CD32B1F7CFCF44
:10ADA000CD3499F782E080932704C9CFC13359F09D
:10ADB00018F4C03221F2E9CF88E0C433A1F38BE06C
:10ADC000C83389F3E2CF83E0EECF84E0C03359F398
:10ADD00086E0C13341F3D9CF85E0C833B1F6E3CF84
:10ADE00087E0C23391F6DFCF89E0C13371F6DBCF64
:10ADF0008AE0C03351F6D7CF8CE0C73331F6D3CFDA
:10AE00008DE0C63311F6CFCFC03209F498CF8EE073
:10AE1000C33549F2BACF80ED8C0F8A3008F08FCF5E
:10AE20009FE0909327048093280489CFCA3019F0BB
:10AE3000CD3009F084CF1092270481CFCA3019F0A9
:10AE4000CD3009F07CCF80919C148823A1F39730FA
:10AE500089F038F4953079F71092440210929E0CE4
:10AE6000EACF9A3059F09F3031F7809128040E9440
:10AE7000D931E1CF81E080932406DDCF81E080935A
:10AE80002306D9CF8EBD0DB407FEFDCF08958FEFF9
:10AE90008EBD0DB407FEFDCF8EB508959091640070
:10AEA0009B7F90936400982F906A96959CBD80FD3F
:10AEB00003C091E0863009F490E09DBD0895CF93E2
:10AEC000DF93EB010E947738CE01DF91CF910C9494
:10AED000DDB12F923F924F925F926F927F928F924D
:10AEE0009F92AF92BF92CF92DF92EF92FF920F9319
:10AEF0001F93CF93DF93009709F0AAC11092F30C30
:10AF00001092F20C9093980580939705BAE0CB2E9F
:10AF1000B0E2DB2EE12CF12C15E002E846015701EE
:10AF2000C4E1D0E01092851310928413109378132B
:10AF300000937B1380927C1390927D13A0927E13DA
:10AF4000B0927F1388E293E10E94BA3421972FEFE9
:10AF5000821A920AA20AB20A209721F744E1C40E8B
:10AF6000D11CE11CF11C8AE5C81680E2D806E10478
:10AF7000F104A1F6C12CA0E2DA2EE12CF12CD5E0EF
:10AF8000C2E81092851310928413D0937813C09363
:10AF90007B13C0927C13D0927D13E0927E13F092CB
:10AFA0007F1388E293E10E94BA34109285131092C5
:10AFB0008413D0937813C0937B13D701C6018C52AE
:10AFC0009F4FAF4FBF4F80937C1390937D13A093FF
:10AFD0007E13B0937F1388E293E10E94BA34EFEFBF
:10AFE000CE1ADE0AEE0AFE0AFAE0CF16F0E2DF061B
:10AFF000E104F10431F6FEEDCF2EF0E2DF2EE12C7C
:10B00000F12CD5E0C2E81092851310928413D093EE
:10B010007813C0937B13C0927C13D0927D13E0927F
:10B020007E13F0927F1388E293E10E94BA342FEFEF
:10B03000C21AD20AE20AF20A46EEC41640E2D40666
:10B04000E104F10401F7CC24C394E2E1DE2EE12C0B
:10B05000F12C0AE010E0D5E0C2E8109385130093CC
:10B060008413D0937813C0937B13C0927C13D09237
:10B070007D13E0927E13F0927F1388E293E10E94A9
:10B08000BA341093851300938413D0937813C0932C
:10B090007B13D701C6018096A11DB11D80937C133F
:10B0A00090937D13A0937E13B0937F1388E293E176
:10B0B0000E94BA348FEFC81AD80AE80AF80AE5E005
:10B0C000CE16E2E1DE06E104F10439F60091F20C5D
:10B0D0001091F30C0115110509F0D6C08091F10C07
:10B0E000882309F4E1C02AE030E240E050E068EE55
:10B0F00073E088E293E10E9497E9C1E0D0E003E0C9
:10B1000010E0E090F20CF090F30C35E0332E42E8C2
:10B11000242E44244A94542C64E0662E712C7FE142
:10B12000C72E74E0D72E8091F20C9091F30C800F13
:10B13000911FE816F90608F0D5C0C7010E94AEEAD3
:10B14000882309F481C08091061269EF71E1882398
:10B1500011F066E072E1FB0101900020E9F7CF01F8
:10B160000197861B970BF4E1FC9F9001FD9F300D2A
:10B170001124265F3F4D50E040E0459710F0FB0161
:10B18000128A88E293E10E9497E9CE018F5F9D4E7B
:10B19000B0E0A0E021964E0124E0880C991C2A958D
:10B1A000E1F7FDEF8F1AFFE99F0AB12CA12C209146
:10B1B000A81424FF7EC0709285136092841330928D
:10B1C000781320927B1380937C1390937D13A0932C
:10B1D0007E13B0937F1388E293E10E94BA34D09239
:10B1E0008513C09284133092781320927B1380923F
:10B1F0007C1390927D13A0927E13B0927F1388E20D
:10B2000093E10E94BA34B70183E798E10E9442417A
:10B210008091061266E072E1811102C069EF71E16E
:10B2200080E798E10E945F576EE57CE08CE698E14C
:10B230000E945F5769EF71E18BE698E10E945F57CA
:10B2400087E698E10E9477382FEFE21AF20A6BCF77
:10B250002091F20C3091F30CA901415051096091F9
:10B260009705709198056817790738F42C5F3F4F60
:10B270003093F30C2093F20C45CE4430510508F482
:10B280003DCE24503109F4CF0430110569F480918A
:10B29000F10C882331F083E090E09093F30C8093DD
:10B2A000F20CD0E0C0E02DCFD0E0C0E004E010E030
:10B2B00028CF109285131092841330927813209225
:10B2C0007B1380937C1390937D13A0937E13B09394
:10B2D0007F1388E293E10E94BA3450928513409222
:10B2E000841381CFDF91CF911F910F91FF90EF9049
:10B2F000DF90CF90BF90AF909F908F907F906F9096
:10B300005F904F903F902F900895AF92BF92CF9251
:10B31000DF92EF92FF920F931F93CF93DF93CDB7FE
:10B32000DEB7E6970FB6F894DEBF0FBECDBF009133
:10B330004B0510914C05F80101900020E9F7319779
:10B340006F01C01AD10AF801CF01801B910B8C1537
:10B350009D053CF481918F32B9F7DF0111971C9262
:10B36000F3CF8BE1E8ECF4E1DE015C9601900D9205
:10B370008A95E1F7F12CE12CEC14FD040CF05DC092
:10B38000F801EE0DFF1D8081811103C08FEFE81AD7
:10B39000F80A5801AE0CBF1CF5018081882309F41E
:10B3A0004CC0FFEFEF1AFF0AF801EE0DFF1D7F0101
:10B3B000E01AF10A81918111FACFCE014C960E94D8
:10B3C00070B68BE1FE017C96DE01119601900D9224
:10B3D0008A95E1F7B501CE0101960E947EAECE01BD
:10B3E00001960E94C62F8FE20E943E38809106127D
:10B3F00081113BC085EF93E00E94DDB18091A814DC
:10B4000084FF1BC019821C8221E0A501BE01645E7D
:10B410007F4FCE0101960E94B2B8811129C08AE007
:10B420000E943E380E944B4EB50182E597E10E9492
:10B430005F57CE0101960E94C62F8AE00E943E38D7
:10B44000CE014C960E94C62FE6960FB6F894DEBF4A
:10B450000FBECDBFDF91CF911F910F91FF90EF9065
:10B46000DF90CF90BF90AF90089586E092E1C4CF77
:10B47000CE014C960E94DFB58BE1FE013196DE01D4
:10B480005C9601900D928A95E1F7CE0101960E949B
:10B49000C62F72CF2F923F924F925F926F927F9200
:10B4A0008F929F92AF92BF92CF92DF92EF92FF92D4
:10B4B0000F931F93CF93DF9300D000D000D01F9243
:10B4C0001F92CDB7DEB7B82E8091F80D843008F00A
:10B4D000D1C10E94D2A96B017C018091F80D81112C
:10B4E00008C080910B0D90910C0D891B8F7709F48A
:10B4F000A4C681E6A82E13C08A3019F08D3009F059
:10B50000F6C01092F30D8091910D9091920DFC0177
:10B51000E357F24F1682892BF1F40E94E0C4809128
:10B52000F80D843008F0ECC080910B0D90910C0D5B
:10B53000891B8F7709F4E4C00E943C5697FFDCCF4B
:10B540000E94474E85EB95E00E94773880910B0D65
:10B5500080930C0DE4CF1092920D1092910D03E99F
:10B560001DE0F8018191803209F446C08E3409F063
:10B57000A9C060EB75E0C8010F942B2A4C01892B00
:10B5800041F06EE470E0C80104960F94CC3400974B
:10B5900009F4C8014AE050E070E060E001960F94C1
:10B5A0009B272B013C0180918D0D90918E0DA091D8
:10B5B0008F0DB091900D0196A11DB11D4816590631
:10B5C0006A067B0629F060E08DE795E0892851F155
:10B5D0006AE270E0C8010F94FB349C01009729F1E6
:10B5E000982F901B912C992349F09150F801E90F65
:10B5F000F11D80819826F7CF8F01B3CF4AE050E04C
:10B6000070E060E0C90101960F949B27292D30E07E
:10B6100050E040E0621773078407950751F060E03F
:10B620008EE595E00E94A0F07ACF60E084E395E09B
:10B63000F9CF40928D0D50928E0D60928F0D7092C9
:10B64000900D8091FC068130E1F067E470E0C80164
:10B650000F94CC340097A9F04AE050E070E060E02D
:10B6600001960F949B27643071058105910548F47C
:10B6700083E994E00E94773860E089E894E00E94D2
:10B68000E63FC092A307D092A407E092A507F092EC
:10B69000A6078091930D8B3309F441CF8091F80D6B
:10B6A000843008F03CCF8091FA0D8A9DC0011124AE
:10B6B00063E97DE08550924F0F94D73480E00E947B
:10B6C0005AF02DCF8091A81480FFBBCF67EB7DE2AD
:10B6D000C8010F942B2A009731F0FC01838180531D
:10B6E0008A3008F0AECF60E08AE095E09BCF21E998
:10B6F0003DE043E95DE063EF7DE00E942F1D0FCF49
:10B700008091A81482FFB6C01A82198271E6F72EC2
:10B71000E0E1EE2EF9E6DF2E8091F80D843008F09E
:10B72000A9C00E94671D8111A5C041E050E0BE0183
:10B730006B5F7F4F8CE096E10E9432B40D8110E088
:10B74000019711F00FEF1FEF8091141690911516CD
:10B75000A0911616B09117168093A4149093A51477
:10B76000A093A614B093A7140E94671D0F3F100763
:10B7700049F4811107C00E94474E83ED95E00E9475
:10B780007738CACF4091FA0D242F30E00A3061F0AB
:10B790000D3051F0882309F45FC089819A810097A8
:10B7A00019F001969A8389831092AE0489819A8157
:10B7B000F29EF001F39EF00D1124E850F24FE80FD5
:10B7C000F91F1382892B69F50E94E0C40E94671D4E
:10B7D000882309F4A1CF0E94AE618CE096E10E941B
:10B7E000DFB580919F14882391F1815080939F143D
:10B7F0008D9DC001112462E08C5C994F0E9434BB86
:10B80000E0919F1424E0E29FF0011124E05DF94FE4
:10B8100060817181828193810E9480220E94E7ADC4
:10B820007BCF1A82198281E00E945AF08091A41481
:10B830009091A514A091A614B091A7148093F40D33
:10B840009093F50DA093F60DB093F70DBFCF0E9426
:10B85000E8B5E092FC0660CF4F9DA0011124455051
:10B86000524F9E012F5F3F4F6EEA74E0802F0E947F
:10B870002F1D52CF0E94D2A96B017C01B11004C0D0
:10B8800080918A11882351F0C092DD11D092DE118F
:10B89000E092DF11F092E011BB24B3948091230574
:10B8A00090912405A0912505B09126050097A1054A
:10B8B000B105B1F04091DD115091DE116091DF11C1
:10B8C0007091E011840F951FA61FB71FA701960165
:10B8D000281B390B4A0B5B0BDA01C901B7FF92C178
:10B8E0008091130290911402A0911502B09116025A
:10B8F000892B8A2B8B2B09F099C10E94D2A94B016D
:10B900005C0180919E0C811108C02091F0129091F1
:10B91000F11281E0291301C080E020915212309190
:10B92000531291E089272A3A31050CF480E091E026
:10B930004091B3045091B4046091B5047091B60481
:10B94000452B462B472B09F490E0981789F0882364
:10B9500009F4BDC1D501C40180569444A24FBF4F24
:10B960008093B3049093B404A093B504B093B60449
:10B970004090750250907602609077027090780245
:10B980002091AF043091B0044091B1045091B204C1
:10B99000C301B2010F94AE2A882319F18091B30438
:10B9A0009091B404A091B504B091B6044092AF0454
:10B9B0005092B0046092B1047092B204892B8A2B29
:10B9C0008B2B09F449C0D501C40180569444A24F81
:10B9D000BF4F8093B3049093B404A093B504B09385
:10B9E000B6048091B3049091B404A091B504B091D1
:10B9F000B6040097A105B10579F1881A990AAA0A37
:10BA0000BB0AB7FC29C01092B3041092B404109280
:10BA1000B5041092B60483E396E00E94773860E0A4
:10BA20008FE196E00E94E63F80915412909155126A
:10BA30001816190624F490E080E00E94371F8091C8
:10BA4000E9119091EA111816190634F41092EA11CE
:10BA50001092E9110E9466C18091BB049091BC04D0
:10BA6000A091BD04B091BE0446015701881A990AFD
:10BA7000AA0ABB0AD501C401B7FDB9C12091F012D1
:10BA80009091F1124091350280913402291323C123
:10BA900090912009899FC0011124880F892F881F48
:10BAA000990B91958D8380912109489FC0011124A4
:10BAB000880F892F881F990B91958E830E94D2A998
:10BAC00069837A838B839C8340E0BE016F5F7F4FE5
:10BAD000CE0105960E94811C6D8170E089E00E9474
:10BAE000C9A841E0BE016F5F7F4FCE0105960E945D
:10BAF000811C6E8170E087E00E94C9A880912F06AA
:10BB0000882309F467C10091200210912102C80125
:10BB100002972091541230915512281739070CF4CE
:10BB200059C18090F1128F82188619861A861B8659
:10BB30008091F0129F80891509F4E7C0892D90E06B
:10BB400037E6A32EA89EF001A99EF00D1124EB5D0F
:10BB5000F64F458956896789708D452B462B472BB3
:10BB600081F4418D528D638D748D452B462B472B6F
:10BB700041F4458D568D678D70A1452B462B472B83
:10BB8000E1F127E6B22EB89E9001B99E300D112446
:10BB9000A9014B5D564F1A01FA01618172818381BF
:10BBA00094810F942C344B015C01F10161A172A1CD
:10BBB00083A194A10F94B32A2B013C01F10165A14B
:10BBC00076A187A190A50F94B32A9B01AC01C30174
:10BBD000B2010F947832A50194010F94142B4B01FC
:10BBE0005C01288539854A855B850F94DE331816FC
:10BBF00024F488869986AA86BB868F818F5F87709A
:10BC00008F8396CF0E94474E6091A1077091A20743
:10BC100082EE95E00E945F578AE00E943E3840E045
:10BC200070E060E090E080E00E9471559091F01229
:10BC30008091F112981749F0C092DD11D092DE1177
:10BC4000E092DF11F092E01158CEBB2019F0109273
:10BC5000BF0453CE0E94D2A90091DD111091DE11D4
:10BC60002091DF113091E011809013029090140226
:10BC7000A0901502B0901602080D191D2A1D3B1D3B
:10BC8000601B710B820B930B97FDE1CF8091BF047A
:10BC9000811133CE81E08093BF045F9A80919F0C25
:10BCA0008E7F80939F0C8A9A80919F0C8D7F8093CA
:10BCB0009F0C80910801809581708093060180918E
:10BCC0009F0C8B7F80939F0C0E94191F16CE80E0E3
:10BCD00090E0DC0145CE2091F11257E6259F9001BE
:10BCE00011242B5D364FF901EF59FF4F9081899F49
:10BCF000C0011124880F892F881F990B91958D837E
:10BD00002E593F4FF9018081D0CE20911A023091F7
:10BD10001B0240911C0250911D02688579858A851D
:10BD20009B850F94142B4B015C01B801012E000C74
:10BD3000880B990B0F94B52A9B01AC01C501B40186
:10BD40000F947E3169837A838B839C8340911E029A
:10BD500050911F02B801CE0101960E949EC48980B5
:10BD60009A80AB80BC804090B7045090B80460903B
:10BD7000B9047090BA04A3019201C501B4010F94F3
:10BD8000AE2A87FF16C028E431EE4AE75FE3C3011D
:10BD9000B2010F94142B20E037ED43EA5CE30F94DB
:10BDA0007E31A50194010F94142B69837A838B83D0
:10BDB0009C8369817A818B819C816093B7047093A5
:10BDC000B8048093B9049093BA040F94EA32CB017B
:10BDD0000E94371FF4E6CF0ED11CE11CF11CC0926B
:10BDE000BB04D092BC04E092BD04F092BE040E9459
:10BDF000E0C48091FC06882309F4E0C1809126020A
:10BE0000882309F4A3C08091FD0481119FC0809113
:10BE10008A11811108C080918B11813021F08091AD
:10BE2000A81482FF93C0F894649B10C080912202F2
:10BE300090912302A0912402B09125028093FD05E8
:10BE40009093FE05A093FF05B09300066091FD0559
:10BE50007091FE058091FF0590910006789420E096
:10BE600030E0A9010F94AE2A87FF70C001E0009373
:10BE7000FD0480918A11811167C088E496E00E94D8
:10BE800077388AE00E943E3884E08093080D82E093
:10BE90008093F40C81E09AE590933F1480933E14D4
:10BEA0008EE490E0909341148093401487E0809357
:10BEB000321482E88093351484E890E0A0E0B0E08A
:10BEC0008093361490933714A0933814B093391498
:10BED00082EE93E10E94BA340E9463400093F8110D
:10BEE00040E36CE876E084E799E00E94684061E016
:10BEF00088E699E00E944A401091270560E01027EB
:10BF00008CE399E069F48AE796E00E94B33F80E30E
:10BF10000E943E388AE00E943E3860E08DE596E05F
:10BF20000E94B33F88E696E00E94773880E30E9443
:10BF30003E388AE00E943E38112331F083E696E0D5
:10BF40009093EE0C8093ED0C0E94AE6190910901EC
:10BF5000892F80958170109100021817C9F02091E7
:10BF6000A81420622093A8148093000290FD3FC182
:10BF700064EF71E080E090E00E9423260E940AB600
:10BF80008091A81483FD7CC1111133C10E940C362D
:10BF90000E94D2A96B017C01109117021123F1F0CC
:10BFA000809128058823D1F04091C0045091C104AC
:10BFB0006091C2047091C30446015701841A950A26
:10BFC000A60AB70AB501A40177FD1AC0833009F4A7
:10BFD0002FC10CF01EC181300CF023C1212F30E0A5
:10BFE000A8EEB3E00F944631C60ED71EE81EF91E28
:10BFF000C092C004D092C104E092C204F092C30483
:10C0000080918B11813009F073C00E94D2A96B011D
:10C010007C018091C8049091C904A091CA04B09198
:10C02000CB04A7019601281B390B4A0B5B0BDA01E5
:10C03000C901B7FD3AC0D701C601805F984DAF4F27
:10C04000BF4F8093C8049093C904A093CA04B093CF
:10C05000CB048090C6059090C705A090C805B0900D
:10C06000C9050E94B02BAB01BC014093C60550939B
:10C07000C7056093C8057093C9058091AB06909180
:10C08000AC06A091AD06B091AE0688199909AA092F
:10C09000BB09840F951FA61FB71F8093AB06909313
:10C0A000AC06A093AD06B093AE068091C404909107
:10C0B000C504A091C604B091C70446015701881A6F
:10C0C000990AAA0ABB0AD501C401B7FD11C020E82C
:10C0D000C20E2EEED21E26E3E21EF11CC092C40454
:10C0E000D092C504E092C604F092C7040E94F353B4
:10C0F0000E94B5390E94804180912205882379F100
:10C100000E94D2A96B017C0180911E0590911F05B0
:10C11000A0912005B091210546015701881A990A7E
:10C12000AA0ABB0AD501C401B7FD19C02091220596
:10C1300030E0A8EEB3E00F944631C60ED71EE81EDD
:10C14000F91EC0921E05D0921F05E0922005F092C4
:10C15000210580E00E94C4BD8AE00E943E388091A3
:10C160001D05882359F10E94D2A96B017C018091A1
:10C17000190590911A05A0911B05B0911C05A70106
:10C180009601281B390B4A0B5B0BDA01C901B7FD7D
:10C1900015C020911D0530E0A8EEB3E00F944631A4
:10C1A000C60ED71EE81EF91EC0921905D0921A05B8
:10C1B000E0921B05F0921C050E94A5AD2B960FB6D0
:10C1C000F894DEBF0FBECDBFDF91CF911F910F91CD
:10C1D000FF90EF90DF90CF90BF90AF909F908F90A7
:10C1E0007F906F905F904F903F902F9008950E94A6
:10C1F000F9B5123008F0CCCE0E940C3660E085EC28
:10C2000096E050C083ED96E09093EE0C8093ED0C99
:10C21000BFCE843009F0E2CE0E944B4E8AED96E00C
:10C2200004C00E944B4E89E097E00E947738D6CE3A
:10C230000E944B4E82EF96E0F8CF8091A307909139
:10C24000A407A091A507B091A607A7019601281BF6
:10C25000390B4A0B5B0BDA01C901885E9340A109D7
:10C26000B109B7FD46C98DEC95E00E947738C092C0
:10C27000A307D092A407E092A507F092A60739C9B8
:10C28000123098F48DE996E00E9477388AE00E9497
:10C290003E380E94DE2C90E080E00E94695760E00A
:10C2A00086EB96E00E94E63F73CE123009F070CE26
:10C2B0000E9464BA882379F081E00E943ABA42EB86
:10C2C00050E06DE278E08DEA94E10E9432B48DEAAC
:10C2D00094E10E94DFB50E94B42F811193CF0E9498
:10C2E0009E2F0E94E0BA0E9435BA52CECF93DF93C0
:10C2F0008091F0129091F112891B8095877019F44A
:10C300000E944A5AF5CF8091F0128F5F8770A091FA
:10C31000F01297E6A99FD0011124FD01EB5DF64FC5
:10C32000EF0119929A95E9F798E09083A65CB64FD1
:10C3300090E1E2E0F3E101900D929A95E1F720910E
:10C34000F0129091F112291303C094E69093ED122C
:10C350008093F012DF91CF910C94CC2F9091F0123A
:10C360008091F112981306C08091230990912409BD
:10C37000892B21F080E00E944A5AF0CF0895CF9295
:10C38000DF92EF92FF92FC01C080D180E280F380C7
:10C390002091C50C3091C60C4091C70C5091C80C2F
:10C3A000C701B6010F94142B0F94EB3360930E1357
:10C3B00070930F138093101390931113C092FE1279
:10C3C000D092FF12E0920013F09201139091F012BC
:10C3D0008091F112981731F0FF90EF90DF90CF909D
:10C3E0000C9476610E94AE610E94232A40910E1344
:10C3F00050910F13609110137091111340931F0609
:10C40000509320066093210670932206882331F012
:10C41000FF90EF90DF90CF900C94CC2FFF90EF9097
:10C42000DF90CF9008954F925F926F927F928F929C
:10C430009F92AF92BF92CF92DF92EF92FF920F93B3
:10C440001F93CF93DF93EC018B017A016901F9010E
:10C4500080819181A281B381FA0140815181628101
:10C460007381F80180809180A280B38048805980D8
:10C470006A807B804092F2125092F3126092F41222
:10C480007092F5128092F6129092F712A092F81222
:10C49000B092F9124093FA125093FB126093FC127F
:10C4A0007093FD128093FE129093FF12A0930013DD
:10C4B000B09301132091C50C3091C60C4091C70C6C
:10C4C0005091C80CF60160817181828193810F9433
:10C4D000142B0F94EB334B015C012091C10C309174
:10C4E000C20C4091C30C5091C40CF7016081718162
:10C4F000828193810F94142B0F94EB336B017C0199
:10C500002091BD0C3091BE0C4091BF0C5091C00CDD
:10C51000F80160817181828193810F94142B0F94B3
:10C52000EB332B013C012091B90C3091BA0C4091B6
:10C53000BB0C5091BC0C688179818A819B810F94DE
:10C54000142B0F94EB3360930213709303138093B7
:10C5500004139093051340920613509207136092B0
:10C56000081370920913C0920A13D0920B13E09231
:10C570000C13F0920D1380920E1390920F13A09251
:10C580001013B09211139091F0128091F11298173C
:10C5900091F0DF91CF911F910F91FF90EF90DF907D
:10C5A000CF90BF90AF909F908F907F906F905F9053
:10C5B0004F900C9476610E94AE610E94232A4091B4
:10C5C0000A1350910B1360910C1370910D1300918D
:10C5D0000613109107132091081330910913C0908E
:10C5E0000213D0900313E0900413F0900513C0924F
:10C5F0001306D0921406E0921506F09216060093E8
:10C600001706109318062093190630931A064093C4
:10C610001B0650931C0660931D0670931E064091E6
:10C620000E1350910F1360911013709111134093DA
:10C630001F065093200660932106709322068823DC
:10C6400091F0DF91CF911F910F91FF90EF90DF90CC
:10C65000CF90BF90AF909F908F907F906F905F90A2
:10C660004F900C94CC2FDF91CF911F910F91FF90A1
:10C67000EF90DF90CF90BF90AF909F908F907F9082
:10C680006F905F904F9008953F924F925F926F929C
:10C690007F928F929F92AF92BF92CF92DF92EF9252
:10C6A000FF920F931F93CF93DF93CDB7DEB76897B9
:10C6B0000FB6F894DEBF0FBECDBFD82E2A013B01C6
:10C6C000480159013E2C20E030E0A901C501B80124
:10C6D0000F94AE2A811110C081E08D1508F0B6C00C
:10C6E00060E070E080E793E420E030E040E752E46F
:10C6F0000F9478324B015C018D8A9E8AAF8AB88E86
:10C700000D2D10E0F801E853F64EE491BB24B394EC
:10C710001E160CF4B12CCC24C39420E030E0A90107
:10C72000C301B2010F94DE3318160CF0C12CBC14F7
:10C7300071F092E0D9120BC0332049F081E00F94E0
:10C74000241B69E170E080E090E00E94232680E0F5
:10C750000E94D22F69837A838B839C8381E00E941D
:10C76000D22F6D837E838F83988782E00E94D22FA1
:10C7700069877A878B879C8783E00E94D22F6D8799
:10C780007E878F87988B000F111F000F111FE1E02C
:10C79000F0E0EC0FFD1F0E0F1F1FF8011082118239
:10C7A000128213829E01235F3F4FAE01475F5F4FAE
:10C7B000BE016B5F7F4FCE0101960E941362F801AC
:10C7C0004082518262827382198A1A8A1B8A1C8A69
:10C7D0008091230990912409892B91F4CE014196EF
:10C7E0007C018E010B5E1F4F9E01235F3F4FAE0108
:10C7F000475F5F4FBE016B5F7F4F40970E94C4F061
:10C800000E94AE61BC1451F092E0D91205C03320F1
:10C8100019F080E00F94241B0E942E5668960FB6E4
:10C82000F894DEBF0FBECDBFDF91CF911F910F9166
:10C83000FF90EF90DF90CF90BF90AF909F908F9040
:10C840007F906F905F904F903F90089560E070E808
:10C850008BE395E449CF4F925F926F927F928F92D4
:10C860009F92AF92BF92CF92DF92EF92FF920F937F
:10C870001F93CF93DF93CDB7DEB72C970FB6F89405
:10C88000DEBF0FBECDBF2B013C0129873A874B8706
:10C890005C8747015801F601E080F1800281138135
:10C8A00020E030E0A901B701C8010F94AE2A882327
:10C8B00009F488C05E2D4F2D302F212F852F942F06
:10C8C000A32FB22F89839A83AB83BC8320E030E00F
:10C8D000A901B701C8010F94AE2A811108C0E090E8
:10C8E0004502F09046020091470210914802C701AC
:10C8F000D8018D839E83AF83B887A5019401609191
:10C9000071027091720280917302909174020F947F
:10C91000AE2A87FF0CC08092710290927202A092A0
:10C920007302B0927402CE0101960E94FE2A4092D8
:10C93000690250926A0260926B0270926C02898561
:10C940009A85AB85BC8580936D0290936E02A0930F
:10C950006F02B0937002CE0105960E94FE2AA501D7
:10C9600094016091710270917202809173029091B2
:10C9700074020F94DE33181664F480927102909260
:10C980007202A0927302B0927402CE0101960E94CC
:10C99000FE2A0E94AE612C960FB6F894DEBF0FBE41
:10C9A000CDBFDF91CF911F910F91FF90EF90DF905E
:10C9B000CF90BF90AF909F908F907F906F905F903F
:10C9C0004F90089550E040E030E820E477CFCF92D8
:10C9D000DF92EF92FF920F931F936A01E090710232
:10C9E000F09072020091730210917402FB01208199
:10C9F000318142815381FC01608171818281938107
:10CA00000E942B641F910F91FF90EF90DF90CF90C9
:10CA10000895CF92DF92EF92FF920F931F936B01D5
:10CA2000FC01E080F18002811381E9E6F2E02481DB
:10CA300035814681578160817181828193810E9415
:10CA40002B641F910F91FF90EF90DF90CF9008958E
:10CA50000F931F93CF93DF93EC018B0181E00F9431
:10CA6000241B69E170E080E090E00E942326B80179
:10CA7000CE010E940965C091FB0680E00F94241B43
:10CA80001092FB0682E00E94FC2F0E94192BC2FB31
:10CA9000CC27C0F981E08C27DF91CF911F910F91B6
:10CAA0000895AF92BF92CF92DF92EF92FF920F93D1
:10CAB0001F93CF93DF9300D01F92CDB7DEB7FC0159
:10CAC000E080F18002811381611112C0A090710297
:10CAD000B0907202C0907302D09074029501A601CA
:10CAE000B701C8010F94AE2A87FF02C07501860105
:10CAF00020E030E048EC53E4B701C8010F94AE2ABF
:10CB000087FD04C0E12CF12C08EC13E4C701D80127
:10CB100089839A83AB83BC836AEF72E0CE0101966E
:10CB20000E9409650F900F900F900F90DF91CF91A9
:10CB30001F910F91FF90EF90DF90CF90BF90AF903B
:10CB400008953F924F925F926F927F928F929F9241
:10CB5000AF92BF92CF92DF92EF92FF920F931F930B
:10CB6000CF93DF9300D01F92CDB7DEB7382E80E091
:10CB700090E0A0E2B1E489839A83AB83BC83C09048
:10CB8000E712D090E812E090E912F090EA1220E06B
:10CB900030E0A901C701B6010F94AE2A87FF0CC08F
:10CBA000A701960160E070E080E291E40F947D318E
:10CBB00069837A838B839C8360E0CE0101960E9417
:10CBC00051654090690250906A0260906B027090CB
:10CBD0006C0280906D0290906E02A0906F02B090F7
:10CBE0007002332089F10E94F95419821A821B8243
:10CBF0001C82E0907102F090720200917302109119
:10CC00007402CE0101966C01A5019401C301B20129
:10CC10000E942B6430929F070E94A12B0F900F90CF
:10CC20000F900F90DF91CF911F910F91FF90EF9098
:10CC3000DF90CF90BF90AF909F908F907F906F903C
:10CC40005F904F903F9008950E94B654CECF809150
:10CC50009F07882319F080E00E94A16580E0089575
:10CC60002F923F924F925F926F927F928F929F92FC
:10CC7000AF92BF92CF92DF92EF92FF920F931F93EA
:10CC8000CF93DF93CDB7DEB766970FB6F894DEBFCC
:10CC90000FBECDBFF82E282E312CF101E853F64EF1
:10CCA000D49022E0821335C080919F07811103C088
:10CCB00081E00E94A1650E94F954811139C184EC80
:10CCC00099E10E94A01D20E030E0A9010F94AE2A56
:10CCD0008823F9F06D2DDD0C770B880B990B0F94E1
:10CCE000B52A2B013C0184EC99E10E94A01D4B0167
:10CCF0005C0120E030E040EA50E40F94AE2A11E0FD
:10CD000087FF1CC0812C912C90EAA92E90E4B92EAB
:10CD100015C06D2DDD0C770B880B990B0F94B52A80
:10CD20002B013C01C101880F991F880F991F845462
:10CD3000964E0E94A01D4B015C0110E0A3019201E0
:10CD4000C501B4010F94142B4B015C016101CC0CA3
:10CD5000DD1CCC0CDD1CC6018055964E0E94A01D2A
:10CD6000EE24E394E12620E030E040EC5FE30F9412
:10CD7000142BA30192010F94142BAB01BC0100E012
:10CD800010E098018F2D0E94446320E030E0A9015B
:10CD9000C501B4010F94AE2AF601EC55F64EFA8B9C
:10CDA000E98B882309F44DC0F2E000E010E020E4B4
:10CDB00031E4FF1619F000E010E09801B501A4017C
:10CDC0007058E12C8F2D0E944463A5019401C50188
:10CDD000B4010F947E316B8B7C8B8D8B9E8B22E00C
:10CDE000F216E9F0F101EF55F64E6491611107C0BA
:10CDF0000E944B4E8FE799E10E9477386AE070E01D
:10CE000090E080E00F94B32A9B01AC0160E070E0F9
:10CE100088E492E40F9478328B019C0104C000E016
:10CE200010E020EC30E4EE24E3944B895C896D89BA
:10CE30007E898F2D0E94446332E0F312D0C00E949D
:10CE4000B65481E090E0A0E0B0E00F2C04C0880F61
:10CE5000991FAA1FBB1F0A94D2F720919F0C282B61
:10CE600020939F0C2091B105822B8093B105898975
:10CE70009A890E94A01DF601E759FD4F60837183D6
:10CE80008283938382E0F8121AC02091E7123091D6
:10CE9000E8124091E9125091EA126091710270918A
:10CEA000720280917302909174020F947D316093AD
:10CEB0007102709372028093730290937402F60170
:10CEC000EB5EF74F10821182128213828F2D0E9427
:10CED000BD1C0E94192BF601E759FD4F80819181FD
:10CEE000A281B381F601E157F84F80839183A28339
:10CEF000B38392E0F916A9F18CE0E6ECF2E0DE01F2
:10CF0000119601900D928A95E1F7E1E0F0E0EC0FC7
:10CF1000FD1FEC0DFD1D80809180A280B38020E07C
:10CF200030E0A901C501B4010F94AE2A81111EC0E1
:10CF300066960FB6F894DEBF0FBECDBFDF91CF91DE
:10CF40001F910F91FF90EF90DF90CF90BF90AF9027
:10CF50009F908F907F906F905F904F903F902F9019
:10CF600008950E9427668111E3CFC6CF20E030E00C
:10CF7000A901C501B4010F94DE3387FF04C0B7FADD
:10CF8000B094B7F8B094F601E759FD4F6F01A301D3
:10CF90009201C501B4010F94142B9B01AC01F60161
:10CFA00060817181828193810F947D31F60160836C
:10CFB000718382839383F2E080E090E0A0E4B1E4A7
:10CFC000FF1621F080E090E0A8E4B2E48D879E8710
:10CFD000AF87B88BCE010D960E94FE2AA9CF81E0C3
:10CFE00090E0A0E0B0E00F2C04C0880F991FAA1FAA
:10CFF000BB1F0A94D2F720919F0C282B20939F0CE3
:10D000002091B105822B8093B10589899A890E946C
:10D01000A01DF601E759FD4F6083718382839383DE
:10D020004ECFCF93DF9300D01F92CDB7DEB780E015
:10D0300090E0A0EAB0E489839A83AB83BC8361E08B
:10D04000CE0101960E9451650F900F900F900F90A6
:10D05000DF91CF9108958F929F92AF92BF92CF921E
:10D06000DF92EF92FF920F931F93CF93DF93CDB791
:10D07000DEB72C970FB6F894DEBF0FBECDBF8B0185
:10D0800040E050E068E472E44D835E836F8378870C
:10D0900040E050E060EA70E449875A876B877C87FC
:10D0A0008130B9F1823009F459C020E030E040E02D
:10D0B00050E46091710270917202809173029091BC
:10D0C00074020F947E314B017C0120E030E048EC8B
:10D0D00053E40F94DE33181634F4812C912C88EC31
:10D0E000E82E93E4F92EF801A084B184C284D3849D
:10D0F0009401A701B501C6010F94DE33181614F090
:10D1000054016701C501D60189839A83AB83BC832F
:10D1100048C0BE01675F7F4FC80108960E9409653D
:10D12000B8016C5F7F4FAE014B5F5F4FC8010E943B
:10D13000E7640E94CC302C960FB6F894DEBF0FBE89
:10D14000CDBFDF91CF911F910F91FF90EF90DF90B6
:10D15000CF90BF90AF909F908F900895F801208559
:10D160003185428553856091710270917202809180
:10D170007302909174020F947E316B017C0120E068
:10D1800030E048EC53E40F94AE2A87FD06C0C12C72
:10D19000D12C28ECE22E23E4F22EC982DA82EB8233
:10D1A000FC82BE01675F7F4FCE010196B7CFEF9241
:10D1B000FF920F931F93CF93DF937C018B010E940B
:10D1C000C631C9E6D2E02091790230917A024091CD
:10D1D0007B0250917C02F701608171818281938191
:10D1E0000F9478322C853D854E855F850F947E3176
:10D1F0006C877D878E879F87C8010E94FE2ADF91FA
:10D20000CF911F910F91FF90EF900C94AE614F92D0
:10D210005F926F927F92AF92BF92CF92DF92EF9226
:10D22000FF920F931F93CF93DF9300D000D01F92F4
:10D230001F92CDB7DEB75C0180E090E0A0E7B2E4DA
:10D2400089839A83AB83BC8380E090E0A0E8B0EC54
:10D250008D839E83AF83B887BE016F5F7F4FCE0102
:10D2600005960E94D76868E873E180E090E00E942C
:10D270002326C12CD12C88ECE82E81E4F82EC9821B
:10D28000DA82EB82FC8280E090E0A0E8B0E48D835B
:10D290009E83AF83B887BE016F5F7F4FCE01059637
:10D2A0000E94D76805EA1CE0F80140AC51AC62ACC2
:10D2B00073ACC0AED1AEE2AEF3AE80E090E0A0E2DF
:10D2C000B2E489839A83AB83BC83F5018081918129
:10D2D000A281B3818D839E83AF83B887BE016F5FC8
:10D2E0007F4FCE0105960E94D768F80140AE51AE3F
:10D2F00062AE73AE129A64E670E080E090E00E9445
:10D30000232681E028960FB6F894DEBF0FBECDBF6E
:10D31000DF91CF911F910F91FF90EF90DF90CF9011
:10D32000BF90AF907F906F905F904F9008951F9344
:10D33000CF93DF93CDB7DEB72C970FB6F894DEBF4F
:10D340000FBECDBF182F882379F020E030E0A9016F
:10D350006091E9057091EA058091EB059091EC05EB
:10D360000F94AE2A8823F9F08091A00C8117D9F090
:10D370000E94AE618CE0E2EDF2E0DE0111960190D8
:10D380000D928A95E1F7CE0101960E944C1F809183
:10D39000A00C882391F089E692E00E942527109244
:10D3A000A00C0E94192B2C960FB6F894DEBF0FBE6E
:10D3B000CDBFDF91CF911F91089581E08093A00CA4
:10D3C00089E692E00E943921ECCF2F923F924F9252
:10D3D0005F926F927F928F929F92AF92BF92CF9205
:10D3E000DF92EF92FF920F931F93CF93DF93CDB70E
:10D3F000DEB7CB54D1090FB6F894DEBF0FBECDBF58
:10D400002DB73EB739AF28AF87E00E945B4E811140
:10D410000BC061E086E50E9471248DA3853060F029
:10D4200087E39EE00E947738A8ADB9AD0FB6F894B7
:10D43000BEBF0FBEADBF40C33DA1332321F087E186
:10D440009EE00E9477386AE080E50E947124182FE0
:10D450008CEF810F8F3218F083EF9DE0E3CF60E017
:10D4600085E40E948D24882309F448C081E08FABB5
:10D47000E090EB12F090EC12D7012D913D914D917F
:10D480005C916091690270916A0280916B02909147
:10D490006C020F947E31AB01BC0188E50E94DF2451
:10D4A00069877A878B879C87F7012481358146813C
:10D4B000578160916D0270916E0280916F02909120
:10D4C00070020F947E31AB01BC0189E50E94DF241C
:10D4D0006D877E878F87988BBE01635F7F4FCE01FC
:10D4E00009960E946C2E382E81110BC063E68FEDD9
:10D4F0009DE00E94E63F87EC9DE094CF92E09FABD9
:10D50000B7CF8CE40E94611E082F882309F431C133
:10D510000E945D248EA3803118F080EA9DE082CFC6
:10D52000FEA1F13009F427C160E083E50E948D245B
:10D530008AAF882321F0011102C037E03EA38DA1FC
:10D54000833020F086E89DE00E9477389091A00C0F
:10D550009DAF80E00E9497690E94F61C1D8A1E8A7A
:10D560001F8A188E198E1A8E1B8E1C8E83EF9FE4D5
:10D57000A3ECB7E48D8F9E8FAF8FB8A383EF9FE4AA
:10D58000A3ECB7EC89A39AA3ABA3BCA3A12FB0E0F3
:10D59000BCA7ABA7EDB7FEB724E0129FE019F109D5
:10D5A00011240FB6F894FEBF0FBEEDBF8DB79EB726
:10D5B00001969CAF8BAF2DA14FA9BE01635F7F4F3A
:10D5C000CE0109960F94061C9B01AC010F94703498
:10D5D000811162C20E94D2A9611571058105910570
:10D5E00011F00F943426212C1BAA1CAA1DAA1EAAD6
:10D5F000AEA1A150BB0B2C96BFAFAEAF2C97E22DC6
:10D60000F0E0F8A7EFA32BA53CA5E217F3070CF079
:10D6100074C23196FEA7EDA73F932F93FF93EF932C
:10D6200082E79DE09F938F938CE79DE09F938F937C
:10D630001F920F94421B8DB79EB709960FB6F894B0
:10D640009EBF0FBE8DBF9EA1992309F458C10F94B0
:10D65000E5252AE030E040E050E00F9414310F94CB
:10D66000B52A20E030E040EA50E40F94DE330FEFBB
:10D670001FEF181614F001E010E00F94E52528E6DE
:10D6800031E040E050E00F9414310F94B52A2B01A3
:10D690003C010F94E52527E230E040E050E00F9494
:10D6A00014316B5F7F4F8F4F9F4F0F94B52A4B0103
:10D6B0005C01ADA1A430D1F4BC01A40184E69DE0DD
:10D6C0000E945441B301A2018CE59DE00E945441A7
:10D6D00086E59DE00E9477380130110519F483E456
:10D6E0000E943E3882E59DE00E947738312CC801C7
:10D6F000110FAA0BBB0B2A968CAF9DAFAEAFBFAF7D
:10D700002A972C96AEADBFAD2C973A161B060CF09F
:10D71000F6C02A966CAD7DAD8EAD9FAD2A970F9465
:10D72000B52A6B017C01BAADBB2341F1AC019B0171
:10D730000F947E3120E030E040E952E40F94142B46
:10D740009B01AC01C301B2010F947E312B013C015E
:10D7500020E030E044EB53E40F94DE331816FCF481
:10D7600020E030E044EB53E4C301B2010F947D317B
:10D77000EDCF1EA2D9CE22E02EA3D6CE0F94E52562
:10D7800024E130E040E050E00F941431675E7F4FB9
:10D790008F4F9F4F0F94B52AA7019601CFCF20E05E
:10D7A00030E0A901C301B2010F94AE2A87FF0BC07C
:10D7B00020E030E044EB53E4C301B2010F947E312A
:10D7C0002B013C01ECCF0091EB121091EC12F8010F
:10D7D00024813581468157816D857E858F85988925
:10D7E0000F947D3122966CAF7DAF8EAF9FAF2297A5
:10D7F0002BED3FE049E450E4C301B2010F94142B38
:10D8000020E030E044E353E40F9478326B017C0174
:10D810000F9473326FA778AB89AB9AABD8012D9177
:10D820003D914D915C9169857A858B859C850F949E
:10D830007D3126966CAF7DAF8EAF9FAF2697A50149
:10D8400094016FA578A989A99AA90F94142B9B011B
:10D85000AC0126966CAD7DAD8EAD9FAD26970F9435
:10D860007E3169837A838B839C83C701B6010F94D1
:10D870001E34A50194010F94142B22962CAD3DADBE
:10D880004EAD5FAD22970F947E316D837E838F8383
:10D89000988740E651E070E060E0CE0101960E947A
:10D8A0009EC448E651E070E060E0CE0105960E941B
:10D8B0009EC4BDA1B43099F449815A816B817C81A9
:10D8C00086E49DE00E9454414D815E816F817885A0
:10D8D00084E99FE20E9454418AE00E943E38198AFE
:10D8E0001A8A1B8A1C8AAE014F5E5F4FBE016B5FB6
:10D8F0007F4FCE0101960E94E764339402CF20E06F
:10D900004FA9BE01635F7F4FCE0109960F94061C9D
:10D910004B015C01312CAC019B010F9470348111DF
:10D9200002C033243394A5019401C501B4010F94BE
:10D9300070348111E2C0EFA1F8A5EE0FFF1FEE0FCA
:10D94000FF1F2BAD3CADE20FF31F80829182A282BC
:10D95000B382A50194016D8D7E8D8F8D98A10F945A
:10D96000DE33181624F48D8E9E8EAF8EB8A2A501DC
:10D97000940169A17AA18BA19CA10F94AE2A87FF83
:10D9800004C089A29AA2ABA2BCA2A50194016BA972
:10D990007CA98DA99EA90F947E316BAB7CAB8DAB1E
:10D9A0009EABADA5BEA5BD01BB0F880B990B0F9417
:10D9B000B52A6FA378A789A79AA79B01AC016BA989
:10D9C0007CA98DA99EA90F9478322B013C014D8A28
:10D9D0005E8A6F8A788EEBADFCADF8ABEFA710E0F6
:10D9E000C12CD12C7601AFA5B8A96D917D918D91F7
:10D9F0009D91B8ABAFA7A30192010F947D319B011C
:10DA0000AC010F94142B9B01AC01C701B6010F941C
:10DA10007E316B017C011F5F211628F72FA138A5ED
:10DA200049A55AA50F9478320F942C34698F7A8FB8
:10DA30008B8F9C8FBDA1B23068F18DA59EA50E94F1
:10DA4000F1E96BA57CA581E49DE00E9476418BE322
:10DA50009DE00E94773843E0C501B4010E9420BDDB
:10DA600080E20E943E3881E0EDA1E3300CF480E0DA
:10DA7000E12C8E010F5D1F4F9E01235E3F4FAE01D3
:10DA8000475E5F4FBE016B5E7F4F0E94353F8AE06D
:10DA90000E943E382394B3CD0E9427660E94DD1C6D
:10DAA0008DAD0E9497690E94CC3088AD99AD0FB6BC
:10DAB000F8949EBF0FBE8DBFE8ADF9AD0FB6F894D8
:10DAC000FEBF0FBEEDBFC55BDF4F0FB6F894DEBFE4
:10DAD0000FBECDBFDF91CF911F910F91FF90EF90BF
:10DAE000DF90CF90BF90AF909F908F907F906F907E
:10DAF0005F904F903F902F9008950E9427663320AB
:10DB000069F280E39DE00E94773881E0FDA11F1655
:10DB10000CF080E0EE24E3948E010F5D1F4F9E0118
:10DB2000235E3F4FAE01475E5F4FBE016B5E7F4F8E
:10DB30000E94353F698D7A8D8B8D9C8D0052110925
:10DB400026E042E00F947B259F938F938FE19DE029
:10DB50009F938F9389E29DE09F938F931F920F94E1
:10DB6000421B2DB73EB7295F3F4F0FB6F8943EBF1B
:10DB70000FBE2DBF93CF2F923F924F925F926F9225
:10DB80007F928F929F92AF92BF92CF92DF92EF924D
:10DB9000FF920F931F93CF93DF93CDB7DEB76A97B2
:10DBA0000FB6F894DEBF0FBECDBF83E50E94611EA5
:10DBB000182F3090A00C882319F00E947D24382E55
:10DBC0004090690250906A0260906B0270906C0203
:10DBD00080916D0290916E02A0916F02B0917002DF
:10DBE0008B8B9C8BAD8BBE8B80917102909172025E
:10DBF000A0917302B09174028F8B988FA98FBA8F06
:10DC0000112329F0311003C080E00E94976986E556
:10DC10000E94611E8A8B20E030E0A9016091E90535
:10DC20007091EA058091EB059091EC050F94AE2A76
:10DC3000882309F4C9C083E40E94611E882309F483
:10DC40009DC00E94B5246B017C01ABEAB7E0B987A7
:10DC5000A887BF83AE83F5E0FD831D861E8628EC72
:10DC60002F8702EC1A86212C88EC8B8792E49C8704
:10DC7000AE81BF81B98BA88B15E0E889F9898190C5
:10DC80009190A190B190F98BE88B2A85322D4B852C
:10DC90005C85C501B4010F94AE2A87FF04C08A8653
:10DCA000292CAB86BC862D853E854F85502FC5011E
:10DCB000B4010F94DE33181624F48D869E86AF8649
:10DCC0000B2D1150D1F6FD81F150FD838E819F8186
:10DCD00044969F838E83F111CBCF2D853E854F8552
:10DCE000502F6A85722D8B859C850F947E3120E0A4
:10DCF00030E040E05FE30F94142BA70196010F94EE
:10DD00007E314B015C012DEB37E346E855EB0F9478
:10DD1000DE3387FD0AC02DEB37E346E855E3C50146
:10DD2000B4010F94AE2A18164CF580E00E94976952
:10DD300010E0E884F98400E0D7016D917D918D9128
:10DD40009D917D016D01B4E0CB1AD108A50194012C
:10DD50000F947D31F6016083718382839383602FFA
:10DD6000812F0F94171A0F5F053031F71F5F8885D9
:10DD700099854496998788871530D9F6AA89AA2368
:10DD800081F020E030E0A9016091E9057091EA0599
:10DD90008091EB059091EC050F94AE2A81110E94C1
:10DDA000BD408AE50E94611E882351F00E94B5247F
:10DDB00069837A838B839C83CE0101960F94DF184D
:10DDC000832D0E9497690BC0311003C09A89992353
:10DDD00041F30E944B4E80E69CE00E94773833204E
:10DDE00051F08091A00C811106C00E94474E81E441
:10DDF0009CE00E9477380E944B4E83E39CE00E9497
:10DE000077388091A00C0E9436410E944B4E86E2EA
:10DE10009CE00E947738C090E708D090E808E09036
:10DE2000E908F090EA0820E030E0A901C701B60156
:10DE30000F94DE3318160CF053C042E0C701B60150
:10DE40000E9420BD8DE00E943E388AE00E943E384C
:10DE5000A30192016091690270916A0280916B0244
:10DE600090916C020F94AE2A81111FC02B893C89BE
:10DE70004D895E8960916D0270916E0280916F0292
:10DE8000909170020F94AE2A81110FC02F89388DA6
:10DE9000498D5A8D60917102709172028091730266
:10DEA000909174020F94AE2A81110E94CC306A9630
:10DEB0000FB6F894DEBF0FBECDBFDF91CF911F919B
:10DEC0000F91FF90EF90DF90CF90BF90AF909F9019
:10DED0008F907F906F905F904F903F902F9008951C
:10DEE00081E29CE00E947738B3CF8F929F92AF92ED
:10DEF000BF92EF92FF920F931F93CF93DF9380E037
:10DF00000E9497691092E5051092E6051092E705C8
:10DF10001092E8051092E1051092E2051092E305D7
:10DF20001092E4051092ED051092EE051092EF05A7
:10DF30001092F0051092E9051092EA051092EB0597
:10DF40001092EC050BEA17E0C0E0812C912C80ECDC
:10DF5000A82E8FE7B82E7801D0E0F7018192919238
:10DF6000A192B1927F016D2F8C2F0F94171ADF5F52
:10DF7000D53099F7CF5F0C5E1F4FC53061F7DF9149
:10DF8000CF911F910F91FF90EF90BF90AF909F9016
:10DF90008F9008959091F0128091F112981308C01B
:10DFA0008091230990912409892B11F40C941B1F53
:10DFB00080E00E944A5AEECF83E50E94AF1E88237C
:10DFC000E9F00E94D2A96093DD117093DE11809375
:10DFD000DF119093E0110E94B52420E030E04AE781
:10DFE00054E40F94142B0F94F13260931302709346
:10DFF00014028093150290931602089580914705AC
:10E0000084FD0AC08091490587FD06C080914A05BC
:10E01000837011F40C94CA6F0E94AE6188E50E946F
:10E02000611E882331F05F9A80919F0C8E7F8093D0
:10E030009F0C89E50E94611E882331F08A9A8091A5
:10E040009F0C8D7F80939F0C8AE50E94611E882320
:10E0500059F080910801809581708093060180912C
:10E060009F0C8B7F80939F0C85E40E94611E811121
:10E070000C94191F08952F923F924F925F926F92C6
:10E080007F928F929F92AF92BF92CF92DF92EF9248
:10E09000FF920F931F93CF93DF93CDB7DEB7A69771
:10E0A0000FB6F894DEBF0FBECDBF8FE897E00E9499
:10E0B000462A80915D0C83FD7EC0209175023091CF
:10E0C0007602409177025091780260919B0770919F
:10E0D0009C0780919D0790919E070F94AE2A8823FC
:10E0E00009F469C010912209111161C08091670281
:10E0F0009091680201972091521230915312281783
:10E1000039073CF40E944B4E82E599E10E94773832
:10E1100011E0209175023091760240917702509182
:10E12000780260919B0770919C0780919D07909168
:10E130009E070F947D316B017C0120E030E0A90146
:10E140000F94DE3387FF04C0F7FAF094F7F8F094E9
:10E150002091790230917A0240917B0250917C02A9
:10E16000C701B6010F94142B20E030E84BE354E4D0
:10E170000F94DE331816ECF40E944B4E83E399E1C2
:10E180000E94773880919B0790919C07A0919D07F2
:10E19000B0919E078093750290937602A0937702C8
:10E1A000B09378028BE997E00E94BF6104C010E051
:10E1B000B0CF1111E7CF2AE037ED43E25CE3609185
:10E1C000490270914A0280914B0290914C020F9447
:10E1D000142B6B017C0160917F0270918002072EED
:10E1E000000C880B990B0F94B52A9B01AC01C70159
:10E1F000B6010F94142B698B7A8B8B8B9C8B80913F
:10E20000A00C882309F18090E7089090E808A0907E
:10E21000E908B090EA08C0909707D0909807E0907E
:10E220009907F0909A0720E030E0A901C501B401F8
:10E230000F94AE2A8823D1F1A7019601C501B4013C
:10E240000F94DE33181694F1C12CD12C76018E0177
:10E250000F5E1F4F2BE937E047E957E063E977E0AE
:10E260008FE897E00F94340080E1EFE8F7E0A9E64B
:10E27000B2E001900D928A95E1F7A6960FB6F89458
:10E28000DEBF0FBECDBFDF91CF911F910F91FF90E9
:10E29000EF90DF90CF90BF90AF909F908F907F9046
:10E2A0006F905F904F903F902F900895209169025A
:10E2B00030916A0240916B0250916C0260918F071D
:10E2C0007091900780919107909192070F947D3102
:10E2D0006D8B7E8B8F8B988F20916D0230916E02AB
:10E2E00040916F0250917002609193077091940772
:10E2F00080919507909196070F947D31698F7A8F61
:10E300008B8F9C8F20917102309172024091730229
:10E3100050917402C701B6010F947D316D8F7E8FCD
:10E320008F8F98A3209175023091760240917702E9
:10E330005091780260919B0770919C0780919D0796
:10E3400090919E070F947D316B017C0120E030E0BD
:10E35000A9016D897E898F89988D0F94AE2A8111CC
:10E360000CC020E030E0A901698D7A8D8B8D9C8DE9
:10E370000F94AE2A882309F467CF2D893E894F89EF
:10E38000588DCA01B9010F94142B4B015C01298DE2
:10E390003A8D4B8D5C8DCA01B9010F94142B9B01F2
:10E3A000AC01C501B4010F947E314B015C012D8D90
:10E3B0003E8D4F8D58A1CA01B9010F94142B9B01BA
:10E3C000AC01C501B4010F947E314B015C01A70182
:10E3D0009601C701B6010F94142B9B01AC01C50136
:10E3E000B4010F947E310F942C344B015C012DEB62
:10E3F00037E346E855E30F94AE2A87FF0FC020E0CD
:10E4000030E0A901C701B6010F94DE334601570180
:10E4100087FF04C0B7FAB094B7F8B0942DEB37E398
:10E4200046E855E3C501B4010F94AE2A87FD1CCF21
:10E4300020E030E040EA51E4C501B4010F947832A5
:10E440000F94F1321B01672B19F422242394312CF1
:10E45000B10190E080E00F94B32A9B01AC0160E031
:10E4600070E080E89FE30F9478322B013C01AC010F
:10E470009B01C501B4010F94142B4B015C01A30156
:10E4800092016D897E898F89988D0F94142B6D8BE5
:10E490007E8B8F8B988FA3019201698D7A8D8B8DE6
:10E4A0009C8D0F94142B698F7A8F8B8F9C8FA30177
:10E4B00092016D8D7E8D8F8D98A10F94142B6D8F91
:10E4C0007E8F8F8F98A3A3019201C701B6010F948D
:10E4D000142B69A37AA38BA39CA380E1E9E6F2E065
:10E4E0008E010F5F1F4FD80101900D928A95E1F7C1
:10E4F0000E94D2A92B013C0128EC420E511C611C48
:10E50000711C0DA31EA381E0281A310809F460C014
:10E510000E94D2A98B019C0104191509260937090B
:10E5200037FD59C02B013C0128EC420E511C611CE7
:10E53000711C80E00E944A5A2D893E894F89588D6E
:10E5400069817A818B819C810F947E3169837A8382
:10E550008B839C83298D3A8D4B8D5C8D6D817E8163
:10E560008F8198850F947E316D837E838F8398870A
:10E570002D8D3E8D4F8D58A169857A858B859C8523
:10E580000F947E3169877A878B879C8729A13AA16E
:10E590004BA15CA16D857E858F8598890F947E3116
:10E5A0006D877E878F87988B750164018E010F5E62
:10E5B0001F4F9E01235F3F4FAE01475F5F4FBE017C
:10E5C0006B5F7F4F8DA19EA10F94340081119BCF73
:10E5D000750164013CCE0E94E0C4AECF8F929F9241
:10E5E000AF92BF92CF92DF92EF92FF92CF93DF93E1
:10E5F0008090490290904A02A0904B02B0904C0249
:10E60000FC01C080D180E280F38020E030E0A901ED
:10E61000C701B6010F94AE2A882341F0C092490287
:10E62000D0924A02E0924B02F0924C02C0917F02DB
:10E63000D091800284E690E09093800280937F02E4
:10E64000C0907902D0907A02E0907B02F0907C0238
:10E6500080E090E0A0E8BFE38093790290937A0293
:10E66000A0937B02B0937C020E943B70809249028F
:10E6700090924A02A0924B02B0924C02D093800238
:10E68000C0937F02C0927902D0927A02E0927B021C
:10E69000F0927C02DF91CF91FF90EF90DF90CF90CE
:10E6A000BF90AF909F908F9008950F931F93CF933B
:10E6B000DF9300D01F92CDB7DEB79C010FE817E0C3
:10E6C00090E1E9E6F2E0D80101900D929A95E1F728
:10E6D000F9012081318142815381F8016085718582
:10E6E000828593850F947E31F801608771878287D8
:10E6F000938780E090E0A0EAB0E489839A83AB83BB
:10E70000BC83CE0101960E94EE720F900F900F9085
:10E710000F90DF91CF911F910F9108952F923F920B
:10E720004F925F926F927F928F929F92AF92BF9221
:10E73000CF92DF92EF92FF921F93CF93DF93CDB7EB
:10E74000DEB72C970FB6F894DEBF0FBECDBF7A01AF
:10E750001901DC012D913D914D915C912D833E83FA
:10E760004F835887FB014080518062807380809086
:10E77000690290906A02A0906B02B0906C02A501B1
:10E7800094016D817E818F8198850F94AE2A8111CD
:10E790000EC011E0A301920160916D0270916E02B2
:10E7A00080916F02909170020F94AE2A811110E057
:10E7B000D1012D913D914D915C9129873A874B87ED
:10E7C0005C87F701C080D180E280F38020910B024A
:10E7D00030910C0240910D0250910E02C701B6011A
:10E7E0000F94AE2A882309F44EC0C0920B02D09237
:10E7F0000C02E0920D02F0920E028091750290914F
:10E800007602A0917702B091780240916D0250910A
:10E810006E0260916F027091700280928F079092E9
:10E820009007A0929107B09292074093930750935C
:10E8300094076093950770939607C0929707D092BC
:10E840009807E0929907F0929A0780939B0790931C
:10E850009C07A0939D07B0939E0720E030E040E026
:10E860005FE36091D10C7091D20C8091D30C9091A8
:10E87000D40C0F94142B69837A838B839C83CE01F1
:10E8800001960E94EE722D813E814F815885209322
:10E890008F073093900740939107509392074092CF
:10E8A0009307509294076092950770929607D10152
:10E8B0002D913D914D915C9160919B0770919C07CA
:10E8C00080919D0790919E070F947E3160939B07E6
:10E8D00070939C0780939D0790939E0711112FC002
:10E8E00020E030E0A90169857A858B859C850F94AD
:10E8F000AE2A811133C060E070E088EC92E4698355
:10E900007A838B839C83CE0101960E94EE722C96B3
:10E910000FB6F894DEBF0FBECDBFDF91CF911F9130
:10E92000FF90EF90DF90CF90BF90AF909F908F902F
:10E930007F906F905F904F903F902F9008952AEFB7
:10E940003EE74AE25FE36091D50C7091D60C80916E
:10E95000D70C9091D80C0F94142BD1CF60E070E0BD
:10E9600080EA91E4CCCF0F931F93CF93DF9300D035
:10E9700000D01F921F92CDB7DEB78B01FC0123A5FB
:10E98000211102C00F94F31D1D821E821F82188662
:10E9900020E030E040E05FE360917102709172022C
:10E9A00080917302909174020F947E3169837A830F
:10E9B0008B839C839E012B5F3F4FAE014F5F5F4F68
:10E9C0006DE672E089E692E00E948E731D821E82DF
:10E9D0001F82188620E030E040E05FE3F8016085A8
:10E9E0007185828593850F947E3169837A838B83C9
:10E9F0009C83B8016C5F7F4F9E012B5F3F4FAE0140
:10EA00004F5F5F4FC8010E948E7328960FB6F8942F
:10EA1000DEBF0FBECDBFDF91CF911F910F91089543
:10EA20009B01AC01485F5F4FBC016C5F7F4F0C9452
:10EA30008E732F923F924F925F926F927F928F923E
:10EA40009F92AF92BF92CF92DF92EF92FF920F937D
:10EA50001F93CF93DF93CDB7DEB7A6970FB6F89489
:10EA6000DEBF0FBECDBF8C011B015A874987409086
:10EA7000690250906A0260906B0270906C02809004
:10EA80006D0290906E02A0906F02B0907002DB0158
:10EA90008D919D910D90BC91A02D8B8B9C8BAD8BFE
:10EAA000BE8B9C01AD01C301B2010F947D316B019E
:10EAB0007C01D10114968D919D910D90BC91A02D5A
:10EAC0008F8B988FA98FBA8F9C01AD01C501B401BE
:10EAD0000F947D316B8F7C8F8D8F9E8FA985BA852A
:10EAE0008D919D910D90BC91A02D8B879C87AD87BA
:10EAF000BE879C01AD01C301B2010F947D316F8FC0
:10EB000078A389A39AA3A985BA8514968D919D911E
:10EB10000D90BC91A02D8F87988BA98BBA8B9C01EF
:10EB2000AD01C501B4010F947D316BA37CA38DA30E
:10EB30009EA3A7019601C701B6010F94142B6B0188
:10EB40007C012B8D3C8D4D8D5E8DCA01B9010F94DA
:10EB5000142B9B01AC01C701B6010F947E314B0110
:10EB60005C012B893C894D895E896B857C858D850F
:10EB70009E850F947D312B013C012F89388D498D65
:10EB80005A8D6F85788989899A890F947D316B01B7
:10EB90007C01A3019201C301B2010F94142B2B013C
:10EBA0003C01A7019601C701B6010F94142B9B01EC
:10EBB000AC01C301B2010F947E310F942C346B0170
:10EBC0007C012F8D38A149A15AA1CA01B9010F9426
:10EBD000142B2B013C012BA13CA14DA15EA1CA012C
:10EBE000B9010F94142B9B01AC01C301B2010F9426
:10EBF0007E319B01AC01C501B4010F94DE331816C0
:10EC0000B4F520E030E0A901C701B6010F94DE336E
:10EC100087FF2AC0C701B601905820E030E040EAE3
:10EC200050E40F94DE33181614F5A10169857A8536
:10EC3000C8010E941975A6960FB6F894DEBF0FBEE4
:10EC4000CDBFDF91CF911F910F91FF90EF90DF909B
:10EC5000CF90BF90AF909F908F907F906F905F907C
:10EC60004F903F902F900895C701B601D6CF20E076
:10EC700030E040E050E4C501B4010F94DE331816D3
:10EC800024F4B101C8010E94B37419821A821B8254
:10EC90001C82BE016F5F7F4FC1010E9410752DEC79
:10ECA0003CEC4CEC5CE3C701B6010F94142B9B01C8
:10ECB000AC01F80160817181828193810F94142BE2
:10ECC0006D837E838F839887D8019B968C919B97C9
:10ECD0008823C9F02AE939E949E95FE314966D917F
:10ECE0007D918D919C9117970F94142B69837A8352
:10ECF0008B839C83BE016F5F7F4F8FE897E00E94FC
:10ED00001075F80113A6BE016B5F7F4F89859A8548
:10ED10000E94107590CF3F924F925F926F927F92B8
:10ED20008F929F92AF92BF92CF92DF92EF92FF921B
:10ED30000F931F93CF93DF93CDB7DEB76C970FB6CA
:10ED4000F894DEBF0FBECDBFDB010C91142F100F66
:10ED5000153008F067C11196DC90C22ECD0CB4E0DE
:10ED6000BC1508F45FC1ED2DF0E0E25FFA4F808042
:10ED7000912CB12CA12C002E04C0B694A79497948A
:10ED800087940A94D2F780FE4DC1EC2DF0E0E25F4B
:10ED9000FA4F8080912CB12CA12C012E04C0B69486
:10EDA000A794979487940A94D2F780FE3BC1322EA1
:10EDB000642F7C014090E1055090E2056090E305EE
:10EDC0007090E4058091E9059091EA05A091EB052A
:10EDD000B091EC05898F9A8FAB8FBC8F660F770B44
:10EDE000072E000C880B990B0F94B52A4B015C0180
:10EDF000602F000F770B880B990B0F94B52A298D84
:10EE00003A8D4B8D5C8D0F94142BA30192010F94BE
:10EE10007E31A50194010F947E316D877E878F87A7
:10EE2000988B612F110F770B880B990B0F94B52AD4
:10EE3000298D3A8D4B8D5C8D0F94142BA30192017B
:10EE40000F947E31A50194010F947D3169837A83FB
:10EE50008B839C834090E5055090E6056090E70524
:10EE60007090E8058091ED059091EE05A091EF0579
:10EE7000B091F005898F9A8FAB8FBC8F632D660F91
:10EE8000770B072E000C880B990B0F94B52A4B01BA
:10EE90005C016D2DDD0C770B880B990B0F94B52A57
:10EEA000298D3A8D4B8D5C8D0F94142BA30192010B
:10EEB0000F947E31A50194010F947E31698B7A8B7A
:10EEC0008B8B9C8B6C2DCC0C770B880B990B0F9438
:10EED000B52A298D3A8D4B8D5C8D0F94142BA3018F
:10EEE00092010F947E31A50194010F947D316D83C1
:10EEF0007E838F839887F70180859185A285B3856E
:10EF000089879A87AB87BC878D8B9E8BAF8BB88F99
:10EF100047E651E061E070E0CE0141960E949EC458
:10EF200047E651E061E070E0CE0105960E949EC484
:10EF30004FE551E061E070E0CE010D960E949EC465
:10EF40004FE551E061E070E0CE0101960E949EC461
:10EF500089889A88AB88BC8827E137EB41ED58EB6C
:10EF6000C501B4010F94DE3387FD5CC023E030E0BF
:10EF700044EB53E4C501B4010F94AE2A18160CF407
:10EF800051C08D849E84AF84B88827E137EB41ED72
:10EF900058EBC501B4010F94DE3387FD43C023E075
:10EFA00030E040EB53E4C501B4010F94AE2A1816CB
:10EFB000CCF18D809E80AF80B88427E137EB41EDA6
:10EFC00058EBC501B4010F94DE3387FD2BC023E05D
:10EFD00030E044EB53E4C501B4010F94AE2A181697
:10EFE0000CF189809A80AB80BC8027E137EB41ED42
:10EFF00058EBC501B4010F94DE3387FD13C023E045
:10F0000030E040EB53E4C501B4010F94AE2A18166A
:10F010004CF0AE014F5F5F4FBE01635F7F4FC70192
:10F020000E9419756C960FB6F894DEBF0FBECDBF67
:10F03000DF91CF911F910F91FF90EF90DF90CF90D4
:10F04000BF90AF909F908F907F906F905F904F9008
:10F050003F9008952F923F924F925F926F927F92CE
:10F060008F929F92AF92BF92CF92DF92EF92FF92D8
:10F070000F931F93CF93DF93CDB7DEB7CC58D10951
:10F080000FB6F894DEBF0FBECDBF80E19CE00E94BA
:10F09000773887E00E945B4E81116EC084E50E9444
:10F0A000AF1E882329F00E94A22481110E940EBD68
:10F0B00080E090E0A0E8BFE389839A83AB83BC83C0
:10F0C0008D839E83AF83B8878DEC9CECACE4BEE36C
:10F0D00089879A87AB87BC8780E090E0A0E2B1E4A3
:10F0E0008D879E87AF87B88B8CE390E09A8B898B56
:10F0F0008DEC90E09C8B8B8B8DEC9CECACECBEE3B0
:10F100008D8B9E8BAF8BB88F80E090E0A0EEBFE33D
:10F11000898F9A8FAB8FBC8F1BA61CA64AE959E931
:10F1200069E97EE38FE40E94DF246D8F7E8F8F8FED
:10F1300098A360E083E40E948D2489A360E08BE4BF
:10F140000E948D248AA382E40E94AF1E882381F14D
:10F150000E94A224009761F19C01285231092536B2
:10F16000310520F16CE870E082EE9BE00E94764170
:10F170008DED9BE00E947738C457DF4F0FB6F894AF
:10F18000DEBF0FBECDBFDF91CF911F910F91FF90DA
:10F19000EF90DF90CF90BF90AF909F908F907F9037
:10F1A0006F905F904F903F902F9008959A8B898B2E
:10F1B0008CE40E94AF1E8823E1F00E94B5246B010D
:10F1C0007C01C986DA86EB86FC8620E030E0A90166
:10F1D0000F94DE3387FD0AC020E030E040E050E4C9
:10F1E000C701B6010F94AE2A18161CF485EB9BE0FC
:10F1F000C1CF81E50E94611E882331F180911705FE
:10F2000090911805892BE9F00E94B5246B017C01CF
:10F21000CD82DE82EF82F8862DEC3CEC4CE45DE39F
:10F220000F94DE3387FD0AC020E030E040E751E470
:10F23000C701B6010F94AE2A181634F484E89BE097
:10F2400099CF89E59BE096CF83E50E94AF1E882386
:10F25000E9F00E94B5246B017C01CD8ADE8AEF8A39
:10F26000F88E2DEC3CEC4CEC5DE30F94DE3387FD27
:10F270000AC020E030E040E050E4C701B6010F943E
:10F28000AE2A18161CF482E39BE074CF80E50E943E
:10F29000611E882341F18091170590911805892BF3
:10F2A00019F48AEF9AE066CF8BA58F5F8BA70E9437
:10F2B000B5246B017C01CD86DE86EF86F88A20E0DE
:10F2C00030E0A9010F94DE3387FD0AC020E030E072
:10F2D00048EC51E4C701B6010F94AE2A18161CF48D
:10F2E00082ED9AE047CF86E40E94AF1E8823E9F0C2
:10F2F0000E94B5246B017C01C98EDA8EEB8EFC8EE8
:10F3000020E030E040E85FE30F94DE3387FD0AC081
:10F3100020E030E040E850E4C701B6010F94AE2A87
:10F3200018161CF489EA9AE025CFC98CDA8CEB8C8C
:10F33000FC8C8D889E88AF88B88CA7019601C70188
:10F34000B6010F94142B9B01AC0160E070E084E4E3
:10F3500090E40F94783229813A814B815C810F943B
:10F36000142B2B013C01A5019401C501B4010F949C
:10F37000142BA70196010F94142B2CEE31E548EBCA
:10F380005DE30F9478329B01AC01C301B2010F948D
:10F39000142B69837A838B839C8388E40E94AF1E3D
:10F3A000882379F00E94A224009759F09C01255AE5
:10F3B00031092838310518F08BE79AE0DBCE9C8BB9
:10F3C0008B8B85E50E94611E8823C9F00E94D2A91B
:10F3D000611571058105910511F00F943426809116
:10F3E000170590911805892B91F00E94B524609320
:10F3F000130570931405809315059093160582E507
:10F400000E94611E811108C087E49AE0B3CE60E0DB
:10F4100070E088E492E4EBCF809117059091180595
:10F42000892B61F00E94A224AD969FAF8EAFAD975D
:10F43000181619064CF083E19AE09CCE2AE130E0E0
:10F44000AD963FAF2EAFAD9789E50E94AF1E8823E2
:10F4500081F10E94B5242091EF083091F00840918D
:10F46000F1085091F2080F947D316B017C0188E521
:10F470000E94AF1E882331F10E94B5242091EB0831
:10F480003091EC084091ED085091EE080F947D31D9
:10F490006BA37CA38DA39EA3CFA2D8A6E9A6FAA6B0
:10F4A000CE0183960E94201E811115C089EE99E03D
:10F4B00061CEC0906D02D0906E02E0906F02F0902D
:10F4C0007002D5CF6091690270916A0280916B02DF
:10F4D00090916C02DDCF84E40E94611E91E0892747
:10F4E0000E94976980E090E0A0EAB0E48DA79EA713
:10F4F000AFA7B8AB60E0CE018D960E945165309108
:10F500001408CD57DF4F3883C358D04010921408E9
:10F510000E941A1C88EC99E00E94773889899A89A0
:10F520008A3191050CF044C08B899C890E94371F59
:10F5300061E080E00E94AEBF811142C06FEF8DEDAF
:10F5400099E00E94E63F8CA5811104C0CE0101968E
:10F550000F94F31D80E090E0A0EAB0E48093970759
:10F5600090939807A0939907B0939A071DA61EA69B
:10F570001FA618AABE01635D7F4F8FE897E00E9427
:10F580001075CD57DF4F5881C358D04050931408A1
:10F590000E941A1C8AA18111EFCD1092EA111092DB
:10F5A000E9110E9466C190E080E00E94371FE4CD1F
:10F5B0000E94752281E00E9437BE8111B5CFBECF77
:10F5C00010927502109276021092770210927802D1
:10F5D00085E792E00E94BF618BA5882309F452C0A1
:10F5E00020E030E040E751E46091D50C7091D60CFA
:10F5F0008091D70C9091D80C0F9478326DA77EA78C
:10F600008FA798AB80E1E9E6F2E0AFE8B7E00190C0
:10F610000D928A95E1F72D853E854F855889609139
:10F620009B0770919C0780919D0790919E070F9476
:10F630007E3160939B0770939C0780939D07909306
:10F640009E07CE018D960E94EE722D853E854F85D8
:10F65000588960919B0770919C0780919D079091BC
:10F660009E070F947D3160939B0770939C07809356
:10F670009D0790939E078CA5811104C0CE01019631
:10F680000F94F31DEEE0F5E085E0DF011D928A9511
:10F69000E9F780E1E9E6F2E0AFE8B7E001900D922A
:10F6A0008A95E1F789859A85AB85BC858093970714
:10F6B00090939807A0939907B0939A071DA61EA64A
:10F6C0001FA618AABE01635D7F4F8FE897E00E94D6
:10F6D0001075BE01635E7F4F8FE897E00E94107542
:10F6E00089A1882309F41CC42091690230916A021F
:10F6F00040916B0250916C02E5962CAF3DAF4EAF3E
:10F700005FAFE59780916D0290916E02A0916F02BC
:10F71000B0917002E1968CAF9DAFAEAFBFAFE197F5
:10F72000312C212C9FEFA4969FAFA497AFEFA89602
:10F73000AFAFA897BFEFC158DF4FB883CF57D040C6
:10F74000EFE4C058DF4FE883C058D040F3ECCF5708
:10F75000DF4FF883C158D04027E4CE57DF4F2883CE
:10F76000C258D04081E090E0A0E0B0E0022C04C09C
:10F77000880F991FAA1FBB1F0A94D2F7CC57DF4FDF
:10F7800088839983AA83BB83C458D040AEE0B5E098
:10F79000E796BFAFAEAFE79710E000E09101032C12
:10F7A000000C440B550BC857DF4F288339834A831D
:10F7B0005B83C858D040C457DF4F2882CC58D04014
:10F7C000E796AEADBFADE7978D91E796BFAFAEAF11
:10F7D000E79790E0B0E0A0E0CC57DF4F2881398177
:10F7E0004A815B81C458D04082239323A423B5234C
:10F7F000892B8A2B8B2B09F024C1C857DF4F6881D6
:10F8000079818A819B81C858D0400F94B52A209174
:10F81000E9053091EA054091EB055091EC050F9414
:10F82000142B2091E1053091E2054091E3055091C0
:10F83000E4050F947E31EB966CAF7DAF8EAF9FAF3A
:10F84000EB97B801012E000C880B990B0F94B52A89
:10F850002091ED053091EE054091EF055091F005B6
:10F860000F94142B2091E5053091E6054091E705B2
:10F870005091E8050F947E316B017C01EB962CAD25
:10F880003DAD4EAD5FADEB97E5966CAD7DAD8EAD0C
:10F890009FADE5970F947D312B013C01A7019601A7
:10F8A000E1966CAD7DAD8EAD9FADE1970F947D314E
:10F8B0004B015C01A3019201C301B2010F94142B0F
:10F8C0002B013C01A5019401C501B4010F94142B37
:10F8D0009B01AC01C301B2010F947E310F942C3413
:10F8E0004B015C01EB962CAD3DAD4EAD5FADEB97A2
:10F8F0006BA17CA18DA19EA10F947D312B013C01B8
:10F90000A70196016FA178A589A59AA50F947D31CD
:10F910006B017C01A3019201C301B2010F94142B6E
:10F920002B013C01A7019601C701B6010F94142BCE
:10F930009B01AC01C301B2010F947E310F942C34B2
:10F9400020E030E040E751E40F947832A5019401C3
:10F950000F947E316B017C0180901305909014050B
:10F96000A0901505B090160520E030E040E85FE378
:10F97000C501B4010F94DE331816F4F4C501B401C7
:10F980000F94EA324B015C0160E070E0CB01181487
:10F9900019041A041B0434F40F94E525A5019401FD
:10F9A0000F9414310F94B52A9B01AC01B601C70125
:10F9B0000F947E316B017C01C158DF4F2881CF57F6
:10F9C000D040C058DF4F3881C058D040CF57DF4FAC
:10F9D0004881C158D040CE57DF4F5881C258D040DF
:10F9E000B601C7010F94AE2A87FF2BC0A4960FAFB4
:10F9F000A497C457DF4F3881CC58D040A8963FAF6A
:10FA0000A897EC96CFAEEC97ED96DFAEED97EE961D
:10FA1000EFAEEE97EF96FFAEEF97C158DF4FC8827B
:10FA2000CF57D040C058DF4FD882C058D040CF57B2
:10FA3000DF4FE882C158D040CE57DF4FF882C2581E
:10FA4000D0400F5F1F4F0530110509F0B9CE4FEFC1
:10FA5000241A340A55E02516310409F083CEA49601
:10FA60008FADA497E82FF0E0E25FFA4F208181E0AC
:10FA700090E0A0E0B0E0A8960FACA89704C0880F73
:10FA8000991FAA1FBB1F0A94D2F7822B8083A896C6
:10FA90009FADA8976A969FAF6A97A496AFADA497BB
:10FAA0006B96AFAF6B97EC968FADEC97ED969FADE5
:10FAB000ED97EE96AFADEE97EF96BFADEF976F96E1
:10FAC0008CAF9DAFAEAFBFAF6F97A896BFADA897F5
:10FAD000BF3F09F409C2A496EFADA497EF3F09F424
:10FAE00003C26B2FBB0F770B880B990B0F94B52AB2
:10FAF0002091E9053091EA054091EB055091EC0524
:10FB00000F94142B2091E1053091E2054091E3051B
:10FB10005091E4050F947E31162F072F382E292E91
:10FB2000862F902FA32DB22D65968CAF9DAFAEAFD3
:10FB3000BFAF6597A496FFADA4976F2FFF0F770B0C
:10FB4000880B990B0F94B52A2091ED053091EE05A5
:10FB50004091EF055091F0050F94142B2091E5058D
:10FB60003091E6054091E7055091E8050F947E310C
:10FB70006B017C016996CCAEDDAEEEAEFFAE69974F
:10FB8000CE018F5A9F4F0E94201E882309F4B0C1D6
:10FB900020E030E040EA50E4612F702F832D922D59
:10FBA0000F947E314B015C01CB01D50121968CAFC6
:10FBB0009DAFAEAFBFAF21972596CCAEDDAEEEAE1A
:10FBC000FFAE2597A8962FADA8972111E3C1A49663
:10FBD0003FADA4973111B3C120E030E040EA50E4DA
:10FBE000C701B6010F947E316B017C01A4964FAD25
:10FBF000A497442309F4C5C1A4968FADA49784307B
:10FC00000CF0BFC122ED422E23E5522E2BE7622ECF
:10FC100021E4722E21968CAC9DACAEACBFAC21978A
:10FC200025968CAD9DADAEADBFAD2597A7968CAF9B
:10FC30009DAFAEAFBFAFA7979C01AD0169966CAD0C
:10FC40007DAD8EAD9FAD69970F947D31AB966CAF56
:10FC50007DAF8EAF9FAFAB97A501940165966CAD5C
:10FC60007DAD8EAD9FAD65970F947D312D966CAFB8
:10FC70007DAF8EAF9FAF2D97AB962CAD3DAD4EAD0A
:10FC80005FADAB9761962CAF3DAF4EAF5FAF619765
:10FC9000A50194016091690270916A0280916B02E2
:10FCA00090916C020F947D314B015C01A7962CADB5
:10FCB0003DAD4EAD5FADA79760916D0270916E0244
:10FCC00080916F02909170020F947D31A7966CAF76
:10FCD0007DAF8EAF9FAFA797812F902FA32DB22D11
:10FCE0008DA79EA7AFA7B8ABC9AADAAAEBAAFCAAB0
:10FCF000C984DA84EB84FC84CDAADEAAEFAAF8AE2C
:10FD00002DEC3CEC4CEC5CE3C301B2010F94142BE2
:10FD100029813A814B815C810F94142B20917502CB
:10FD20003091760240917702509178020F947E31A3
:10FD300069AF7AAF8BAF9CAFA5019401C501B40147
:10FD40000F94142B4B015C01A7962CAD3DAD4EAD2D
:10FD50005FADA797CA01B9010F94142B9B01AC01A9
:10FD6000C501B4010F947E3120E030E040E050E462
:10FD70000F94DE331816ACF420E030E040E05FE38F
:10FD8000C701B6010F947E3129966CAF7DAF8EAF5F
:10FD90009FAF2997BE01635C7F4FCE0101960E9401
:10FDA000B37489859A85AB85BC8529968CAF9DAF48
:10FDB000AEAFBFAF2997A3961CAE1DAE1EAE1FAE51
:10FDC000A397BE01615A7F4FCE01CD960E94107558
:10FDD0008CA58823C1F02AE939E949E95FE36D81FF
:10FDE0007E818F8198850F94142BA3966CAF7DAF85
:10FDF0008EAF9FAFA397BE01615A7F4F8FE897E008
:10FE00000E9410751CA6E090CD0CF090CE0C0091D5
:10FE1000CF0C1091D00CA090C90CB090CA0CC0901F
:10FE2000CB0CD090CC0C9501A601B701C8010F9462
:10FE3000DE33181614F47501860180904902909003
:10FE40004A02A0904B02B0904C022DEC3CEC4CECE2
:10FE50005DE3B701C8010F94142B609349027093BE
:10FE60004A0280934B0290934C0240E0BE01675BD4
:10FE70007F4FCE018D960E9420C980E1E9E6F2E035
:10FE8000AFE8B7E001900D928A95E1F780924902C0
:10FE900090924A02A0924B02B0924C0220E04FEFA7
:10FEA000BE01675A7F4FCE0101960E948B7620E0FB
:10FEB00041E0BE01675A7F4FCE0101960E948B76CA
:10FEC0002FEF40E0BE01675A7F4FCE0101960E949E
:10FED0008B7621E040E0BE01675A7F4FCE0101964C
:10FEE0000E948B760E94AE6180910B0D80930C0D69
:10FEF000AD964EAD5FADAD9741505109AD965FAF38
:10FF00004EAFAD97452B09F419CB6A968FAD6A9722
:10FF100087FD14CB6B968FAD6B9787FFE1CB0ECB34
:10FF20002BA13CA14DA15EA1E5962CAF3DAF4EAFFC
:10FF30005FAFE5978FA198A5A9A5BAA5EBCB812FB7
:10FF4000902FA32DB22D21968CAF9DAFAEAFBFAF3A
:10FF5000219720E030E040EA50E4C701B6010F9459
:10FF60007D3125966CAF7DAF8EAF9FAF2597A49660
:10FF70005FADA49754300CF42FCE182D092D3A2CD8
:10FF80002B2C92ED492E93E5592E9BEF692E90E490
:10FF9000792E40CEA8969FADA89794300CF452C00D
:10FFA000A496AFADA497A4300CF120E030E040EA75
:10FFB00050E4612F702F832D922D0F947D31219667
:10FFC0006CAF7DAF8EAF9FAF219720E030E040EA6D
:10FFD00050E4C701B6010F947D316B017C01A496FA
:10FFE000EFADA497E4300CF40DCECBCF812F902F42
:10FFF000A32DB22D21968CAF9DAFAEAFBFAF219791
:020000021000EC
:1000000020E030E040EA50E4C701B6010F947E31B1
:1000100025966CAF7DAF8EAF9FAF2597A496BFADF1
:10002000A497B111D2CF20E030E040EA50E4612F34
:10003000702F832D922D0F947D31162F072F382E80
:10004000292E9FCFA496FFADA497F1110DC020E0FB
:1000500030E040E251E4B401C5010F947D31162F28
:10006000072F382E292ECECDA4962FADA49724305D
:100070009CF020E030E040E251E4B401C5010F946F
:100080007D3121966CAF7DAF8EAF9FAF2197182D3C
:10009000092D3A2C2B2CB6CD182D092D3A2C2B2CB2
:1000A00082ED482E83E5582E8BEF682E81E4782E62
:1000B000B1CD2F923F924F925F926F927F928F922B
:1000C0009F92AF92BF92CF92DF92EF92FF920F93E7
:1000D0001F93CF93DF93CDB7DEB7C054D1090FB6CE
:1000E000F894DEBF0FBECDBF8091A00C888B87E552
:1000F0000E94611E882309F423C120E030E0A90199
:100100006091E9057091EA058091EB059091EC050D
:100110000F94AE2A811108C00E94474E8DE09DE0E9
:100120000E94773810E01FC18AE50E94AF1E882325
:1001300039F10E94B5242091F3083091F4084091E0
:10014000F5085091F6080F947D316B017C0120E099
:1001500030E040E251ECC701B6010F94DE3387FD79
:100160000AC020E030E040E251E4C701B6010F943C
:10017000AE2A181674F40E94474E80E09DE0D0CF5E
:10018000C0907102D0907202E0907302F0907402FD
:10019000DECF40E050E060EC7FE788E50E94DF249E
:1001A0002091EB083091EC084091ED085091EE0859
:1001B0000F947D312B013C0140E050E060EC7FE783
:1001C00089E50E94DF242091EF083091F0084091EA
:1001D000F1085091F2080F947D314B015C016FEFF3
:1001E00089E40E947124182F6FEF8AE40E94712421
:1001F000082FA3019201C301B2010F947034811141
:100200006EC0A5019401C501B4010F947034811131
:1002100066C08BA19CA1ADA1BEA18BAB9CABADABCD
:10022000BEAB2091E1053091E2054091E30550918C
:10023000E405C301B2010F947D312B013C0120E0A4
:1002400030E040E05FE36BA97CA98DA99EA90F94E3
:10025000142B9B01AC01C301B2010F947E312BA979
:100260003CA94DA95EA90F9478320F94EA32162F5B
:100270004FA058A469A47AA42091E5053091E60521
:100280004091E7055091E805C501B4010F947D3117
:100290004B015C0120E030E040E05FE3C301B201CC
:1002A0000F94142B9B01AC01C501B4010F947E3156
:1002B000A30192010F9478320F94EA32062F812F16
:1002C000012E000C990B97FD33C005979CF5802FEC
:1002D000002E000C990B97FD2FC005977CF515306B
:1002E00008F020CF053008F01DCF80E00E9497690C
:1002F00095E01902F0011124E00FF11D07FDFA95B8
:10030000EE0FFF1FEE0FFF1FE555F84FC082D182A1
:10031000E282F382602F812F0F94171A88890E943E
:1003200097698889882309F4FDCE0E94CC30FACEE3
:1003300010E0CDCF14E0CBCF00E0D1CF04E0CFCFA1
:100340008AE40E94611E182F811128C070E060E0CD
:1003500086E50E94A6249A838983059710F18BED88
:100360009CE00E947738812FC05CDF4F0FB6F89475
:10037000DEBF0FBECDBFDF91CF911F910F91FF90D8
:10038000EF90DF90CF90BF90AF909F908F907F9035
:100390006F905F904F903F902F9008950E94756FDF
:1003A000C1CE60E084E40E948D248F8740E050E05D
:1003B000BA018AE50E94DF246BA77CA78DA79EA7C0
:1003C00040E050E86BE376E483E50E94DF2420E020
:1003D00030E040E752E40F94783260934502709326
:1003E00046028093470290934802E090EB12F0900F
:1003F000EC12D7014D905D906D907C9020E030E044
:10040000A901C301B2010F947E31962E872E382E9A
:10041000292E20E030E040E450E40F94AE2A87FF1C
:1004200006C0912C812CB0E43B2E00E4202E20E06D
:1004300030E040EB53E4C301B2010F947E316BAB6B
:100440007FAB88AF99AF20E030E84EEA53E40F94D9
:10045000DE3318163CF41BAAB0E8BFABEEEAE8AFF7
:10046000F3E4F9AFD70114964D905D906D907C90B8
:10047000179720E030E0A901C301B2010F947E314B
:100480005B016C0120E030E040EE51E40F94AE2AB5
:1004900087FF06C0A12CB12CF0EECF2EA1E4DA2EFE
:1004A00020E030E044EB53E4C301B2010F947E310D
:1004B0007B01082F9AAF20E030E046EA53E40F9426
:1004C000DE3318162CF4E12CF12C06EAB3E4BAAFB3
:1004D00088E40E94611E882309F41AC20E94B52490
:1004E0000F94EA322B0177FF02C06F5F7F4F759543
:1004F0006795EE27FF27E61BF70B2196FFAFEEAFC0
:100500002197BF016C547F4F072E000C880B990B6D
:100510000F94B52A6BAF7CAF8DAF9EAF9501A6014E
:100520000F94DE33181624F0ABAEBCAECDAEDEAE0B
:1005300021966EAD7FAD219760557F4F072E000C41
:10054000880B990B0F94B52A5B016C01292D382D6E
:10055000432D522D0F94DE33181624F0A92CB82CFD
:10056000C32CD22CC501D6018B8B9C8BAD8BBE8B43
:100570008BAD9CADADADBEAD8F8B988FA98FBA8F73
:10058000B201550C880B990B0F94B52A2B013C0135
:10059000AC019B016BAD7CAD8DAD9EAD0F947E31FA
:1005A0001B014C019701402F5AAD0F94AE2A87FFD3
:1005B00003C07101082D9AAEA3019201B501C601D5
:1005C0000F947E315B016C012BA93FA948AD59AD59
:1005D0000F94AE2A87FF04C0ABAABFAAC8AED9AE9B
:1005E0008BA99FA9A8ADB9AD8B8F9C8FAD8FBE8F06
:1005F000C701A02FBAAD8F8F98A3A9A3BAA3BE013C
:10060000695E7F4FCE0143960E946C2E882309F4C9
:10061000ADC1BE01615E7F4FCE014B960E946C2E34
:10062000E82E882309F4A2C12F89388D498D5A8D6F
:100630006F8D78A189A19AA10F947D3120E030E0DF
:1006400040E85EE30F94142B4B015C012B893C893D
:100650004D895E896B8D7C8D8D8D9E8D0F947D3146
:1006600020E030E040E85EE30F94142B6BA37CA302
:100670008DA39EA38FA298A6A9A6BAA689819A81C6
:100680001816190674F489EA9CE00E9477388F8561
:10069000882321F08FE99CE00E9477388AE00E944D
:1006A0003E380E94AE610E94F61C80E00E9497696D
:1006B00080E090E0A0E2B1E48FA798ABA9ABBAAB21
:1006C00060E0CE018F960E9451652091E90530913E
:1006D000EA054091EB055091EC056BA17CA18DA141
:1006E0009EA10F94AE2A811130C02091ED0530916A
:1006F000EE054091EF055091F0056FA178A589A511
:100700009AA50F94AE2A811120C02091E105309165
:10071000E2054091E3055091E4056B897C898D8960
:100720009E890F94AE2A811110C02091E505309169
:10073000E6054091E7055091E8056F89788D898D30
:100740009A8D0F94AE2A8823A9F00E94756F88E0D5
:10075000FE01B396A9EEB5E001900D928A95E1F7FE
:1007600088E0FE017396A1EEB5E001900D928A95A6
:10077000E1F7188A60E085E40E948D24882309F45B
:10078000F8C0F1E0FBAB1B861C861D861E861A8A0C
:100790009E2C4FE6C42E4CE0D42E5DE7A52E5CE0E7
:1007A000B52E1A8915300CF0F4C06B857C858D85CB
:1007B0009E859B01AC010F9470348111EAC0992091
:1007C00009F4DAC031E03FAB35E0232E91E0992601
:1007D000F12EFF0CFF0CF10EF394898B19896A89B5
:1007E000121509F4D2C0062E000C770B880B990B5A
:1007F0000F94B52A2FA138A549A55AA50F94142BFB
:100800002F89388D498D5A8D0F947E312B013C01F3
:10081000612F110F770B880B990B0F94B52A2BA121
:100820003CA14DA15EA10F94142B2B893C894D89CD
:100830005E890F947E316B837C838D839E834F8290
:10084000588669867A8689819A81892B79F06F2DFD
:100850008BE89CE00E944C4169E170E089E89CE0F3
:100860000E94764186E89CE00E9477381F9299E1C9
:100870009F931F92FF92DF92CF92BF92AF921F92EF
:100880000F94421B29814BA9BE01695F7F4FCE01A6
:1008900003960F94061C2B013C014B865C866D86EB
:1008A0007E860FB6F894DEBF0FBECDBFAC019B01B4
:1008B0000F947034811166C089883A8825E0382DFC
:1008C000320380011124030D111D37FC1A95000F0E
:1008D000111F000F111F0555184FA30192016BA5A1
:1008E0007CA58DA59EA50F947E31D8016D937D9337
:1008F0008D939C931397632D882D0F94171A188A44
:1009000081E00E944A5AF3948989BFA98B0F65CF71
:10091000A501B60186E40E94DF242B013C01492D8C
:10092000582D632D722D8CE40E94DF246B8B7C8B01
:100930008D8B9E8B4F8A588E698E7A8EA701602F81
:100940007AAD82E40E94DF246B017C014BA95FA990
:1009500068AD79AD82E50E94DF246B8F7C8F8D8F2F
:100960009E8FCF8ED8A2E9A2FAA249CE8FEB9CE04F
:10097000F8CC22E02BAB07CF8FEF8FAB22242A9449
:1009800084E024CF88890E9497698A898F5F8A8B47
:1009900008CF0E94A3ED0E942766882359F088891A
:1009A0000E94976980E090E0A0ECBFE78B879C876E
:1009B000AD87BE876B857C858D859E859B01AC014F
:1009C0000F947034811159C08F85811126C082E047
:1009D000F82E02E094E0C92E12E0DC2CD11A21E0BE
:1009E00041E0612F802F0E948E2221E04FEF612F86
:1009F0008F2D0E948E222FEF41E06D2D802F0E94BF
:100A00008E222FEF4FEF6D2D8F2D0E948E221150D1
:100A100020F70150F3940F3FF9F60E94BD400E9469
:100A2000BC1E8F85811124C081E792E00E94A61D23
:100A30004B015C0189E692E00E944C1F9B01AC01D6
:100A4000C501B4010F94142B9B01AC01609171029C
:100A50007091720280917302909174020F947D31B3
:100A60006093710270937202809373029093740288
:100A70008F858111E888E092A00C0E94DD1C809196
:100A8000A00C81110E94192B0E9411680E94CC3089
:100A90006B857C858D859E8511E09B01AC010F9453
:100AA0007034811160CC3ECB8F929F92AF92BF92F7
:100AB000CF92DF92EF92FF920F931F93CF93DF932A
:100AC00000D01F92CDB7DEB75C016B017A01122F07
:100AD0000023E1F10E944B4E88E999E00E947738AB
:100AE00061E0812F0E946B3A9090280583E080930B
:100AF000280581E080939E0C0E94634082E08093F1
:100B0000F81140E368E879E084E799E00E946840E2
:100B100040E069E171E18DE699E00E94684061E0A2
:100B200088E699E00E944A408AE799E00E944A22BA
:100B300080919E0C882341F060E0812F0E946B3AE7
:100B400081E00E944A5AF4CF9092280520E030E0DC
:100B5000A901F50160817181828193810F94AE2A90
:100B6000882371F080E090E0A0ECB0E489839A8360
:100B7000AB83BC83BE016F5F7F4FC5010E94D76806
:100B800020E030E0A901F6016081718182819381CA
:100B90000F94AE2A882351F18090DD0C9090DE0CEA
:100BA000A090DF0CB090E00C80E090E0A0E7B1E412
:100BB0008093DD0C9093DE0CA093DF0CB093E00CDF
:100BC00080E090E0A0EAB1E489839A83AB83BC83A0
:100BD000BE016F5F7F4FC6010E94D7688092DD0C17
:100BE0009092DE0CA092DF0CB092E00C20E030E09E
:100BF000A901F70160817181828193810F94DE33B5
:100C0000181674F480E090E0A0E4B0E489839A833D
:100C1000AB83BC83BE016F5F7F4FC7010E94D76863
:100C20008091FD0429E131E1882311F029E439E0C4
:100C300047E559E061E679E081E00E948B400E943F
:100C4000634081E00F900F900F900F90DF91CF9154
:100C50001F910F91FF90EF90DF90CF90BF90AF90DA
:100C60009F908F900895CF93C82F80915D0C83FD46
:100C700014C080912209811110C080916702909167
:100C800068029C0121503109409154125091551233
:100C90004217530714F40E94371FCC2329F061E058
:100CA00080E0CF910C94AEBF8091220991E089271A
:100CB0008093440280914402882389F080915212EB
:100CC000909153122091541230915512821B930B24
:100CD00097FF03C0919581959109029744F4109272
:100CE000440280915D0C83FF06C0C1E01AC080E021
:100CF0000E944A5ADFCFC0912209C11112C08091CF
:100D00006702909168020197209154123091551218
:100D10002817390754F70E944B4E8BE299E00E9446
:100D200077388C2FCF910895AF92BF92CF92DF92F8
:100D3000EF92FF920F931F93CF93DF93CDB7DEB760
:100D400064970FB6F894DEBF0FBECDBF0E944A4F26
:100D500087FDAFC08AE50E94AF1E882309F4BAC0A0
:100D600040E050E0BA018AE50E94DF247B018C015B
:100D7000209171023091720240917302509174027D
:100D800060E070E088EC93E40F947D315B016C01CE
:100D90009701A8010F94DE33181614F0750186012F
:100DA00020E030E0A901B701C8010F94DE33181626
:100DB00024F4E12CF12C00E010E0B701C8010F94FD
:100DC000EA32072E000C880B990B0F94B52A698B19
:100DD0007A8B8B8B9C8B20E030E0A9010F94AE2A9C
:100DE000882321F0CE0141960E94557380E090E067
:100DF000A0EAB1E48D879E87AF87B88B19861A86E3
:100E00001B861C868CE40E94611E882309F467C03F
:100E10000E94B5246B017C0120E030E0A901C701EC
:100E2000B6010F94DE3387FF04C0F7FAF094F7F8A9
:100E3000F094CD82DE82EF82F886209154123091B8
:100E400055122430310574F0809152129091531252
:100E5000821B930B97FF03C091958195910901E047
:100E600004970CF400E080E00E943386882359F058
:100E700022E0AE01435F5F4FBE016B5F7F4FCE014B
:100E800009960E94548569897A898B899C898B018E
:100E90009C01305809831A832B833C8320E030E087
:100EA000A9010F94AE2A882321F0CE0101960E9459
:100EB000557364960FB6F894DEBF0FBECDBFDF91B9
:100EC000CF911F910F91FF90EF90DF90CF90BF9047
:100ED000AF900895E12CF12C00E211E449CFC090CD
:100EE000DC05D090DD05E090DE05F090DF0594CFC5
:100EF0007F928F929F92AF92BF92CF92DF92EF92AA
:100F0000FF920F931F93CF93DF9300D000D01F92D7
:100F10001F92CDB7DEB76C015B014A01722E7801DA
:100F2000009129060E94431F8091541290915512FE
:100F30008E159F051CF4C7010E94371F80E00E9498
:100F40003386882331F0272DA401B501C6010E9404
:100F500054851E141F043CF4C7010E94371F60E033
:100F600080E00E94AEBF81E00E94338680E090E086
:100F7000A0E7B2E489839A83AB83BC8380E090E0EE
:100F8000A0E8B0EC8D839E83AF83B887BE016F5F0E
:100F90007F4FCE0105960E94D76887E00E94302AD5
:100FA000811158C08091710290917202A0917302D8
:100FB000B0917402409102055091030560910405BF
:100FC00070910505C090FE04D090FF04E0900005EC
:100FD000F0900105C0928F07D0929007E0929107A0
:100FE000F09292074093930750939407609395076C
:100FF000709396078093970790939807A09399070B
:10100000B0939A0780E090E0A8E4B2E489839A83E1
:10101000AB83BC83CE0101960E94EE7280910605DF
:1010200090910705A0910805B09109058093970755
:1010300090939807A0939907B0939A0780E090E067
:10104000A0EAB0E489839A83AB83BC83CE01019686
:101050000E94EE72C12CD12C80E7E82E82E4F82E9B
:10106000C982DA82EB82FC8280E090E0A0E8B0E402
:101070008D839E83AF83B887BE016F5F7F4FCE01A4
:1010800005960E94D76820E030E0A90160910A052A
:1010900070910B0580910C0590910D050F94AE2A6F
:1010A00087FF0BC0C982DA82EB82FC82BE016F5FD0
:1010B0007F4F8AE095E00E94D76880910A05909161
:1010C0000B05A0910C05B0910D05809375029093CE
:1010D0007602A0937702B093780280939B07909357
:1010E0009C07A0939D07B0939E078BE997E00E9411
:1010F000BF618091E00581110F945D1961E087EB7C
:1011000099E00E94B33F80918A11815080938A11A7
:1011100048E958E16FEB79E085E00E94B1EB8091FE
:101120008A11882339F00E94E7AD80918A1181509D
:1011300080938A1180E00F94241B0E94C631809115
:101140008B11823011F40E9485380E94A3ED2896FD
:101150000FB6F894DEBF0FBECDBFDF91CF911F91C8
:101160000F91FF90EF90DF90CF90BF90AF909F9046
:101170008F907F900895CF92DF92EF92FF920F931E
:101180001F93CF93DF9300D01F92CDB7DEB77C01C2
:101190006B018A0161E08CE399E00E94B33F48E96A
:1011A00058E163E479E085E00E94B1EB90918A1107
:1011B00081E0890F80938A118091A81482FF06C074
:1011C0008B7F8093A8149E5F90938A110E94773939
:1011D00080E1E9E6F2E0AEEFB4E001900D928A958D
:1011E000E1F70E94AE6181E00F94241B20E030E023
:1011F000A901F70160817181828193810F94AE2AE8
:101200008823F1F08091220981110CC0809167023E
:101210009091680201972091521230915312281731
:10122000390774F080E090E0A0E7B2E489839A8304
:10123000AB83BC83BE016F5F7F4FC7010E94D7683D
:1012400087E00E94302A811103C0B6010E942B68FA
:1012500020E030E0A901F8016081718182819381F1
:101260000F94AE2A882341F080E00E9433868823C1
:1012700019F0C8010E940769129A64E670E080E0E4
:1012800090E00E94232681E00F900F900F900F9026
:10129000DF91CF911F910F91FF90EF90DF90CF9052
:1012A0000895CF92DF92EF92FF92CF93DF936B017D
:1012B0007C01D42FC091280583E08093280581E02C
:1012C00080939E0CC114D104E104F10431F00E941A
:1012D000D2A9C60ED71EE81EF91E80919E0C882347
:1012E00089F0C114D104E104F10421F48D2F0E948E
:1012F0004A5AF3CF0E94D2A96C197D098E099F0921
:1013000097FDF4CF10929E0CC0932805DF91CF91EA
:10131000FF90EF90DF90CF9008950F931F93CF939E
:10132000DF93C82F162F0E944B4EC11194C0CFE8F7
:10133000D8E0CE010E94773861E0812F0E946B3A9D
:101340000E94D2A9685370458F4F9F4F6093250626
:1013500070932606809327069093280610922906FC
:101360000091280583E08093280530E020E049E1E2
:1013700051E16DE179E082E00E948B408DE199E0DE
:101380000E944A2281E080939E0C80919E0C8823CB
:1013900009F464C060E0812F0E946B3A80912906B5
:1013A000882309F454C00E944B4E83E099E00E94C8
:1013B000773830E020E04DEE58E064EF78E082E0EE
:1013C0000E948B4084EF98E00E944A2241E060E056
:1013D00070E0CB010E94518930E020E050E040E015
:1013E00060EE78E085E00E948B4080EE98E00E94FD
:1013F000CD350E94431F80E00E9433860E944B4EF1
:10140000CE010E9477380E94D2A9685370458F4F51
:101410009F4F60932506709326068093270690932E
:1014200028061092290630E020E049E151E164ED00
:1014300078E082E00E948B4083EC98E00E944A2290
:1014400081E080939E0C61E0812F0E946B3A81E0E5
:101450000E944A5A9ACFC4EAD8E06BCF009328057D
:10146000DF91CF911F910F910895CF92DF92EF926C
:10147000FF920F931F93CF93DF93CDB7DEB7A09763
:101480000FB6F894DEBF0FBECDBF0E944A4F87FD56
:10149000CCC085E40E94611E882309F4D5C00E9457
:1014A000B5246B017C0120E030E0A9010F94DE330C
:1014B00087FF04C0F7FAF094F7F8F094F7FAF09485
:1014C000F7F8F094CD8EDE8EEF8EF8A28CE0EEED84
:1014D000F2E0DE01119601900D928A95E1F78AE51E
:1014E0000E94AF1E882351F040E050E0BA018AE527
:1014F0000E94DF2469877A878B879C8788E50E9412
:10150000AF1E882351F040E050E0BA0188E50E9408
:10151000DF2469837A838B839C8389E50E94AF1ED5
:10152000882351F040E050E0BA0189E50E94DF24B1
:101530006D837E838F83988785E50E94611E882353
:1015400009F489C00E94B5246B017C0120E030E0E1
:10155000A901C701B6010F94DE3387FF04C0F7FA73
:10156000F094F7F8F094F7FAF094F7F8F094C98E45
:10157000DA8EEB8EFC8E1D8A1E8A1F8A188E8CE4F2
:101580000E94611E882309F46FC00E94B5246B017C
:101590007C0120E030E0A901C701B6010F94DE33E1
:1015A00087FF04C0F7FAF094F7F8F094C98ADA8A52
:1015B000EB8AFC8A62E070E082E40E94A624F82EA6
:1015C00080918A11811131C021E0AE01475E5F4FE9
:1015D000BE016F5F7F4FCE014D960E94BB8888236E
:1015E00021F16F2D81E00E948D8982E50E94AF1E5E
:1015F000882309F442C00E94A22440E050E060EA3F
:1016000071E44D875E876F87788B20918A11222342
:1016100061F08C012F2DAE01435F5F4FBE016F5E05
:101620007F4FCE0145960E947887A0960FB6F8941A
:10163000DEBF0FBECDBFDF91CF911F910F91FF9005
:10164000EF90DF90CF900895C12CD12C80E8E82E48
:1016500080E4F82E33CFC090D805D090D905E09023
:10166000DA05F090DB0572CFC090DC05D090DD0587
:10167000E090DE05F090DF058CCF90E080E0BDCFFC
:10168000CF92DF92EF92FF920F931F93CF93DF934E
:10169000CDB7DEB76C970FB6F894DEBF0FBECDBFE7
:1016A0008CE40E94611E882309F4B0C00E94B52416
:1016B0006B017C0120E030E0A9010F94DE3387FF4D
:1016C00004C0F7FAF094F7F8F094F7FAF094F7F80A
:1016D000F094C98EDA8EEB8EFC8E8CE0EEEDF2E0AB
:1016E000DE01119601900D928A95E1F788E50E943E
:1016F000AF1E8823A1F040E050E0BA0188E50E94C7
:10170000DF242091EB083091EC084091ED085091D6
:10171000EE080F947D3169837A838B839C8389E5FE
:101720000E94AF1E8823A1F040E050E0BA0189E595
:101730000E94DF242091EB083091EC084091ED08E5
:101740005091EE080F947D316D837E838F8398874F
:101750008AE50E94AF1E882351F040E050E0BA01B4
:101760008AE50E94DF2469877A878B879C871D869C
:101770001E861F86188A80918A11811138C020E048
:10178000AE01435F5F4FBE016F5F7F4FCE01499651
:101790000E94BB88882359F18091E00581110F9444
:1017A0005D1960E080E00E948D89898D9A8DAB8DF6
:1017B000BC8DB0588D8B9E8BAF8BB88F198A1A8ACF
:1017C0001B8A1C8A1D861E861F86188A80918A1194
:1017D000882369F010E000E020E0AE014B5E5F4F2F
:1017E000BE016F5E7F4FCE010D960E9478876C968A
:1017F0000FB6F894DEBF0FBECDBFDF91CF911F9122
:101800000F91FF90EF90DF90CF900895C12CD12CD5
:1018100080E8E82E80E4F82E58CF2F923F924F9226
:101820005F926F927F928F929F92AF92BF92CF9270
:10183000DF92EF92FF920F931F93CF93DF93CDB779
:10184000DEB7E5970FB6F894DEBF0FBECDBF8DAB08
:10185000209128052CAB81E08093280580914605D6
:101860008D3409F4C6C4843511F40C946CA087340B
:1018700009F091C180914405909145058B31910506
:1018800009F4DDC108F079C18430910508F030C158
:101890002091FC068230910508F48EC1213009F0B8
:1018A00091C111E0029709F010E00E94F62419821C
:1018B0001A821B821C821D821E821F82188682E56C
:1018C0000E94AF1E882309F490C10E94B5246B01C9
:1018D0007C0120E030E0A9010F94AE2A882309F4AE
:1018E000EAC04090690250906A0260906B0270906A
:1018F0006C0280916D0290916E02A0916F02B09186
:1019000070028CA79DA7AEA7BFA780908F0790906D
:101910009007A0909107B0909207809193079091C3
:101920009407A0919507B091960788AB99ABAAABA5
:10193000BBABA5019401C301B2010F94AE2A811182
:101940000DC028A939A94AA95BA96CA57DA58EA5BA
:101950009FA50F94AE2A882309F4ADC0A30192017C
:10196000C501B4010F947D3120E030E040E05FE339
:101970000F94142B68A779A78AA79BA72CA53DA530
:101980004EA55FA568A979A98AA99BA90F947D3165
:1019900020E030E040E05FE30F94142B2B013C018A
:1019A00020E030E0A901C701B6010F94AE2A881FDC
:1019B0008827881F181709F40FC180E090E0A0E87D
:1019C000BFEB8CA79DA7AEA7BFA728A539A54AA5A1
:1019D0005BA5CA01B9010F94142B4B015C01A30153
:1019E0009201C301B2010F94142B9B01AC01C501FC
:1019F000B4010F947E310F942C344B015C01AC0187
:101A00009B01C701B6010F947D3168AB79AB8AABFE
:101A10009BABA5019401C701B6010F947E319B01D8
:101A2000AC0168A979A98AA99BA90F94142B6B0111
:101A30007C0120E030E0A9010F94DE3387FDD1C0A6
:101A4000C701B6010F942C346B017C01C301B201B4
:101A50009058A50194010F9478322CA53DA54EA570
:101A60005FA50F94142BA70196010F94142B28A5A2
:101A700039A54AA55BA50F947E3169837A838B8350
:101A80009C83A501940168A579A58AA59BA50F94BF
:101A900078322CA53DA54EA55FA50F94142BA70168
:101AA00096010F94142BA30192010F947E316D8344
:101AB0007E838F83988720E030E0A90169817A8155
:101AC0008B819C810F94AE2A8111A3C020E030E06D
:101AD000A9016D817E818F8198850F94AE2A811135
:101AE00098C00E94474E8BEB9FE00E9477386AC0F7
:101AF0008531910509F466C08A31910509F49CC0CD
:101B0000049709F048C080E50E94AF1EC12CD12C7B
:101B10007601882321F00E942F246B017C0183E54C
:101B20000E94AF1E882361F00E94B52420E030E0BF
:101B30004AE754E40F94142B0F94F1326B017C01AB
:101B40000E94AE6180918C11811105C060E081ED31
:101B50009FE00E94E63F0E94D2A9C60ED71EE81E53
:101B6000F91E0E94D2A96C197D098E099F0997FF61
:101B700029C080E00E944A5AF4CF8A32910509F4C4
:101B8000ADC160F48D31910509F4D6C008F470C080
:101B90004E9709F429C10F94C91B14C08B359105C8
:101BA00009F47FC28C35910509F47FC28A3591050D
:101BB00091F710920F0806C0213021F40E94F624FC
:101BC0000E943B703DA9311102C00F94761B8CA975
:101BD000809328050C948E9880E090E0A0E8BFE305
:101BE000F0CEC12CD12C760131CF89E40E94AF1EFA
:101BF000882331F00E94B52469837A838B839C8388
:101C00008AE40E94AF1E882309F455CF0E94B524B0
